:020000040800F2
:1000000000A00020293A0108913A01085D2A010860
:10001000913A0108913A0108913A01080000000064
:10002000000000000000000000000000913A0108FC
:10003000913A010800000000913A01086FDD0008C4
:10004000913A0108913A0108913A0108913A010860
:10005000913A0108913A0108ED870008E987000804
:10006000913A0108913A0108913A0108913A010840
:1000700075D30008913A01088B960008913A01085F
:10008000913A0108913A0108913A0108913A010820
:10009000913A0108913A0108913A0108E587000870
:1000A000510401088D04010841040108B10401084C
:1000B000810401087104010861040108913A0108F2
:1000C000913A0108913A0108913A0108913A0108E0
:1000D000913A0108D5060108C9060108BD060108C4
:1000E0007DDD0008913A0108913A0108913A010832
:1000F000913A0108913A0108913A0108913A0108B0
:10010000000000000000000000000000913A01081B
:10011000913A0108913A0108913A0108913A01088F
:10012000913A0108913A0108913A0108913A01087F
:10013000913A0108913A0108000000000000000017
:10014000913A0108913A0108913A01080000000033
:10015000000000000000000000000000000000009F
:100160000000000000000000913A0108913A0108E7
:10017000913A0108000000000000000000000000AB
:0801800000000000913A0108A3
:100188002DE9F04F2DED028B6A4F6B4B3B60AFB002
:1001980000237B6011F028FA18B911F049FA0AF027
:1001A80019FF0AF0D1FF654A654C137843F0010343
:1001B8001370644B4FF47002C3F88820002309932E
:1001C8000A93236843F480332360236803F40033DD
:1001D8000A93099B013309930A9B1BB9099BB3F541
:1001E800A04FF2D1236813F4003318BF01230A93F8
:1001F8000A9B012B68D0534E534BF360636ABB6074
:10020800636ADFF874B1DFF87481DFF874A143F032
:1002180080736362636943F4FC032EAD6361032357
:100228008DF86A3041F6FF7325F8503D4FF0904045
:1002380029460DF08FF94FF6FF7358462946ADF859
:1002480068300DF087F9414829460DF083F9404898
:1002580029460DF07FF93F4829460DF07BF92946DC
:100268003D480DF077F9284607F02AF91A9B3B4AD2
:10027800B3FBF2F33A4A3B4913603B4B00221A6046
:100288005A603A4B5960F02186F823109A60384E2C
:1002980007221A60B368CAF8003098E80300636957
:1002A80085E8030043F4802363610823CBF8183002
:1002B8001A981BA90DF04EF9DAF8003013F0080F60
:1002C800A8F10C0829D163E02A4B12221A6063684E
:1002D800636063686360636843F480636360636852
:1002E80023F47C136360636843F4E8136360236852
:1002F80043F0807323602268114B9001FBD55A6844
:1003080022F003025A605A6842F002025A60636897
:1003180003F00C03082BFAD16DE796F89031012B06
:1003280036D8044B96F891219B6813F0805900F059
:10033800CB852DE0F800002047A80008F8330020FE
:100348000010024000ED00E00005FA050008004832
:10035800000C0048001000480014004840420F00FC
:10036800542200203F1901005822002010E000E02C
:100378009C27002000200240000400484C8301080C
:100388003C270020BD4B002283F891210BF078F820
:1003980064200DF0DEFCBA4800214FF48C7215F091
:1003A80008FEE369B74843F00703E361A36943F430
:1003B800E123A361636943F4C023636100F5887492
:1003C800837B416890F80FE003F00702DB0801EB3C
:1003D80083039200196A4FF00F0C0EFA02FE0CFA12
:1003E80002F221EA02021A62196A10304EEA010288
:1003F800A0421A62E4D10022A349002353540132D7
:10040800112AF9D1A14AFF2199540133072BF9D1B7
:100418009F4BDAF800409F4A1A609F4800213C220F
:1004280015F0C7FDC4F3801905234FF0000E9B4A51
:1004380099481EF802100C2202FB0EF21154B9F171
:10044800000F07D11E3901299FBFFF2103F1FF3398
:100458001154DBB20EF1010EBEF1050FE7D1904A3F
:1004680096F805B013708F4B8F4983F800B08F4B07
:100478007B62C0330B608E4B8E4A03EBCB03A10625
:100488005B7848BF0123936200238B4A40F2DC511A
:1004980022F813100133082BF7D113A800211C22CE
:1004A80015F087FD14F4007A1DBF844B199503934A
:1004B800CDF80CA0BBF10E0F03D00BF0EF03082B07
:1004C80002D101238DF85E30022005F017FE18B125
:1004D8004088003018BF0120C4F340038DF8523023
:1004E800C4F340338DF84C30C4F3C03300F001003E
:1004F8008DF84F3014F400638DF851008DF8549046
:1005080007D096F8843103F1FF3EDEF1000343EB98
:100518000E038DF85030C4F300438DF85530BB6A94
:10052800B6F84801ADF862001AF1000A18BF4FF09A
:10053800010A003318BF01238DF85730C4F3005364
:100548008DF85830B6F84A31ADF85C30B6F8563107
:10055800ADF85A3004F00101C4F38043C4F3C0027B
:10056800E40448BF45488DF85330B6F8543144BFC9
:10057800B0F85001ADF86200B3F5FA7FADF860301D
:1005880084BF0023ADF862304D4896F8CC3187F827
:100598002C30002387F82D3043709DF85E308DF89D
:1005A8004D10002B8DF84E208DF856A00CBF00235F
:1005B800022301B902B1013308EB83084FF00009A7
:1005C800D8F81430A3F1020A203304933AF8023F12
:1005D8004FF6FF72934200F0B1819DF85110DAB2E4
:1005E8001B0ADEB279B12748364C00EB021041688D
:1005F800A14208D10189B1F5806F00F09B81B1F566
:10060800006F00F097819DF8541031B111011D4819
:1006180040582D49884200F08D819DF8551079B1D8
:100628001101184C6018645828498C4200F08281E6
:100638004168B1F1904F03D1817B082900F07A819C
:100648009DF8521051B10F4800EB02104168B1F10A
:10065800904F03D10189102900F06C819DF84F104B
:10066800B1B30848174C00EB02104168A1422FD1E2
:100678000189042900F05E812AE000BF9C27002040
:100688007022002098A5010804010020150100200F
:10069800CC12002082290020D01200200AAD0108C7
:1006A800B1100020B809002004240020B027002041
:1006B800F0AA0108F80000201A1000204083010861
:1006C800250100200004004800040040002C0140DF
:1006D8009DF8501051B1BE4800EB02104168B1F1CD
:1006E800904F03D10189202900F02481199C7CB105
:1006F800B74F216807EB02177868884208D1398913
:10070800A088884200F01681E088884200F01281B3
:10071800022B02D19DF84C3003E0012B04D19DF847
:100728004D30002B00F006819DF85710A84B17019B
:1007380059B19DF85E1041B9A2F10E01012904D802
:10074800D959A448814208BF04269DF85810DC19DD
:1007580031B19DF85E1019B9043A032A40F2D280EB
:10076800012E49D1DFF878820693D919FF2291F832
:100778000DE088F8742088F875204868C8F8844027
:1007880001F108020989ADF868104FF0000B022149
:100798008DF86B1088F878B01AA98DF86AE0059280
:1007A80088F830B0C8F834B0C8F838B0C8F83CB0E9
:1007B800C8F870B088F876B088F877B00CF0CAFE40
:1007C800069B059AD85991785A4609F0A1F920460E
:1007D800594632460FF0BEFE7F4BC8F888307F4B33
:1007E800C8F88C30C8F890B0204608F1880108F1A4
:1007F8008C020FF005FF9DE0022E4BD15FFA89F3C2
:100808001C2101FB03FC764BCDF81CC003EB0C0B41
:1008180001238BF8783006936D4B8BF87990D919B2
:100828004FF0000891F80DE048688BF87A8001F1E4
:1008380008020989ADF868108BF882801AA9CBF8EC
:1008480084408DF86AE005928DF86B600CF082FEAA
:100858005F4B059AD8599178424609F059F9069B99
:1008680020461A4641460FF075FE5D4BDDF81CC068
:100878005C4ACBF8882003EB0C015B4ACBF88C2050
:100888008831CBF8908020460A1D0FF0B9FE09F197
:1008980001094FE0032E33D19DF85330504E534F8A
:1008A8003BB196F82E80204608214FF6FF720023B0
:1008B8001AE0BDF8602096F82E80BDF86230B2F5D7
:1008C800FA7F0BD94A49B1FBF2F22046082192B2CD
:1008D8000CF069FE474B47F828000AE04649B1FB8F
:1008E800F2F22046012192B20CF05DFE434B47F82C
:1008F8002800C36096F82E30013386F82E3019E0B0
:10090800042E17D1364EBDF85A2096F82D703A4B62
:1009180093FBF2F22046BDF85C30012192B20CF054
:1009280042FE96F82D3006EB87070133C7F85801C9
:1009380086F82D30049B9A457FF448AE284F304BFB
:1009480097F82D2087F878212E4A1678A6F11702F5
:100958000024022A1C709E461BD87B6A2344D3EDD0
:10096800007AF5EE407AF1EE10FA03D1BB6A002B5B
:1009780050D126E0244A04EB020C0FCB8CE80F0080
:100988009EF8003010340133C02C8EF80030E4D1CA
:10099800ECE71E4B13F836808EF8008003EBC60395
:1009A800D3F80490B9F1000FE0D04445DEDA164AD6
:1009B800230103EB020C4B440FCB01348CE80F00EE
:1009C800F3E7134B1A6812F4805F984648D141E068
:1009D80098A5010800400140BDD100089DD200083B
:1009E800F800002001D3000895D100080425002054
:1009F80000127A00BDD2000840420F00ADD20008B4
:100A080000250020B8090020F4080020F0AA0108F9
:100A18003C2700202B4B2C4A13F83600107003EBB0
:100A2800C6035C68002CCCD000238342C9DAC3EB30
:100A3800C3016218DFF89C80D2F8009041F8089052
:100A480001EB080C9188ACF8041092798CF8062018
:100A58000133EAE706F0EF03082B1C4B20D121E015
:100A68009EF80020012AF5D9194B03EB0212103227
:100A780010339342EED053ED047AB6EE007A67EE67
:100A8800877A43ED047A53ED057A67EE877A43ED6A
:100A9800057A53ED037A67EE877A43ED037AE7E741
:100AA8000E2E08D11A7842F010021A70182E13D19F
:100AB8000DF0C2FB10E01A7822F010021A70192EFD
:100AC800F5E700BFA894010890230020201100201A
:100AD800FC080020912300200DF092FBD8F800308C
:100AE800AD4CAE4E580358BFAD4BAE485CBF01226B
:100AF8001A70AD4A137843F0040313704FF400439F
:100B0800ADF8683063694FF0020943F400234FF0F1
:100B1800010B8DF86B9029468DF86AB063610CF073
:100B280019FDA24BA24A1A6000200DF033F9E369BF
:100B380043F48043E361236943F480432361636999
:100B480043F480236361736A23F470037362736AE6
:100B580043F4A0037362736A23F070637362736A69
:100B680043F0A0637362736A23F070437362736A1D
:100B780043F0A04373624FF460431A938DF86C906E
:100B880003234FF00009304629464FF4805A8DF868
:100B98006D3004938DF86E908DF86F9006F0FEFD21
:100BA800049B8DF86D3030462946CDF868A08DF845
:100BB8006CB08DF86E908DF86F9006F0EFFD23699C
:100BC80043F480432361236923F480432361794BF1
:100BD8009A8822F480521204120C9A809A8892B24F
:100BE80042EA0A029A801A8802F4415242F4457293
:100BF80042F003021A809A8822F470621204120CDE
:100C080042F4E0629A809A8B22F400621204120C79
:100C18009A8307221A821A8892B242F040021A80F6
:100C2800C6F818A0D8F8003003F41073B3F5107F95
:100C380000F09E80604B614E1E606369DFF85C9136
:100C480043F480236361E36943F40013E361236B96
:100C580023F010032363236B43F010032363D9F8B5
:100C6800203023F07063C9F82030D9F8203043F0E1
:100C78008063C9F82030D9F8203023F07043C9F8D0
:100C88002030D9F8203043F08043C9F820304FF0A5
:100C980000084FF0020C4022484629464FF0030B4B
:100CA8008DF86CC0CDF818C01A928DF86E808DF84A
:100CB8006F808DF86DB006F071FD80224846294698
:100CC8001A9206F06BFD3268DFF8089122F00102F3
:100CD800326031683A4A0A4032603A4A32613268D0
:100CE80042F001023260C6F80880C6F80C80C6F8E7
:100CF8000880B26842F40042B260326832607268BA
:100D080022F0784222F400427260326842F0010216
:100D18003260D9F800502C4E05F400434FF0100A09
:100D28000493524605F4006330464146059315F096
:100D380040F94FF6FF72DDF818C00E9215F0020563
:100D48008DF83DC08DF83E808DF83F808DF83CB021
:100D580042D02EA94FF0904041F880AD06F01EFD1C
:100D680001250723357086F80180F370B57033E0EC
:100D780016490A784B4616481E561F2E02BFFF26F4
:100D88001E5402F1FF3203F10C0308BFD2B23C2B10
:100D9800F1D10A704EE700BF00100240000400487D
:100DA800200E002000080048F833002008340020F6
:100DB8005DD9000800380040EC0F002000540040C6
:100DC800FFE0CF007A25E0005D130020B11000207D
:100DD800D01200203C270020049B7BB12EA90423BD
:100DE80041F8803D924806F0D9FC0C233371072363
:100DF800F371012375711D44B371EDB2059B83B185
:100E08002EA9202341F8803D4FF0904006F0C6FC03
:100E1800022333730723F373012375731D44B373DC
:100E2800EDB2E36A834823F4F873E362E36A43F4B8
:100E3800D873E362636943F0805343F0020363614C
:100E480006F0EDF91AA806F0BFF97B4B1A937B4B15
:100E58001B93012D4FF0000394BF1A4680221F9266
:100E68004FF48072734C20924FF4806221922022BA
:100E7800204622921AA94FF400521C931E932392E3
:100E88002493ADF8745006F0ACF9236843F00103DD
:100E980023606B4CA36823F04053A360A36843F01E
:100EA8008053A3600A200CF054FFA36823F080430A
:100EB800A360A368A360A36843F00043A360A2688B
:100EC8005F4B002A31DAFAE7531E092B3FF660AA76
:100ED800D8F858002860294658460CF03BFB4FF4D8
:100EE8000063CBF818303C200CF033FF96F89131B2
:100EF8009945BFF647AADFF838B108224FF40063D6
:100F0800CBF8182078200492ABF8283003930CF023
:100F180015FF049A039BABF828207820CBF81830EB
:100F28000CF00CFF09F10109E0E79A68454922F045
:100F380040529A609A6842F000529A608868424A21
:100F4800024042F468328A60D968404A0A4042F452
:100F58000052DA601A6B013D22F00F0215431D633F
:100F68000021012372189078002800F084805C1C0E
:100F7800042B16F801E0D278DFF8C4C0E4B20ED82A
:100F880003EB4303DCF830505B001F20984025EA50
:100F980000000EFA03F30343CCF8303031E0092B9C
:100FA8000ED80620053B4343DCF834501F209840F8
:100FB80025EA00000EFA03F30343CCF8343020E0AE
:100FC8000E2B4FF006050ED8A3F10A006843DCF893
:100FD80038801F23834028EA03050EFA00F32B43C9
:100FE800CCF838300DE00F3B05FB03F0DCF83C8013
:100FF8001F23834028EA03050EFA00F32B43CCF89D
:101008003C30BEF1090F0E4822D983698569AEF1DB
:101018000A0303EB43034FF0070E0EFA03FE25EA1B
:101028000E05856185699A402A43826122E000BFE6
:101038000004004808040240400100506E130020DC
:101048000001005000030050E010FCFF07C0FFFD46
:10105800436945690EF1FF3303EB43034FF0380E44
:101068000EFA03FE25EA0E054561456903339A40E9
:101078002A4342612346043110297FF473AFBC4BE5
:101088009A6842F001029A601A461168B84BC9077B
:10109800FBD5DA68B74E22F00202DA60DA6842F06D
:1010A8000202DA60DA6842F00102DA609A6842F015
:1010B80004029A60B6F85C31002B41F08C80B6F9D6
:1010C8005E21002A41F08780B6F96021002A41F0AC
:1010D8008280D9F800309B031FD5C8200CF039FE58
:1010E800AE2009F09AFA08B109F09CFAA24C87F8E8
:1010F8007901C8200CF02DFEA04BC7F87C310021E7
:101108000C22204614F055FF0223E37007F0E8FD97
:101118000CF0F8FD9A4B0344A3609A4BDFF8A082C9
:101128001B689948B3F85630049300210C22B6F88E
:10113800645196F863B196F86B41B6F80C9096F83E
:101148000FA014F036FF00211422404614F031FF9E
:101158008E4B069300221A708D4AC7F8802105929B
:101168000FF055F9069B059A06461946002836D011
:10117800884BC8F80030884BC8F80430874BC8F84B
:101188000C30B5F5807F864BC8F81030854B01D1FF
:10119800002016E0BB2D01D9012012E0612D01D9F4
:1011A80002200EE0292D01D903200AE0132D01D9D0
:1011B800042006E0092D01D9052002E0002DE7D022
:1011C8000620187004230B707748784902230370AF
:1011D8000B6843F001030B60804659460EE003207C
:1011E8000CF034FE40E24FF0010B0BFA01F040F234
:1011F800B233034043B1012960D900216C48002370
:1012080009290370F9D8EEE710F04D0FF3D00691D5
:10121800C7F8802105920FF0FAF8059A0699002878
:10122800E9D0062168200A460DEB00030CF0A8FA65
:101238009DF86D1001EA0B029DF86B1001EA0B0195
:1012480001FA0BF343EA82019DF8692002EA0B03D5
:101258000B430AD05BB25B4501D1002302E0022BAD
:101268000ED1012387F8843111E00EAB68200C21E0
:101278005A460CF085FA9DF8383013F00F0303D165
:1012880005200CF0E3FD02E0042BEAD1E5E73E4B34
:10129800484A1A60484A5A6097F88421002A0CBFC5
:1012A8006F226E221A72424B04221A703F4A03239D
:1012B80088F80130136843F0020313600A200CF029
:1012C80048FD7720A02101220EAB0CF059FA10B985
:1012D8004FF0000B90E01E21012277200CF0CCFA91
:1012E8004FF42F600CF02AFD4FF0000BABF16001BA
:1012F8004FF00008C9B202221AAB77208DF8688037
:101308008DF869800CF03CFA9DF869309DF86820EA
:1013180043EA0222294B03F5C3712BF801200BF194
:10132800020BBBF1100FE1D1B3F8942102F00F0CBE
:1013380002F47F42A3F89421012043464146DFF896
:101348007C8021F0010EC644BEF886E1BEF1000F94
:1013580018BF002011F0010F06D05FFA8EFE83EA55
:101368000E034FF0080E2DE083EA1E23F9E700BFB5
:10137800000100509C2700209820002024290020EC
:10138800404B4C002C10002034250020A20E0020D9
:1013980064830108F1020108890101086901010853
:1013A80090C1793D00000020840000201C1100201D
:1013B8002034002069030108C9010108F800002051
:1013C800B833002013F4004F18BF83F4C053BEF1A4
:1013D800010E4FEA4303F5D101311029AFD16E490F
:1013E80042EA0C02A1F8942100287FF471AFC3F3FC
:1013F80003339C4536D06BE7DFF89C8198F896312B
:10140800002B40F0D78614200CF0A3FC08F29713A9
:101418007620D02101220CF0B3F998F89731582B97
:101428003AD108F5CC738821182276200CF0A8F957
:1014380031227620F4210CF01FFA012388F8963126
:10144800564B574A9A60574A5A6045F6D8125A80FE
:10145800554ADA60554A1A61554AA3F800B05A61EC
:1014680000F0A8BE4D4A42F2107313805380514BCE
:101478005360514B9360514BD360514B1361514BA7
:101488005361B346002EB7D003234F4A93704F4A97
:10149800136843F0040313604C4B1A6812F0020FF0
:1014A800984602D04A4B1B6898474A4ABAF1000F3F
:1014B80026D015F0FF0F0BD1D8F8003013F0020F2B
:1014C8004FF07D0140F2712308BF4FF4FA7302E038
:1014D8004FF47A731946994505DBB9F57A6FA8BFB9
:1014E8004FF47A6900E099464B1E4B44B3FBF1F385
:1014F800013BDBB203FB011187F8B431116004E052
:10150800254BC2F8009083F8B4A1334B1B68984769
:10151800324D0023022C2B7004D0032C1DD0002C3C
:1015280040F04F862EAB002203F8502D2C4AC7F806
:10153800B8211E200A2101220CF022F968B19DF879
:101548006830482B09D1274B274A1A60274A5A6026
:101558001EB104232B7002234EE02EAB4FF000097E
:1015680003F8509D0C20494601220CF009F9002887
:1015780000F059869DF86830482B0AD1194B1C4A4F
:101588001A601C4A5A603046002E00F04C8603232D
:1015980032E0484600F047BEF80000205C06002014
:1015A800B99D0008BB9D00088B9F000829A0000872
:1015B800BB9B000817010108590101080D0101082A
:1015C800490101084DFF0008840000201C1100207B
:1015D80034250020FC2F0020B833002023340020BD
:1015E8007C8301083C13002099A10008959F0008FE
:1015F80001A1000875A00008BE4AD370D8F80030D1
:1016080043F00803C8F80030BB4B93F858210AB1DF
:10161800BA490A7093F859210AB1B9490A7093F87E
:101628005A3103B12B70D8F80030B64913F0080FBF
:1016380000F0C385BDF91000DFEDB36A642290FBAA
:10164800F2F302FB130212B207EE902AB8EEE77A21
:1016580007EE903AF8EEE77AE7EE267AB2EE047AE9
:1016680067EE877AC1ED007AA84B1A7842F0020239
:101678001A70A74A082191610A240493A44DAB8AE1
:101688009BB283F00803AB8219200CF062FB0120A7
:101698000CF080FB19200CF05CFB013C00200CF0E6
:1016A80079FB14F0FF04E9D108239A4CAB61236855
:1016B8001F0705D5984B1B689847984B01221A704D
:1016C800974B9FED988A1B68974D1B7B00EE103A4D
:1016D800B8EEC00A20EE080A09F07EFB2B8807EE58
:1016E800903AF8EEE77A27EE800A14F071FE8F4BF5
:1016F8009FED8F7A18802B888E4D07EE903AF8EE82
:10170800E77A8D4BC7EE277A2846FF211A229FEDEC
:101718008B7AC7EE877A9FED8A7AC3ED007A894B78
:10172800D3ED047A884B67EE887A67EE877AC3ED43
:10173800007A14F03EFC00222A702268834B0121B3
:1017480012F0020F18BF697019701FBF03211970BA
:101758000221A970560748BF1978284641BF4D1C79
:101768001D700325455412F00A0F0CD01A78042175
:101778008154511CC9B205254554D11C0232D2B23C
:10178800197006218154724E31688D0641BF1A784E
:10179800551C1D70072548BF85540A0608D51A78B8
:1017A80009258554951C0132D2B21D700A2585542D
:1017B800514F7D79082D01D00E2D08D11A7802F1EC
:1017C800010E83F800E04FF00B0E00F802E01A78E3
:1017D80011F4803F4FF00C0C00F802C002F1010E2A
:1017E8001CBFDFF868C102325FFA8EFE83F800E0A2
:1017F8001FBF8CF800204F4A4FF00E0C02F80EC0A5
:101808004A0741BF1A7802F1010E83F800E04FF051
:10181800100E48BF00F802E01A7802F1010E5FFAD4
:101828008EFE4FF0120C11F4806F83F800E000F880
:1018380002C00ED097F810C2BCF1000F09D0DFF833
:101848000CC102328CF800203A4A4FF0130C02F80F
:101858000EC01A7811F4007F4FF0140C00F802C083
:1018680002F1010E1CBFDFF8E4C002325FFA8EFEFF
:1018780083F800E01FBF8CF800202E4A4FF0150CAB
:1018880002F80EC0182D13D11A784FF0160E00F872
:1018980002E002F1010E5FFA8EFE4FF0170C00F81D
:1018A8000EC002F1030E0232D2B283F800E0855472
:1018B8000A0341BF1A78511C1970192348BF835471
:1018C80000219822234814F074FB05F09CFB224B5E
:1018D800224A23491A6000234B800B7121490A6070
:1018E800B7F8962190B2204921F813000133122B42
:1018F800F9D13BE0840000209C270020A20E0020A4
:1019080020340020BC2100208988883CF83300203E
:10191800000400481C1100203C1300205C13002028
:101928001024002035FA8E3C2000002034240020AA
:101938000AE81C41F90F00207407002000401C46EB
:10194800BD378635B83300200C240020F80F00205E
:101958003C27002030120020040F002024290020FA
:10196800F0330020B83200207827002033681B07A6
:1019780040F1D48097F89011062900F2C980DFE879
:1019880001F00404305A718D8D008B4A8B4B136023
:1019980001298B4D8B488C4A08D14FF0030E85F8EE
:1019A80000E00725117005700C2206E0022129705D
:1019B800032101700021117007221A70834B844A99
:1019C8001A60402004F074FC002800F0A180012374
:1019D8004FF0000A90F900007E4A8DE80804402183
:1019E8003DE007EE902ADFED7C6AB8EEE77ADFED9E
:1019F8007B7AE7EE267A0023FCEEE77A784A17EE40
:101A0800901A42F823100133122BF7D16F4A754907
:101A180011606A4A4020137004F04AFC002877D00D
:101A280001234FF0070990F900006F4A8DE808027A
:101A380040216E4B66E0654B6D4A1A605F4B102281
:101A480040201A7004F034FC002861D001234FF0C4
:101A5800000890F90000674A8DE8080140214FF41A
:101A6800E1334FE0594B644A1A60544B0822402036
:101A78001A7004F01DFC00284AD001234FF0000C16
:101A880090F900005D4A8DE8081040214FF4E133D9
:101A980004F0E4FA5A4BC3F8BC0135E0474ADFF8D2
:101AA8008CC1DFF88CE1574D57480C231370062979
:101AB8004FF000028CF800208EF800202A7009D020
:101AC8001B220270514A1370514B05221A704FF4B1
:101AD800E13506E0212202704C4A4E4D13704C4B02
:101AE80019703A4B4C4A1A60402004F0E1FB78B177
:101AF80001234FF0000E494A90F9000040218DE87B
:101B080008402B4604F0AAFA003018BF012028B973
:101B1800082009F025FA2D4B00221A603368274A5D
:101B280013F4804F1FBF0821117028493C4818BF83
:101B3800086042F20101194003F0010003F4005566
:101B480051B12249DFF8ECE0C1F800E00DB10821FD
:101B5800117008B10C21117011781806A1F1040157
:101B6800517040F1A48026482E4DDFF8CC80C0F893
:101B7800C0814FF000094946152200F5E270DFF8F0
:101B8800BCA085F80190C5F80490C5F8089014F039
:101B980010FAA8F105034846CAF8003006F02CFBF5
:101BA800214B02201B68EB6004F082FB002847D120
:101BB800802009F0D5F972E03C0600204C33002063
:101BC8003806002040060020C43100204833002099
:101BD8009121010889220108CDCCCC3F0000B0C476
:101BE80058320020DD21010891230108A086010058
:101BF800C921010821230108B5210108D5220108BE
:101C0800F8000020081200202B1200204333002087
:101C18002C12002090D00300E96E0008FD6E000829
:101C2800112201089007002060270020443300207B
:101C3800091200201D22010882290020B007002077
:101C480090F805E06B78CC490C2202FB031252781D
:101C5800724504D00133DBB2042BF4D900236B7036
:101C6800DAF800306A781B7890F90000002B4FF002
:101C78000C0303FB021314BF4FF0030E4FF0010EC9
:101C880000225B78CDF800E00192022104F0E6F929
:101C9800BA4B186000288BD0012006F0ADFAB84B7B
:101CA8001868B84B00F5C5721A6006F053FB336824
:101CB80013F4007F0DF168085DD0DFF81493039BDF
:101CC800C9F80030B04BB1485A6942F480225A61D1
:101CD8009A6942F001029A61039B1B88ADF8303083
:101CE800012502230CA98DF833308DF832500BF002
:101CF80031FCD9F80030A5485B88ADF830304FF09A
:101D0800000A0CA98DF832A00BF024FCD9F8003099
:101D18002846197A05F0FCFAD9F80030586805F019
:101D280047FAD9F800305B681A93404610238DF8BB
:101D38006D308DF86CA08DF86E500FF08DF9D9F8D4
:101D480000305B7A8DF838300EA803238DF83930CF
:101D58008DF83AA08DF83B500FF060F98C4B8D4A06
:101D68001B683C3B1360236843F0100323608A4BD5
:101D78004FF0FF321A60894A894B1360894A8A4DAD
:101D88008033136033680024D9032C7040F1AF808E
:101D98000EF012FDDFF83CC2DFF8ECA1CDF818C058
:101DA80040F22A334FF001091A466046214605934E
:101DB80085F8009014F0FDF8DAF814207B4D4FF008
:101DC800904042F40032CAF81420426A22F00F020E
:101DD8004262426A032142F0060242624FF4807B6B
:101DE80002228DF835100CA98DF8342003928DF855
:101DF8003640CDF830B08DF8379005F0CFFCDAF8E2
:101E08001810039A41F40061CAF81810298821F4BF
:101E18005C710904090C29801D21E96228462A857C
:101E28000EA92C866022C5F814900E92ADF83E409B
:101E38001094ADF84440ADF84640ADF84840ADF8D0
:101E48004A40ADF83C9005F0FDFAAA6942F0080254
:101E5800AA616A6C42F400426A64DAF8142042EA21
:101E68000902CAF81420AAF6E47A504605F0D7F910
:101E7800404605F0A9F9059B4D4AADF8743080231A
:101E88001A92DDF818C01F9310224FF400535046E1
:101E980041462393CDF86CC01C921E94CDF880B0B7
:101EA80021942294249405F09CF9EB6843F4007380
:101EB800EB60DAF8003043F00203CAF800300BA8F0
:101EC8000C238DF82C308DF82D908DF82E408DF840
:101ED8002F900FF0A3F8374B1A68374B43F824209C
:101EE8000134202CF7D10BF057FA0BF055FA336870
:101EF8005A0540F18880314C314BD4F80495C3F829
:101F08000090042004F0D4F90421C4F8080504F072
:101F1800ABF92C4B84F80C050820C3F8009004F0AA
:101F2800C7F90821C4F8100504F09EF9264D84F875
:101F38001405002128462C2214F03BF88E236B70E0
:101F48004FF07C0BE0234FF07D0AEB7085F800B072
:101F580085F82BA01D4D2C220021284614F029F8C5
:101F68008A236B701020A023EB7085F800B085F8E9
:101F78002BA0C4F818952FE018840108942000209D
:101F88002C100020600F00200010024000040048C0
:101F980060270020880700204C100020B410002083
:101FA800BC290020D8200020210E0020002C014050
:101FB800342C014094830108220E0020F8000020F0
:101FC8001011002068110020381100206D11002028
:101FD8008C070020D102002004F06AF91021C4F80F
:101FE8001C0504F041F984F820052020C4F8249544
:101FF80004F05EF92021C4F8280504F035F984F8C6
:102008002C0506F06DFD8B4A138823F040031B0452
:102018001B0C1380138823F038031B041B0C13803C
:1020280013889BB243F04003138000249F2332207F
:102038008DF838308DF839408DF83A408DF83B40AE
:102048000BF087FE8DF869407B4C4FF480550422D5
:10205800258540460EA90EF0ABFFA5619DF86A20C4
:102068009DF86930120242EA03429DF86B301A4328
:10207800724B9A42724B17D008D872498A420CD0D8
:1020880001F51A4102318A4209D01CE06E498A42A0
:1020980005D001318A4207D015E0202200E08022D5
:1020A8001A804FF4807202E04FF480721A805A80CE
:1020B8009A88198812029A604A43DA60634A0121B1
:1020C80082F82D1504E000221A805A809A60DA609E
:1020D800DC68FCB1240CA1464FF0000AA24512DAD4
:1020E8000AEB04056D1028044146102208F046FA50
:1020F800002358F82320013269D10133042BF8D189
:10210800A9462C46EAE706F003FB504B4FEA094282
:10211800C3F8302533684E4A13F4002318BF01234F
:1021280013700BF0EFFD4B4B18607B79052B02BF4A
:10213800494B4FF4C8721A80484B4FF47A721A8090
:10214800474BC8221A80474A137843F00803137094
:10215800454A137823F002031370326840F60203ED
:1021680013406BB1414B42491960424B032119702E
:10217800414B01211970414900230B8040490B80D4
:10218800930341BF3F4B04221A71DA7844BF42F0EF
:102198000102DA70BB6833603B4B01221A70049B62
:1021A800049A1B7863F07F0313702FB0BDEC028B89
:1021B800BDE8F08F0423FFF768B900230B60FFF731
:1021C80053BA012C7FF620AA1C46FFF7A1B905F1E6
:1021D800010A254695E71BB207EE903ADFED2B6A18
:1021E800B6F95E312A4AF8EEE77A07EE103A67EE5A
:1021F800A67AB6F96031CDED1A7A07EE903AB8EEC4
:10220800C77AF8EEE77A002127EE267A67EEA67AF3
:1022180011701AA81F498DED1B7ACDED1C7A08F0B4
:10222800E3FDFEF756BF012C7FF6EEA900242870C7
:10223800FFF778B9003800400004004818BA2000B9
:1022480010000020152020001740EF00F8000020A3
:10225800F82F002034080020160F00201A34002020
:1022680018340020201100202234002008110020FA
:10227800162900206C1100207D000020C00E0020CF
:10228800C20E002098200020200E002035FA8E3C37
:1022980054000020141300202DE9F04FC14BB3F96E
:1022A8000610C14B2DED028B1F687A8985B09142CB
:1022B80001930EDBB1F5FA6FFC79BDBF8B1A63434E
:1022C800A2F5FA64C4F16404BCBF93FBF4F464346B
:1022D80000E06424B54BB64AB3F896B193F962317D
:1022E800126802929BB2154603930022AD4B33F954
:1022F80012E0CBEB0E0303F2F31640F2E63086420F
:102308004FEA420C03D8002BB8BF5B4201E04FF400
:10231800FA73022A2ED0029E96F811611EB1B342BA
:10232800CCBF9B1B0023A34E6FF0630A642093FB72
:10233800F0F836F818900AFB083A08F1010836F95F
:1023480018600FFA89F8C8EB060606FB0AF696FB32
:10235800F0F699484E4420F80C60BE18642036798F
:102368007343964E93FBF6F364339BB2634393FB3C
:10237800F0F02DE0029890F812611EB1B342CCBF84
:102388009B1B0023DFF860926FF06308642093FBC7
:10239800F0F008FB003A39F910600130002B39F9E8
:1023A8001000A0EB060000FB0AFABDF80C009AFB2F
:1023B800F8FAC6EB0A0A1AFB00FA7F48A0F804A04C
:1023C800B879B8BF5B4243437C4893FBF0F0643074
:1023D8006B787B4E4FF06408434393FBF8F3B35498
:1023E800784EEB7A434393FBF8F3B3546B7D724E0C
:1023F8005843754B90FBF8F0022A9854734B0ED152
:10240800DE4583F802800DDB684CB4F898219142D0
:1024180014DBB1F5FA6FA8BF4FF4FA610FE0DE459F
:102428009C5404DA36F80C305B4226F80C30013242
:10243800032A05F101057FF459AFE5E71146DFF8F6
:10244800BCE15D4D891A4FF47A736FF06307594305
:10245800C2F5FA626423B1FBF2F191FBF3F23EF8A4
:10246800120007FB0211013207B23EF91220D21BFB
:10247800514391FBF3F30344F380554B1B885F06EC
:1024880035D5544B544A1B881288DFED547A9B1A71
:102498001BB208EE103AB8EEC88A28EE278AB0EECA
:1024A800480A08F099FCF0EE408AB0EE480A08F0B5
:1024B80030FCB5F9023006EE903AB5F90030F8EE86
:1024C800E66A07EE903A20EE667AF8EEE77AA7EE2B
:1024D800A87A67EE807ABDEEC77AE6EEA87A17EE9C
:1024E800103AFDEEE77A2B8017EE903A6B803C4D60
:1024F8002B68980740F1A1803A4B3B4F1A687B69DB
:1025080045F20721D31A8B4240F397807A6105F090
:1025180005FB364BDFF8E8901A78032A9846B9F895
:10252800003022D10A2B2AD90023282088F800302D
:102538000BF00FFC05F0F2FA2D4B188805F0D8FACD
:102548002C4B1A68D37890FBF3F0013008282A4BFB
:10255800A8BF08201870537980B213FB00F33B839F
:10256800137913FB00F0788309E00A2B07D80323BB
:10257800214A88F80030002313703B837B8398F846
:1025880000301A4A012B3DD002D3022B4CD054E024
:102598003A8BB9F800309A424FDD012388F80030B1
:1025A80040E000BF78270020541000209C2700201E
:1025B8002C100020D2100020001100200CFEFFFF7C
:1025C80088240020B60E00208B240020C021002083
:1025D800E0110020F81000205A0F002035FA8E3C38
:1025E8003C27002000340020A80E00206C11002099
:1025F80076130020081100207D000020BA1000206A
:102608000C110020B9F800107B8B8B4202DD0223ED
:1026180013700FE0A24B1B8B0133994202DD00239C
:1026280013700AE0082006E07B8BB9F8002001331C
:102638009A42B2DC07200BF0CBFB2D68290575D533
:10264800984B974F1A68FB69C3EB020845F20723BA
:1026580098456BDDB6F90630FA61A3F57A7B924BA3
:10266800B4F85201D3F80090904E99F80A30012B33
:102678004FF47A7198FBF1F803D040D3022B1FD0A6
:102688003FE08B4B386A5A7B8A4B33F812204FF065
:10269800080E92B290FBFEF3C01A8318BA843B620C
:1026A80040F6E44293FBFEF39BB25343B9F808208B
:1026B800C2EB13334B43B9F9062093FBF2F31FE047
:1026C8007D4BB9F808A01B78C6F800A05A0718D5A2
:1026D8000EF071FF20B915F0100F18BF4FF0000B66
:1026E800B9F906200BFB0BF1322391FBF3F35B44A2
:1026F8005A434FF47A7392FBF3F3534400E00023F8
:102708003360D7E90A0133686C4A03FB08F84FF4D1
:102718007A7398FBF3F810EB080041EBE87100239B
:10272800C7E90A0110F0B0F9654B1860654E3368C7
:10273800DB0427D52F0622D5634B1B789D071ED5B2
:10274800624B187804281AD90022614BD718052142
:10275800951C4FF00A0E122AD154E9B287F801E00D
:1027680004D0B0EB510F2A46EFD800E014215A18D4
:10277800322002F8010CFF225A540F2000E00A20F0
:102788000BF026FB534D2A68002A50D0524B534F6A
:10279800186839688142984649D8514BDFF84C91FE
:1027A80019785268E1B94FF0010A83F800A0B9F826
:1027B8000030D35C23B350460BF0ECFA494B83F856
:1027C80000A00FF025FFB9F80030CBB92B681B78B3
:1027D800053B534514D80BF095FA434B18600FE0AE
:1027E8004FF0000A83F800A0B9F80030D35C3BB181
:1027F80050460BF0CFFA3B4B83F800A00FF008FFD0
:102808002A68B9F8003052683848D25CFE2A01D1EB
:1028180000230BE0FF2A02D10BF0C2FA07E0D8F838
:1028280000500A2111FB02523A6001330380224D05
:102838002B78580703D52E4B08221A8570E032688A
:10284800D1075CBF43F001032B701F4B1B781F0798
:102858005EBF2B7823F001032B70D60248BF2B787C
:10286800204A44BF23F001032B70224B1B6813F04E
:10287800040F02D02049098851B92049098809B1B3
:10288800980705D41E4B1B88003318BF0123CBB310
:10289800022313702B7823F001032B7037E000BF5D
:1028A800A80E002000340020081100201411002078
:1028B8005D1300206E13002022340020407E0500A6
:1028C80018110020F40F00202011002026110020EC
:1028D800402500206C220020602700206422002070
:1028E80060220020B2330020B4310020682200208A
:1028F800000400481C11002018340020160F002086
:102908001A3400202978C90758BF022313700BF026
:10291800F9F9AF4B1B68C01A002801DB0FF078FEED
:1029280006F0DEF8AB4B1E789846002E00F0A98022
:10293800A94E3368002B00F0D78630680BF0D6FA22
:10294800002800F0D186A44BA44C18680BF0CBFAF1
:10295800092801D03F2850D14FF0000AD4F8009040
:102968009F4D5746B9F1000F05D09E4829684A4641
:1029780013F06CFB10B9AA4607B92F469A4B1035CD
:102988009D42EFD3C7B1D7F800E0DAF800C023685A
:102998001EF803501CF80300A8420DD15A1C914997
:1029A80038B92D2B05D88D4D2A602025CD54885453
:1029B80002E0CD542260EAE723680BB1574511D0F5
:1029C8008A480DF043F8574507D857F8100B0DF013
:1029D8003DF809200DF032F8F5E785480DF036F896
:1029E8004FF0000923689945A7D27E4B13F80900D8
:1029F8000DF024F809F10109F4E72368002B40F0F1
:102A08005886042840F09386764809F0F9FE00F0CD
:102A18006BBED9F80000DFF8E8A10BF067FA30B315
:102A2800DAF800000BF05FFADBF8003093F8481092
:102A38000246002933D124286AD1012283F848208C
:102A4800DBF80030DFF8B4A193F84820062AE0D17B
:102A580093F8490001F00EFF834600287BD03B68BD
:102A680098790CF03CFF3B68002283F84820614BC2
:102A780093F83530002B40F00A864C36982E00F03B
:102A880033865D4BF21892F84A100129F5D15B4F55
:102A9800F3583A605A4ABB4613609146B9E7012990
:102AA80004D14D2814BF00220222C7E7022904D10D
:102AB8003C2814BF00220322C0E703290CD1402878
:102AC8004FF0000102D983F84810B9E7587119711D
:102AD800D97198710422B1E7042906D1997983F84C
:102AE80049004A409A710522A8E70529A8D15879D2
:102AF80019798842987906D950409871481C1871FC
:102B08000B441A729CE790420CBF0622002295E7FC
:102B18002B78580794D4232ADAF800300ED10121F3
:102B280088F800102C4937480B60324902920B6331
:102B38000CF08CFF2E480CF089FF029A324B1B6870
:102B48001B78934201BF314B314A1A60314B04BFA5
:102B5800314ADA6074E7DAF8002092F849304A2BF3
:102B680000F0608100F28480332B00F0D38421D8F8
:102B7800292B00F06D8409D8252B00F02984272BF8
:102B880000F02C84232B40F0CE8550E22D2B00F052
:102B9800708407D82B2B40F0C6850CF083FE60713B
:102BA80000F070BD2F2B00F02085312B00F032850E
:102BB80000F0B9BD3E2B00F02B8144D8372B00F034
:102BC800DC842BD8352B00F0858200F0ACBD00BF2B
:102BD800B433002025340020FC240020D420002019
:102BE80008920108A4200020E8930108A8A9010878
:102BF800ADA90108A80E002030120020C011002045
:102C0800C4110020DDA90108CC120020FC9F00207F
:102C1800EFBEADDE00ED00E00400FA05392B00F050
:102C2800EA833C2B40F07F85DFF87894D9F800A040
:102C38000CF038FE8AF80000D9F8003018780BF04C
:102C480029FD00F01FBD432B00F0758406D8412BE9
:102C580040F069854FF0000900F061BC442B00F09A
:102C68000D85482B40F05F8505F090FD00F00ABD0A
:102C7800D02B00F0268368D8CA2B00F0D8801CD847
:102C88004E2B00F0198410D84C2B40F04C850CF0DA
:102C980009FE84F8CE010CF005FE84F8CF010CF093
:102CA8000BFEA4F8D00100F0EDBCC82B00F0838027
:102CB800C92B00F0278300F036BDCD2B00F00C8324
:102CC80004D8CC2B00F02E8200F02DBDCE2B00F0C6
:102CD8000C83CF2B40F027850CF0EEFD6FF4AF622C
:102CE80083189BB2C62B98BFA4F896010CF0E4FD9C
:102CF800A4F844010CF0E0FDA4F846010CF0DCFD5A
:102D0800A4F848010CF0D8FDA4F8D0010CF0CAFDD5
:102D180084F8E1010CF0C6FD0CF0C4FD84F8E20172
:102D28000CF0C0FD84F885010CF0BCFD84F892011C
:102D38000CF0B8FDDB4BD3F800900CF0BDFD00EBB8
:102D480080004000A9F8560055E3D62B00F03D82DC
:102D58000AD8D22B19D0C0F0FC82D32B25D0D42B83
:102D680000F03F8200F0DFBCEF2B41D005D8D82B14
:102D780040F0D9844FF0000AEBE0F22B00F07982A2
:102D8800FA2B00F0BB8200F0CEBC2B78590700F17B
:102D980079840CF087FD022884F8A80740F297820E
:102DA800C14B002283F8A82791E20CF085FDBF4BA8
:102DB800188000F067BC92F805904FEA5909B9F1FC
:102DC800120F03D904F0BCF900F05CBC4FF0000A04
:102DD800CA4507D20CF070FDB54B23F81A000AF16A
:102DE800010AF5E7B34B012283F8342000F04ABC0E
:102DF800DFF8B092D9F800A00CF05EFDAAF85A00EE
:102E0800D9F800900CF058FDA9F8580000F03ABC29
:102E18000CF048FD84F8D4010CF044FD84F8D3018B
:102E280000F030BC0CF048FDA08100F02BBC9D4B9D
:102E38001A681278022A824699466FD1D9F800B0EA
:102E48000CF030FD07EE900AF8EE677AB2EE048ACD
:102E5800C7EE887A0BEB8A0BCBED087AD9F800B06D
:102E68000CF020FD07EE900A9FED937AF8EE677A52
:102E78000BEB8A0BC7EE877ACBED0B7AD9F800B04B
:102E88000CF010FD07EE900A9FED8C7AF8EE677A49
:102E98000BEB8A0BC7EE877A0AF1010ABAF1030F26
:102EA800CBED0E7ACAD1BAF1070FD9F800B01CD110
:102EB8000CF0F8FC07EE900AF8EE677AC7EE887A0D
:102EC800CBED117AD9F800B00CF0ECFC07EE900AC3
:102ED800F8EE677AC7EE887ACBED127AD9F800B0A7
:102EE8000CF0E0FC8BF84C0012E00CF0DBFCD34457
:102EF8008BF80100D9F800B00CF0D4FCD3448BF85F
:102F08000B00D9F800B00CF0CDFCD3448BF81500B9
:102F18000AF1010ABAF10A0FC5D1B3E3D9F800B032
:102F28000CF0C0FCD3448BF80100D9F800B00CF0C9
:102F3800B9FCD3448BF80B00D9F800B00CF0B2FC04
:102F4800D3440AF1010ABAF10A0F8BF81500E5D14A
:102F580098E3DFF850919FED598AD9F800B00CF04A
:102F6800ABFC07EE900AF8EE677A0BEB8A0BC7EE1C
:102F7800887ACBED087AD9F800B00CF09DFC07EE02
:102F8800900AF8EE677A0BEB8A0BC7EE887ACBEDDE
:102F98000B7AD9F800B00CF08FFC07EE900AF8EE27
:102FA800677A0BEB8A0BC7EE887A0AF1010ABAF145
:102FB800030FCBED0E7ACCD1BAF1070FD9F800B0D8
:102FC8001CD10CF079FC07EE900AF8EE677AC7EE90
:102FD800887ACBED117AD9F800B00CF06DFC07EEC9
:102FE800900AF8EE677AC7EE887ACBED127AD9F8AC
:102FF80000B00CF061FC8BF84C0012E00CF05CFCAB
:10300800D3448BF80100D9F800B00CF055FCD34438
:103018008BF80B00D9F800B00CF04EFCD3448BF8B9
:1030280015000AF1010ABAF10A0FC5D12AE30CF01A
:1030380039FC132883463FF6C5AEDFF868A0DAF8F6
:1030480000900CF02FFC00231D4A0C2101FB0322E9
:10305800117A814222D10FFA8BFB09EB8B09137885
:1030680089F879300CF01EFC89F87A000CF01AFC0B
:1030780089F87B000CF016FC124B134A1A6089F889
:103088007C00124BDAF8000018600021793003F058
:103098009FF90F4B80F001001870F3E201331B2BEE
:1030A800D2D18FE62C1000209C270020580F00203A
:1030B80078270020A80E00200000C84200007A44AB
:1030C8006C880108500F0020E0280020540F0020D1
:1030D8000C0000200CF0E6FB0B2882463FF672AE8F
:1030E800CD4BD3F800900CF0DDFB03283FF66AAE19
:1030F800062303FB0A9989F8CE000CF0D3FB89F864
:10310800C9000CF0CFFB89F8CA000CF0CBFB89F89A
:10311800CB000CF0C7FB89F8CC000CF0C3FB89F896
:10312800CD00AFE25379092B7FF64CAE019BD3F863
:1031380000900CF0B7FB019B89F80000D3F80090D1
:103148000CF0B0FB89F801000CF0ACFB019B642883
:103158001B68A8BF642018710CF0A4FB019B6428AD
:103168001B68A8BF642058710CF09CFB019BFF28CA
:103178001B68A8BFFF2098710CF094FB019B642882
:10318800D3F8009028BF642089F807000CF08AFB68
:10319800019B89F80200D3F800900CF083FB019B97
:1031A80089F80300D3F800900CF086FB3B68A9F877
:1031B8000A005B790A2B40F26582984BD3F800909D
:1031C8000CF070FB89F808005CE282460CF074FB96
:1031D800934B23F81A000AF1010ABAF1080FF5D146
:1031E80050E253790F2B7FF4EDAD0CF05BFB072811
:1031F80081463FF6E7ADDFF820A2DAF800B00CF020
:103208005BFB0E2303FB09F9CB44ABF81901DAF891
:1032180000B00CF051FBCB44ABF81B01DAF800B05E
:103228000CF04AFBCB44ABF81D01DAF800B00CF007
:1032380039FBCB448BF81F01DAF800B00CF032FBF5
:10324800CB448BF82001DAF800B00CF02BFBCB4410
:103258008BF82101DAF800B00CF024FBCB44DAF843
:1032680000A08BF822010CF031FBD144C9F82301EE
:1032780008E20CF017FB0F2881463FF6A3AD0CF0CF
:1032880011FBC9EBC909A14489F8D4000CF00AFB69
:1032980089F8D5000CF006FB89F8D6000CF002FB83
:1032A80089F8D7000CF0FEFA89F8D8000CF0FAFA81
:1032B80089F8D9000CF0F6FA89F8DA000AF0BCFFB0
:1032C800E0E12B785B0700F1DD810EF0B1F907F042
:1032D80081FE07F039FFD5E12B78580700F1D2813C
:1032E800504B4FF4C8721A80CCE12B78590700F183
:1032F800C9814D4A137843F0040328E02B785A0714
:10330800E5D510E20CF0CEFA474B1A7810B142F02E
:10331800020201E022F002021A700CF0C3FA434BD9
:10332800DFF8289118700CF0D1FAC9F800000CF0F9
:10333800CDFAC9F804000CF0BFFA3D4B18800CF028
:10334800BBFA3C4B3C4A1880137843F002031370D5
:1033580098E10CF0A7FA02900CF0B8FA83460CF04A
:10336800B5FA82460CF0B2FA81460CF0A5FA0CF0D8
:10337800A3FA0CF097FA029BA3B9304B1020C3F8BC
:1033880000B0C3F804A007F0CAFD274A137843F039
:1033980001031370B9F1000F00F07481284BC3F8D2
:1033A80000906FE1102B40F06D81264BC3F800B000
:1033B800C3F804A0B9F1000F02D0214BC3F8009064
:1033C8002048214B0222011D1A7004F079FF59E1AF
:1033D800A0600CF07BFA07F0CBFD53E10CF06CFA1F
:1033E800A4F85C010CF068FAA4F85E010CF064FA29
:1033F800A4F8600146E10CF055FA84F87A010CF063
:1034080051FA84F87E010CF04DFA84F87D010CF035
:1034180049FA84F87F0135E12C100020541000206F
:10342800E2240020160F0020201100202611002081
:1034380024110020221100205A1000205C100020C6
:103448006C100020641000205C0F00202811002060
:103458000CF032FAA4F880010CF02EFAA4F88201DC
:103468000CF020FA84F884010CF026FAA4F88601FE
:1034780008E10CF017FA84F890010CF01DFAA4F892
:103488009A010CF019FAA4F896010CF015FAA4F8B0
:1034980098010CF007FADAF8003084F891015B79AA
:1034A800082B40F2EF800CF007FAA4F89C010CF00E
:1034B80003FAA4F89E01E5E092F805900323B9FB0E
:1034C800F3F9B9F10E0F3FF67DACDFF878A34FF0B2
:1034D800040BCB4580F0D6800CF0E4F98AF8A00103
:1034E8000CF0EAF940F2ED23984205DD40F6CA03F4
:1034F8009842A8BF184601E040F2EE20A0F2EE2064
:1035080019230BF1010B90FBF3F00AF1020A8AF878
:103518009F01DEE70CF0C6F984F89201B2E00CF0E6
:10352800C1F904EB090309F10109B9F1080F83F89E
:103538008801F4D1A6E00CF0B5F9C4F808B06071C0
:103548000CF0C4F907F014FD0CF0ACF984F8900104
:103558000CF0B2F9A4F85C010CF0AEF9A4F85E0125
:103568000CF0AAF9A4F860010CF0A6F9A4F88001FF
:103578000CF0A2F9A4F8820184E053794FF0070A0D
:10358800B3FBFAF2C2EBC2029A1A12F0FF0F7FF4F1
:1035980019ACB3FBFAFA0AF1FF3A5FFA8AFABAF100
:1035A800FF0F6FD00CF07EF95FFA80FB4FFA8BF0BB
:1035B80002F0A4FD814600283FF404AC80F800B076
:1035C8000CF07AF9A9F802000CF06CF989F80400FB
:1035D8000CF068F989F805000CF064F989F807001F
:1035E8000CF060F989F80600D5E7DFF8589209F180
:1035F800400A0CF061F9A9F8A0020CF053F989F817
:10360800A2020CF04FF909F1040989F89F02D1458B
:10361800EFD137E00CF046F91F2881463FF6D2ABD0
:103628003B685B79082B7FF4CDAB0CF045F909F1C9
:10363800880904EB890A00F03F00AAF802000CF0A0
:103648003BF9BAF80230800100F4FE501843AAF89A
:1036580002000CF027F9000104F829000CF022F907
:1036680014F8293000F00F00184304F829000CF072
:1036780019F98AF801000DF09FF803E05F4B012269
:1036880083F8352000200CF059F9FFF7E8B95C4BB6
:1036980098590AF022FC18B932200AF05AFBF6E7CA
:1036A8000AF088FD07F06CFC564B574ADA60FFF7C2
:1036B800E4B90C283DD00A2844D1544D54480CF0A4
:1036C800C5F92846232112F0AAFC08B1401B206046
:1036D8002368002B59D14D4823600021302212F075
:1036E80068FC98F800303BBB4A4B1B689B060FD51B
:1036F800494B42491B688A6B9A1A002A08DB474AD9
:103708001278042A82BF03F5123303F5F8738B632A
:10371800434B9B68002B6BD0424805B0BDEC028B35
:10372800BDE8F04F184703F00BFDFFF798B90C28D8
:1037380004D13D480CF08AF93C480DE07F2812D1AD
:10374800FFF7FBB80D28B8D07F2809D1013B2F4AD5
:10375800374823600021D1540CF078F9FFF7EDB811
:103768002F2B3FF6EAA8A0F12002D2B25E2A3FF63C
:10377800E4A813B920283FF4E0A85A1C2260234A81
:10378800D0540CF05BF9FFF7D8B85A1EA95C202971
:1037980001D113469DE71D4A23600021D154254BD2
:1037A800254DD3F800A0D5F800B0DFF86090584652
:1037B80012F043FC07463A464846594612F046FC82
:1037C8001E4A28B919F8073053445B785B0703D0C1
:1037D80010359542E7D306E0954204D2781CEB6891
:1037E8004844984702E016480CF030F9002372E785
:1037F80005B0BDEC028BBDE8F08F00BFA80E00201D
:103808003012002000ED00E00400FA05A42000209A
:1038180001B901081C1100200034002026110020E5
:10382800B8330020E40E0020B2A90108ADA90108B0
:10383800D9A901088C00002008920108E893010822
:10384800BDA901089C2700202DE9F04FAA4FAB4DD8
:103858003B68AB4CAB4E03F59C4320332DED028BFC
:1038680023602B88326801332B8042F20103134016
:1038780087B01BB1A44A1378013313700EF0F8FD1A
:103888003368D80405D5A14B1B68D90701D40EF0BD
:1038980047FC9F4B39681868837AD3B1013B9D4F29
:1038A800027B37F813301AB1C3F53B6308339BB278
:1038B8001BB2A3F57A73B3F57A7FA8BF4FF47A7376
:1038C80023EAE37307EE903A9FED937AF8EEE77AEE
:1038D80036E0326812043FD56268DFF824E28A1ABB
:1038E800002A39DB01F59C422032CEF804208B4AAD
:1038F800C07A57798A4A32F817209EF8087001373B
:1039080092B292FBF0F207F00F008EF808007044B4
:1039180042721A468348185C01330244102B92B253
:10392800F8D112B292FBF3F31BB2642BA8BF642345
:1039380023EAE37307EE903A9FED7B7AF8EEE77A95
:10394800C7EE877A794A9FED7A7A67EE877AFCEE36
:10395800E77A17EE903A13803368DF0540F19280DA
:10396800744B994204D92B7913B9644B01221A710B
:10397800714AB5F900E01778604BBEF1140FC7F330
:103988008002CCBF4FF0000E4FF0010E0192BEF145
:10399800000F06D04FF0000883F8068083F80580F2
:1039A80001E04FF003085B4AA879D4F81CB0D4F8BA
:1039B80020C0B5F9009069796B881288032856D819
:1039C800DFE800F002122242BEF1000F03D0514896
:1039D8000280002236E00198002840F0B1864D4868
:1039E80002809DF804202DE09CF8000000EB800088
:1039F800814503DC47480280012223E0019F012022
:103A0800002F34D000F00BBF019850B14148BBF8EB
:103A18000E20428082803F4FBCF80200F8804FF0B1
:103A280002089CF800A09CF80100504400EB8000BC
:103A3800814500F388860198002800F0848635487F
:103A480002800222AA7115E032486B80019B028035
:103A58000322AA7169717BB1374A137843F00203D4
:103A68001370264B00225A710EF05AFB04E0294FBE
:103A7800A8713A8069716B80B8F1000F02D0404696
:103A88000AF0A6F92D4FB7F852010DF094FD8346C0
:103A980068B90EF0C5FF2A4BC3F800B0C3F804B0EC
:103AA800C3F808B0274B00221A605A609A60224B6C
:103AB8001A7812F0040F984664D03368D80661D596
:103AC800214B1B78D9065DD4204B1B78002B41D0A5
:103AD80097F8D431BBF1000F44D1002B3DD01C4BDB
:103AE8001A68636A9B1A002B37DA0EF019FB044B2D
:103AF80083F828B046E000BF00340020F0330020EF
:103B0800E80E00203C2700204F330020F40F00204F
:103B1800B83200207827002000007A445D13002086
:103B28006E130020F10E00200000C8425010002043
:103B380000C07F44404B4C00223400209C270020CA
:103B4800E021002074240020201100200C00002017
:103B580060270020BBF1000F0CD110200AF038F9C3
:103B680001230DE033B1AF4A12684FF47A7101FBBB
:103B78000323636294F8283023B10AF011F9002373
:103B880084F8283097F8D231019397F8D311B7F811
:103B980098E1B7F89AC100231846A34A32F91320CE
:103BA80080087245C4BF60F07F00C0B2013362452F
:103BB800B8BF40F04000042BEFD194F829309B4A5D
:103BC800834205D192F82A30F92B04D8013300E05A
:103BD800002382F82A30964B84F829001A78DFF8F7
:103BE8006C929A46EAB9D9F80030DA0709D5BBF1E0
:103BF800000F16D198F80030DB0712D50EF0F2F856
:103C08000FE098F8003058070BD58A4B1B7843B162
:103C18006B7933B911B10EF083FA02E0BBF1000FF2
:103C2800F9D094F82A30814ADFF824B2142B40F0F6
:103C38009080019B003318BF012301939AF800304C
:103C480073B392F829305F2B12D198F8003003F043
:103C5800040303F0FF0113B10EF062FA08E00B2031
:103C6800039102920AF0B4F8029A039982F82A1092
:103C7800019BABB194F829307D2B11D198F8003015
:103C880003F0040303F0FF0213B10EF049FA07E052
:103C98000B2002920AF09CF8644B029A83F82A20BF
:103CA80098F8003003F0040303F0FF01002B50D113
:103CB80094F829305D4A572B15D15F4B4FF47A722F
:103CC8001A803368190601D504F0A6FB5B4B1B6804
:103CD8005A0742BF5A4A0A21118013F0080338D103
:103CE800584A138035E03068400717D55A2B15D14C
:103CF80092F82B302BB1012382F82B1082F82C304C
:103D080027E092F82D3083F0010382F82D300BB1B3
:103D18000C2000E00D200AF05BF81AE05D2B00F0A3
:103D280015855B2B00F014855E2B02D1032000F073
:103D380010BD562B01D107F0A3FB9AF80030002BD9
:103D480000F01B8594F829306F2B40F011850EF098
:103D580049F833685B0738D594F82D30334A9BB15E
:103D680098F8003058070FD52F4BB3F90610B7F85D
:103D78009831994208DDD9F8003013F0010302BFE9
:103D88003221118682F82D30D9F80030D9030CD5AC
:103D980094F83220254B22B993F82B200AB9322205
:103DA8001A86012384F832300FE094F82B301F4A2A
:103DB8005BB198F8003003F0040303F0FF0123B966
:103DC800012382F82B1082F82C30DBF800800023C6
:103DD800C9F8003008F17B0708F1CB0A3A787B78FC
:103DE80017F8010C9A420DD2394602F0CBFA48B1C5
:103DF80017F8022C012303FA02F2D9F80030134312
:103E0800C9F8003004375745E8D10F4B1B780BB37E
:103E18000E4FDFF828803B6813F0020F40F04D8307
:103E280046E300BF6027002078270020E80E002026
:103E38000C0000204E3300201A3400201C110020F2
:103E480018340020F810002025340020F40F00203A
:103E58002C10002008F1CA0708F589783A787B7891
:103E680017F8010C9A4222D2394602F08BFAF0B1C7
:103E7800BB7897F804E0C34A97F80390C2480C212E
:103E8800013B01FB0E4103EB430313448A6B9A4247
:103E98000DD08B63002390F86420CB63012303FAD1
:103EA8000EF322EA030381F8349080F86430063771
:103EB8004745D3D1B54BDFF8E8A21F68B44B1B6860
:103EC8000293B44B1B78039300230193DAF8003074
:103ED800002B00F0E48293F80090B9F1000F00F095
:103EE800DE82DAF8042002998A1A002A0CDB01F52E
:103EF800FA720199CAF8042001228A4094F86410E1
:103F080021EA020284F86420039A002A00F0C7829A
:103F18001AF8042C59780432D2B2002940F07E8273
:103F28009D4931F912109D4AB2F8962102F1C80054
:103F3800814202DD93F802B015E0C83A914203DAF3
:103F48009978C1F1000B0EE0019A0123934094F88F
:103F5800642022EA030384F86430029B03F5FA73B1
:103F6800CAF804309BE2019A94F864301341DA07E6
:103F780000F19582BBF1000FCCBF0220012009F0AF
:103F88004DFF09F1FF33DFF80082132B00F27F8227
:103F9800DFE813F01400250037004B0064006B00C5
:103FA800D2004B01B201E20112027D024B005A001D
:103FB8006B00D2004B01A2001D01820197F800801E
:103FC800D844B8F1FA0FA8BF4FF0FA0828EAE87801
:103FD800384687F8008002F0BBF901200FE097F817
:103FE8000180D844B8F1640FA8BF4FF0640828EAEC
:103FF800E878384687F8018002F0AAF9022041469D
:10400800D7E197F80390D944B9F1640FA8BF4FF0EE
:10401800640929EAE97987F803903846D8F86810DE
:1040280002F04CF903204946C3E1797959446429DF
:10403800A8BF642121EAE17179710D2009F04EFED3
:10404800B9F10D0F00F02382397959446429A8BFCA
:10405800642121EAE17139710E20AAE1B979594444
:1040680081F30801B9710520A3E1D8F86C301A78FA
:10407800022A22D107EE90BAF8EEE77AB2EE040AE5
:1040880087EE800AD3ED097A30EE270AB5EEC00A2A
:10409800F1EE10FA09D4DFED447AB4EE670AF1EED6
:1040A80010FAC8BFB0EE670A01E09FED400A83ED41
:1040B800090A0F2002F09DF90AE099785944C829A5
:1040C800A8BFC82121EAE17199700F2009F006FE06
:1040D800B9F10F0F00F0DB81D8F86C301A78022A9A
:1040E80020D107EE90BAB8EEE78AB2EE040A88EE5D
:1040F800008A93ED080A38EE000AB5EEC00AF1EE20
:1041080010FA09D4DFED287AB4EE670AF1EE10FA56
:10411800C8BFB0EE670A01E09FED240A83ED080AE4
:1041280012206EE159785944C829A8BFC82121EA4C
:10413800E171597012203CE1D8F86C301A78022AE3
:1041480036D107EE90BAB8EEE70ADFED177A93EDAD
:104158000C7A80EE270A30EE070AB5EEC00AF1EEB7
:1041680010FA07D4B4EE670AF1EE10FAC8BFB0EE41
:10417800670A01E09FED0D0A83ED0C0A102002F09A
:1041880038F920E000880108E80E002054100020CB
:10419800602700204E330020782700209C2700202D
:1041A800200F002000007A440000C84200000000F0
:1041B800197B5944C829A8BFC82121EAE17119739C
:1041C800102009F08BFDB9F1100F00F06081D8F8CC
:1041D8006C301A78022A1ED107EE90BAB8EEE78A38
:1041E8005FED0F7A93ED0B0A88EE278A38EE000A06
:1041F800B5EEC00AF1EE10FA07D4B4EE670AF1EE94
:1042080010FAC8BFB0EE670A01E01FED180A83ED87
:104218000B0A1320F5E0D97A5944C829A8BFC82148
:1042280021EAE171D9721320C3E0D8F86C301A780A
:10423800022A22D107EE90BA1FED260AF8EEE77A95
:1042480087EE800AD3ED0F7A30EE270AB5EEC00A62
:10425800F1EE10FA09D45FED2C7AB4EE670AF1EEAC
:1042680010FAC8BFB0EE670A01E01FED300A83ED0F
:104278000F0A112002F0BDF80AE0997D5944C829B7
:10428800A8BFC82121EAE1719975112009F026FD1E
:10429800B9F1110F00F0FB80D8F86C301A78022AB7
:1042A80020D107EE90BA1FED410AB8EEE78A88EEF2
:1042B800008A93ED0E0A38EE000AB5EEC00AF1EE58
:1042C80010FA09D45FED487AB4EE670AF1EE10FAF5
:1042D800C8BFB0EE670A01E01FED4C0A83ED0E0A75
:1042E80014208EE0597D5944C829A8BFC82121EA65
:1042F800E171597514205CE0D8F86C301A78022AFC
:1043080020D107EE90BAB8EEE78AB2EE040A88EE3A
:10431800008A93ED0A0A38EE000AB5EEC00AF1EEFB
:1043280010FA09D45FED607AB4EE670AF1EE10FA7C
:10433800C8BFB0EE670A01E01FED640A83ED0A0A00
:1043480009205EE0D9785944C829A8BFC82121EAC4
:10435800E171D97009202CE0D8F86C301A78022A5B
:104368001ED107EE90BAB8EEE78A5FED717A93ED49
:104378000D0A88EE278A38EE000AB5EEC00AF1EE7B
:1043880010FA07D4B4EE670AF1EE10FAC8BFB0EE1F
:10439800670A01E01FED7B0A83ED0D0A0A2030E071
:1043A800597B5944C829A8BFC82121EAE17159732A
:1043B8000A2009F093FC6AE0D8F86C301A78022ACF
:1043C80022D107EE90BA1FED890AB8EEE78A88EE87
:1043D800008A93ED100A38EE000AB5EEC00AF1EE35
:1043E80010FA09D45FED907AB4EE670AF1EE10FA8C
:1043F800C8BFB0EE670A01E01FED940A83ED100A0A
:104408000B2001F0F6FF42E0D97D5944C829A8BF26
:10441800C82121EAE171D9750B20CAE7012936D1F3
:104428009878B64B33F91230B3F5617F05DB40F667
:1044380033029342A8BF134601E04FF46173B9F108
:104448000C0F24D14FF4966292FBF0F0AC4AA3F51E
:10445800617393FBF0F35FFA83F81378434516D042
:10446800B8F1040F34BF434602231370A54A09FB71
:104478000323A54A0233136006F042FE484641462C
:1044880009F02CFC08F10100C0B209F0C7FC019A40
:104498000123934094F86420134384F86430019B0B
:1044A8000133042B01930AF10C0A7FF40FADAFE43A
:1044B8003368DB0510D56B7973B1D8F800309D07E8
:1044C8000AD5924B1B8813F001050AD10EF0A8FA01
:1044D800012006F035FD04E0012006F020FD01234F
:1044E80000E000233A6850070DD563B1012006F0BB
:1044F80016FD864B1B88990708D40EF091FA022006
:1045080006F01EFD02E0022006F009FDD8F8003092
:1045180013F00A0F26D03B68DA060BD57B4B1B88B5
:104528005B070AD4042006F00BFD794B1B88A4F81E
:10453800703002E0042006F0F2FC3B689D0607D5C7
:10454800724B1B88580606D4402006F0F9FC02E09E
:10455800402006F0E4FC3B68590642BF6C4B1B88C0
:10456800A4F87230D8F800309A0608D43B681B05C6
:1045780040F191804FF4807006F0E2FC8FE0654BCB
:10458800DFF888811B7813F0020F50D0624B1B783C
:10459800042B4CD93B6813F400790FD0B8F80030DD
:1045A800DD0638D4102006F0CBFC202006F0B7FC3E
:1045B8005A48011D03F084FE022328E0B8F8005091
:1045C80005F01005ADB22DB1102006F0A8FC0125AC
:1045D80084F874903B68580511D5A36F50495A89DF
:1045E800B1F90030002BB8BF5B42934207DAB1F94A
:1045F8000230002BB8BF5B429342C0F21681B8F874
:104608000030990608D5202006F089FC002384F89C
:104618007430012500E0002594F87C30BBB90E20E9
:1046280009F0D6FB3F4B012283F87C200FE0B8F855
:10463800003003F03003002B98D0102006F06FFCF8
:10464800202006F06CFC002384F8743001E0002D73
:104658008CD0354B002003F1280503F15004334A70
:10466800002122F81010324A596022F81010043242
:10467800696022F8101000221A609A602A60AA6005
:1046880022606160A26014331435143400287FF46A
:104698006DAF0120E3E74FF4807006F040FC254B36
:1046A8005A79082A1C4601D00E2A02D1402006F069
:1046B80036FC33685A0540F1CE8094F8103223B99D
:1046C8001D4B1B7813F0040F02E03B6813F4002F16
:1046D8000BD01A4B00221A703C2002F035FD00283E
:1046E80000F0B9800BF0BEF8F6E704F0F9F907B06E
:1046F800BDEC028BBDE8F04F02F085BC78270020A6
:10470800E0240020442F002054100020E011002055
:10471800F810002020110020261100205C10002035
:1047280000110020E80E0020680F00201C34002033
:10473800E00F00209C27002022340020C81200200F
:104748000120FFF73BB90320FFF738B9012000E04B
:1047580002205FFA80FA0AF1FF3387F8A83706F0DB
:1047680039FC06F0F1FC504609F058FBFFF7F1BAA6
:10477800019A12B17E2B3FF4EAAA94F82930972BBC
:1047880005D1374B4FF4C872DA85FFF7E2BAA72B89
:1047980006D1344A137843F004031370FFF7D9BAEB
:1047A8000022BB2B059201D1022303E0B72B04D1D1
:1047B8004FF6FE73ADF8163009E0BE2B01D1022387
:1047C80003E0BD2B1AD14FF6FE73ADF81430DBF8B9
:1047D8000020BDF81410B2F858300B44A2F8583035
:1047E800BDF81610B2F85A300B44A2F85A3006F049
:1047F80047FE002384F82A30FFF7ABBA792B04D19F
:10480800194AD37823F0010306E07A2B7FF4A1AA92
:10481800154AD37843F00103D370FFF79ABA0133EE
:1048280001469BB20220FFF7C9B8B8F800309B06D2
:104838003FF5F2AE202006F083FB0C480C4B011D1F
:104848001A685B684360026003F03AFD044B012577
:1048580083F87450E0E607B0BDEC028BBDE8F08F3A
:10486800E80E00202011002098200020641000206D
:10487800281100202DE9F0472DED028B4B28A0B020
:10488800044600F0558600F2B480302800F0E08637
:1048980051D8222800F0A18423D8032800F0608191
:1048A80014D8012800F05081022840F03C870420E9
:1048B8000BF044F843200BF012F84C200BF00FF8E3
:1048C80046200BF00CF84C2000F068BE042800F0DD
:1048D8005181052840F027871A200BF02FF8002473
:1048E80059E1282800F0F28515D8242800F0D98548
:1048F800262840F01887B44C06200BF01FF8B4F8AF
:104908005C010BF01EF8B4F85E010BF01AF8B4F86D
:10491800600100F0C3BD2C2800F0EB852E2800F0C4
:1049280081862A2840F0FF8601200BF007F8A64B65
:10493800587900F033BE3D2800F018831ED8362879
:1049480000F056860BD8322800F02286342840F032
:10495800EA8648200AF0F2FF002500F060BC3A28F9
:1049680000F0B4823B2800F03184382840F0DB8620
:1049780004200AF0E3FF944C00F099BD452800F0AC
:10498800BF8627D8402800F02586422840F0CB86ED
:104998008D4C10200AF0D2FF60790AF0A0FFA068C1
:1049A8000AF0D8FF94F890010AF099FFB4F85C0176
:1049B8000AF0C7FFB4F85E010AF0C3FFB4F860015B
:1049C8000AF0BFFFB4F880010AF0BBFFB4F8820117
:1049D80000F064BD472800F07186C0F05E86492863
:1049E80040F0A18602200AF0A9FF774B988900F0D1
:1049F80055BD702800F0ED8258D8692800F046822D
:104A08002AD8652800F0FA8015D84D2800F09F852F
:104A1800642840F0888607200AF090FFE7200AF013
:104A28005EFF694B58790AF05AFF00200AF057FFD9
:104A3800042000F074BE672800F0AB8100F21982F0
:104A480012200AF07BFF614B1B88B3F5806F8CBF87
:104A58000825012500247EE16C2800F02A8217D859
:104A68006A2800F0A0846B2840F05D8605200AF0D3
:104A780065FF574B18880AF064FF564B18880AF0F0
:104A880060FF554B93F8720000F0010000F086BDFE
:104A98006E28514D00F0218200F2738206200AF040
:104AA8004DFF286E0AF056FF4C4B0DE2782800F0B7
:104AB8007D8119D8742800F0DD830BD8722800F0A6
:104AC8003284732840F02F8608200AF037FF01242B
:104AD80000F062BC762800F0868400F204842F205F
:104AE8000AF02CFF3E4C69E3A42800F0A38414D8F4
:104AF8007B2800F00983A02840F015860C200AF0D6
:104B08001DFF384B18680AF025FF374B18680AF064
:104B180021FF364B186800F002BEF12800F08281B0
:104B2800FE2800F0AE84F02840F0FD852A4C0420D1
:104B38000AF004FF636CB3F85A000AF002FF636CD2
:104B4800B3F8580000F0AABC03200AF0F7FE0020D2
:104B58000AF0C5FE20460AF0C2FE0C2000F01EBD79
:104B68000AF0ECFE01200AF0BAFE0A200AF0B7FEAD
:104B780000F05EBC06200AF0E1FE53200AF0AFFE0A
:104B880052200AF0ACFE46200AF0A9FE33200AF0B3
:104B9800A6FE00F082BC164B185D01340AF09FFE99
:104BA8000B2CF8D10024134B185D01340AF097FE42
:104BB800082CF8D10024104B185D01340AF08FFE40
:104BC800072CF8D100F0ADBD9C2700202000002064
:104BD8009A1100209C110020E80F0020F0100020FE
:104BE8003B880108ACF7FF1FB0F7FF1FB4F7FF1FA2
:104BF80000A701080CA70108E1A60108C94C0B2071
:104C08000AF09CFE20880AF09CFE6268C64B9A4215
:104C18000CBF2089608980B20AF093FEC34B1B68E1
:104C2800C3F3C000C3F38002800040EA4200C3F32C
:104C380040021043C3F3401240EAC20003F01003DD
:104C480018430AF07EFEBA4B1A88E36812F0010F87
:104C580014BF4FF0020C4FF0000C12F0020F02F0DC
:104C6800080814BF4FF0040E4FF0000E03F4475924
:104C780012F0040F14BF1027002749EA080912F0A0
:104C8800400F03F4804814BF2026002649EA08098B
:104C980012F0100F03F4004814BF4FF400750025FC
:104CA80049EA080912F0200F03F4803814BF4FF4C2
:104CB8008060002049EA080912F4807F03F4003874
:104CC80014BF4FF40061002149EA080912F4007F7B
:104CD80003F48028974A49EA080903F4002849EAB6
:104CE8000809127803F4801849EA080903F00073E8
:104CF80049EA0303C2F3800243EA020343EA0C03CE
:104D080043EA0E0E4EEA070746EA070645EA060595
:104D180040EA050041EA000114BF4FF400184FF0C3
:104D2800000841EA08080020217C03468B420BD288
:104D3800814A9C5C012202FA04F414EA080F1CBFA1
:104D48009A4010430133F1E70AF004FE7B4B93F8D5
:104D5800A80700F023BC7A4B33F9140090FBF5F058
:104D6800013480B20AF0EDFD032CF4D16D4CA08D16
:104D78000AF0E7FDE08D0AF0E4FD208E714C0AF0A0
:104D8800E0FD20880AF0DDFD60880AF0DAFDA088E1
:104D980084E310200AF0D2FD00246B4B185D013427
:104DA8000AF09DFD102CF8D100F0BBBC70200AF071
:104DB800C5FD00265B4D0E246B6C744323440136FD
:104DC800B3F819010AF0BDFD6B6C2344B3F81B015D
:104DD8000AF0B7FD6B6C2344B3F81D010AF0B1FD6E
:104DE8006B6C234493F81F010AF079FD6B6C234424
:104DF80093F820010AF073FD6B6C234493F82101AA
:104E08000AF06DFD6B6C234493F822010AF067FDEC
:104E18006B6C1C44D4F823010AF09CFD082EC9D100
:104E280000F07FBC7020454C0AF088FD04F1700545
:104E380094F8D4000AF053FD94F8D5000AF04FFD19
:104E480094F8D6000AF04BFD94F8D7000AF047FD15
:104E580094F8D8000AF043FD94F8D9000AF03FFD11
:104E6800073494F8D3000AF03AFDAC42E0D100F0E0
:104E780058BC10200AF062FD0024344B185D013440
:104E88000AF02DFD102CF8D100F04BBC304D2878DD
:104E9800400000F0FE000AF051FD00242B789C42EF
:104EA80080F03F842B4B33F814000AF04AFD01349C
:104EB800F4E7294C06200AF041FD20880AF041FD5C
:104EC80060880AF03EFD254B1888E7E204200AF0C6
:104ED80035FD144B586E00F022BC07200AF02EFD59
:104EE8001F4B1888FF28A8BFFF20C0B20AF0F7FCA4
:104EF8001C4B186880F3100080B20AF022FDB5F848
:104F080068000AF01EFD0D4B93F88521164B1868B2
:104F180022B10A23584380F3100001E000F30F0088
:104F280080B2BBE2E80F0020005400401C110020B2
:104F3800E011002022340020F90F00209C270020D7
:104F4800EA100020441300201A100020301000201E
:104F58004C3300207827002034270020F810002048
:104F68000C1100201811002014110020BC4C022044
:104F78000AF0E4FC94F8D4010AF0B1FC94F8D301E7
:104F88000CE30B200AF0DAFCEB6E18780AF0A7FCA9
:104F9800EB6E58780AF0A3FC0026EB6EB14C334454
:104FA800013618790AF09BFC032EF6D1E36ED87906
:104FB8000AF095FCE36E98780AF091FCE36ED878D5
:104FC8000AF08DFCE36E58890AF0BBFCE36E187A90
:104FD800E4E2A44C1E200AF0B1FC636C1B78022B9F
:104FE8004FF000057DD1636C03EB850393ED080A50
:104FF800B2EE048A20EE080A11F0EAF9FA28A8BFEE
:10500800FA2020EAE070C0B20AF069FC636CDFEDB8
:10501800967A03EB850393ED0B0A20EE270A11F02D
:10502800D7F9FA28A8BFFA2020EAE070C0B20AF03F
:1050380056FC636CDFED8D7A03EB850393ED0E0A66
:1050480020EE270A11F0C4F96428A8BF642020EADA
:10505800E070C0B201350AF042FC032DC3D1072D20
:10506800636C2CD193ED110A20EE080A11F0B0F907
:10507800FA28A8BFFA2020EAE070C0B20AF02FFC94
:10508800636C93ED120A20EE080A11F0A1F9FA28D0
:10509800A8BFFA2020EAE070C0B20AF020FC636CD6
:1050A80093F84C3000EE103AB8EE400A11F090F93F
:1050B800FA28A8BFFA2020EAE070C0B20BE02B441F
:1050C80058780AF00CFC636C2B44D87A0AF007FC79
:1050D800636C2B44587D01350AF001FC0A2DBED1C2
:1050E8001FE3636C2B4458780AF0F9FB636C2B447C
:1050F800D87A0AF0F4FB636C2B440135587D0AF02A
:10510800EEFB0A2DEDD10CE33C200AF017FC00243D
:10511800544D9FED568A6B6C03EB840393ED080A9C
:1051280020EE080A11F054F980B20AF00AFC6B6C00
:1051380003EB840393ED0B0A20EE080A11F048F9FB
:1051480080B20AF0FEFB6B6C03EB840393ED0E0A4E
:1051580020EE080A11F03CF9013480B20AF0F1FBA4
:10516800032CD5D1072C6B6C16D193ED110A20EEC8
:10517800080A11F02DF980B20AF0E3FB6B6C93ED8D
:10518800120A20EE080A11F023F980B20AF0D9FBBE
:105198006B6C93F84C000BE0234458780AF0D1FB71
:1051A8006B6C2344D87A0AF0CCFB6B6C2344587D93
:1051B80001340AF0C6FB0A2CD4D1B2E214F8010F6C
:1051C800002800F0AE820AF08AFBF7E701200AF017
:1051D800B5FB244B5B6C1878E0E150200AF0AEFB7D
:1051E8000025204B5C6C224B04EB85040C2194F8C1
:1051F800792001FB0233013593F838000AF06FFB80
:1052080094F87A000AF06BFB94F87B000AF067FBCD
:1052180094F87C000AF063FB142DE2D181E2114B73
:105228005C6C062303FB0544013594F8CE000AF0B4
:1052380056FB94F8C9000AF052FB94F8CA000AF029
:105248004EFB94F8CB000AF04AFB94F8CC000AF025
:1052580046FB94F8CD000AF042FB0C2DDFD160E24A
:105268009C270020E80F00200000C84200007A4474
:105278003C8801084FF0000801260027C94B1A7C1A
:10528800974227DA11330024FA5CC74D0C2305F145
:1052980030016343595C914207D12B44586B10F09D
:1052A800CCFE82462EB9B14605E001341B2CECD168
:1052B8000EE080440CE0D1450ADA0C2303FB0453CA
:1052C8005B6B13F809000AF00AFB09F10109F2E720
:1052D8000137D3E7002E00F024825FFA88F00AF045
:1052E8002DFB0026C9E7AF4D287C0AF027FB0024D8
:1052F8002B7C9C4280F01582AC4BE65C0021AA48CE
:105308000C2200F1300702FB01F3DA5DB24205D14D
:10531800034493F838000AF0E2FA02E001311B294D
:10532800EDD10134E4E7A24C16200AF007FBB4F8EB
:1053380096010AF006FBB4F844010AF002FBB4F83F
:1053480046010AF0FEFAB4F848010AF0FAFAB4F88D
:10535800D0010AF0F6FA94F8E1010AF0C0FA002048
:105368000AF0BDFA94F8E2010AF0B9FA94F8850156
:105378000AF0B5FA94F892010AF0B1FA00200AF09E
:10538800AEFA884B5B6C0A20B3F9563093FBF0F009
:1053980080B20AF0D6FA8AE0E0B201340AF09FFA45
:1053A800092CF9D1BDE110200AF0C8FA814B824CD2
:1053B800187800F002000AF092FA804B18780AF088
:1053C8008EFA20680AF0C6FA60680AF0C3FA7C4BC5
:1053D80018880AF0B6FA7B4B18880AF0B2FA714BB3
:1053E800B3F870005AE00AF05DFA074612200AF096
:1053F800A5FA6C4C17B9666FA56F06E0102F13BF9E
:105408000025E66FD4F880502E4638460AF067FA31
:1054180030460AF09FFA28460AF09CFAD4F884002D
:105428000AF098FA00200AF08CFA00200AF089FAAB
:105438000020B3E05B4D95F8880080000130C0B2D1
:105448000AF07CFA95F888000AF049FA00242E46FA
:1054580096F888309C4280F064815B4D285D0AF0A4
:105468003EFA05F11003185D0AF039FA05F1200338
:105478003035185D0AF033FA285D0AF030FA013445
:10548800E6E708200AF05AFA00200AF05AFA002043
:105498000AF057FA00200AF054FA00200AF051FAEC
:1054A8003FE104200AF04AFA414B986837E194F842
:1054B8007A010AF014FA94F87E010AF010FA94F8C6
:1054C8007D010AF00CFA94F87F0167E0384C072058
:1054D8000AF034FAB4F880010AF033FAB4F8820119
:1054E8000AF02FFA94F884010AF0F9F9B4F8860161
:1054F800D4E72F4C0C200AF021FA94F890010AF016
:10550800EEF9B4F89A010AF01CFAB4F896010AF018
:1055180018FAB4F898010AF014FA94F891010AF00C
:10552800DEF9B4F89C010AF00CFAB4F89E01B5E76C
:105538001F4C04200AF002FA94F8CE010AF0CFF9C1
:1055480094F8CF010AF0CBF9B4F8D001A6E71F4CC4
:105558001F4D2078043800EB4000C0B20AF0EEF985
:10556800042623789E4205F1020580F0DA8015F8BA
:10557800020C0AF0B4F915F8010C00EB800000EBFE
:10558800800000F2EE2080B20AF0DBF90136E8E78D
:1055980001200AF0D3F9064B93F892010AF09FF91B
:1055A800BFE000BFE80F00203C880108F90F002089
:1055B8009C270020201100202811002026110020FF
:1055C8002411002022110020711000204C330020EB
:1055D8003C29002008200AF0B1F90024614B23443B
:1055E800013493F888010AF07AF9082CF6D198E08A
:1055F8005D4B5C4C93F8C900C0EBC000C0B20AF028
:105608009DF904F1280594F8E8010023574AD25C73
:10561800904200F08A800C333C2BF7D10834AC421E
:10562800F1D17EE040204F4C0AF088F904F14005A2
:10563800B4F8A0020AF085F994F8A2020AF04FF92A
:10564800043494F89F020AF04AF9AC42F0D168E0B9
:10565800E020444C0AF072F904F18005B4F8220203
:1056680000F03F000AF06DF9B4F82202C0F386108A
:105678000AF067F994F8200200090AF030F994F862
:10568800200200F00F000AF02AF9043494F81D02F1
:105698000AF025F9AC42E1D143E0354C0D200AF07F
:1056A8004DF904F037FF0AF01AF920880AF052F988
:1056B800E0680AF04FF902F073FF30E00AF006F9EB
:1056C800054684200AF03AF928460AF043F9284B9F
:1056D800DC6805F18003A3428CBF641B802403F0BF
:1056E80017F828462246694604F048FF0024054674
:1056F800AC4216DA1DF804000AF0F1F80134F7E7B5
:1057080013200AF01BF900241A4B185D01340AF023
:10571800E6F80B2CF8D100200AF01CF900200AF05A
:1057280019F9012018E0002016E00AF0D8F8B4F8BA
:10573800EA010AF006F994F8EC010AF0D0F894F8B6
:10574800ED010AF0CCF894F8EF010AF0C8F894F8E3
:10575800EE010AF0C4F861E720B0BDEC028BBDE8A9
:10576800F08700BF9C270020E80F0020D0120020FF
:105778001000002000A70108F8B504460E46174699
:1057880000252046202110F04AFC0446D0B10134FF
:10579800204610F0A9FCB0F5617F05DB40F6340324
:1057A8009842A8BF184601E04FF46170A0F56170F7
:1057B800192390FBF3F00DB9307000E070703B785E
:1057C80001333B700DB90125DBE72046F8BD7FB5F5
:1057D80004780646E4B9364B1B6803EB84031921A9
:1057E80093F87B0093F87C6093F8792093F87A30EB
:1057F8004FF4617511FB005011FB065100900191A7
:105808002C482146013405F055FA142CE3D14CE01C
:1058180010F06AFC1328054641DC254B701C1C68F7
:10582800202100238DF80F3010F0F9FB1E350646B5
:1058380070B10136304610F057FC19289FBF04EBB1
:10584800850358709DF80F30013398BF8DF80F30DD
:105858003046202110F0E3FB064670B10136304691
:1058680010F042FC0D289FBF04EB850398709DF84B
:105878000F30013398BF8DF80F3004EB85043046A4
:10588800E11C0DF10F02FFF777FF9DF80F30042B95
:105898000BD0601C0021042210F08BFB05E00648A9
:1058A80006490022132305F005FA04B070BD00BFB5
:1058B8002C100020C0AB0108D5AB0108F4AB0108DF
:1058C80001480AF0C3B800BFFAAB01082DE9F0435C
:1058D80004788FB00546002C59D17B4B0021142247
:1058E80009A807AED3F8008010F063FB0722304602
:1058F800002110F05EFB05A80023A700059308EB24
:10590800070583801A467149B5F802E031F813C0DB
:105918001CEA0E0F0AD00DF1380C0E3102F1010EFF
:105928006244595C02F81C1C5FFA8EF20133072BA3
:10593800E9D100210B46664AB5F802E011F802C029
:105948001CEA0E0F0AD00DF1380C063203F1010ED5
:1059580063448A5C03F8242C5FFA8EF3013106292C
:10596800E9D118F807305B498DE841006A7802925E
:1059780009A81A0903F00F0305F087F921465648CC
:1059880009AA013405F096F9202CA6D199E010F067
:10599800ABFB1F28044600F3868028462021E4B28A
:1059A80010F03DFB1F2C02D9FFF78AFF89E0464B18
:1059B8001B6803EB8404451C00212046042210F0D8
:1059C800F8FA0027454B09AE304600210A2217F89D
:1059D80003905FFA87F810F0ECFA002315F8012B12
:1059E80032B10A2B04D04A4502D0F2540133F5E70C
:1059F8004A455FD108F1FF33032B09D8DFE803F0EC
:105A08001005023F0DF1230134E00DF123011EE0E2
:105A1800304610F069FB2378C0B243EA001006E074
:105A2800304610F061FB237800F00F001843207017
:105A380031E00133062B0AD0244800F11B069E5D95
:105A48009642F6D103445A7D63881343638011F864
:105A5800012F02B30023EFE70133072B0AD01B48BD
:105A680000F10E069E5D9642F6D130F81320638849
:105A78001343638011F8012F6AB10023EFE7304622
:105A880010F032FB0F2804DC304610F02DFB60705C
:105A980001E0002363700137052F93D101240AF038
:105AA8008BFE74B980E70E490E4800221F2305F0CB
:105AB80001F906E020460021042210F07AFA0024B9
:105AC800EDE70FB0BDE8F083B4100020BC890108F1
:105AD800D189010808AC010817AC0108DD89010863
:105AE800F4AB0108D5AB01082DE9F041047807466D
:105AF8007CB9344DB5F8BC21B5F8BE3132482146E1
:105B0800013405F0D7F8042C05F10405F2D1BDE8FD
:105B1800F0812E4910F056FAB0B92A4B4FF47A7139
:105B28004FF4FA62A3F8BC11A3F8BE21A3F8C01180
:105B3800A3F8C221A3F8C411A3F8C621A3F8C81179
:105B4800A3F8CA21BDE8F081384610F0CDFA032841
:105B580005462ED83846202110F061FA044630B1A7
:105B68000134204610F0C0FA0127064600E0074637
:105B78002046202110F053FA10B9BDE8F0419FE605
:105B8800013010F0B1FA012FF7D1A6F2EE2240F25F
:105B9800DC539A42F1D8A0F2EE229A42EDD886421E
:105BA800EBDA084B6E3503EB85039E80D880BDE8A1
:105BB800F0810748074900220323BDE8F04105F0BA
:105BC80079B800BF9C27002023AC010836AC010837
:105BD800D5AB010849BA01082DE9FF41047805460B
:105BE800002C39D17348744D09F030FFD5ED057A92
:105BF800F5EE407AF1EE10FA00F0D98021466F48B0
:105C080005F058F895ED050A684604F0D3FE0146FC
:105C18006B4805F04FF895ED060A684604F0CAFE91
:105C28000146674805F046F895ED070A684604F00E
:105C3800C1FE0146624805F03DF895ED080A684640
:105C480004F0B8FE013401465E4805F033F80C2C28
:105C580005F11005CAD1AAE05B49052210F0F6F952
:105C680040B9554B03F1C0020021596110339342EA
:105C7800FAD19CE028465549042210F0E7F9044679
:105C88002846002C40D1202110F0C9F9002800F046
:105C98008E80451C284610F0D0F907464C4B53F827
:105CA80024601EB94B4809F0D1FE80E028463146F1
:105CB800FAB210F0CBF901340028EFD13E4B03F1D2
:105CC800C0029E460021596110339342FAD1424BDB
:105CD80003EBC4029846D2F804C0BCF1000F04D10B
:105CE80031463E4804F0E6FF57E0002718F8343004
:105CF8009F42F5DA3B010EEB030563440FCB1435E5
:105D080085E80F000137F1E710F0EEF90B28064699
:105D180047DC2846202110F082F9054650B10135AC
:105D2800284604F0BDFD244B03EB061383ED050A5A
:105D3800012400E004462846202110F070F90546A9
:105D480048B10135284604F0ABFD1B4B03EB0613A5
:105D580083ED060A01342846202110F060F9054633
:105D680048B10135284604F09BFD134B03EB06139D
:105D780083ED070A01342846202110F050F910B9A4
:105D8800FFF79EFD13E0013004F08AFD0A4B032C57
:105D980003EB061686ED080AF2D11148FFF71CFF3F
:105DA80005E01048104901220C2304F083FF04B0D9
:105DB800BDE8F0813CAC01089C27002057AC0108E5
:105DC8005DAC0108A5B7010836AC010861AC010853
:105DD800E893010866AC0108F0AA010875AC01084F
:105DE800DCA90108D5AB0108F4AB0108F0B50478CB
:105DF80087B006461CBB524B1968062303FB0411E7
:105E0800192091F8CA5091F8CB7091F8CE2091F8EA
:105E1800C9304FF4617610FB056510FB07600095EB
:105E2800019091F8CC000290C83146484979039115
:105E38002146013404F03EFF0C2CDCD17DE010F04B
:105E480053F90B28044672DC3D4B701C1D68202159
:105E580000238DF8173010F0E2F8064680B10136BD
:105E6800304610F041F903289FBF062303FB045373
:105E780083F8CE009DF817309CBF01338DF817309A
:105E88003046202110F0CBF8074680B1013738465C
:105E980010F02AF90D289FBF062303FB045383F84B
:105EA800C9009DF817309CBF01338DF817300626BE
:105EB8006643A9193846CA310DF11702FFF75CFC91
:105EC800202110F0ACF8074670B10137384610F0C1
:105ED8000BF914289FBF9DF817307619013386F8FF
:105EE800CC0098BF8DF817303846202110F097F86D
:105EF80078B1013010F0F8F80D289FBF062303FB96
:105F0800045383F8CD009DF817309CBF01338DF8FA
:105F180017309DF81730062B0FD0062202FB0450CD
:105F28000021C93010F045F8FFF7CAFC05E0064823
:105F3800064900220B2304F0BDFE07B0F0BD00BFE8
:105F48002C10002081AC0108D5AB0108F4AB010886
:105F5800F7B5047805464CB9204601A90BF01AFBA1
:105F68000134FFF7F5FF0E2CF6D151E010F0BCF824
:105F7800C6B20D2E48D8681C202110F050F80346F0
:105F880058B15B78682B00F1010007D0732B01D161
:105F9800012704E0FFF794FC3AE000E00027202105
:105FA80010F03DF81B4C06F1D005C8B1013010F0D7
:105FB8009BF840F2ED2380B2984205DD40F6CA0313
:105FC8009842A8BF184601E040F2EE2004EB4503D2
:105FD80004F81570A0F2EE20192290FBF2F0587028
:105FE80014F815300C4804EB4504012B63784FF086
:105FF800190540F2EE2431460CBF7322682205FBD6
:10600800034304F057FE03E004480E2104F052FE57
:1060180003B0F0BD9C270020A1AC0108B3AC010877
:1060280010B50446204607F058FF18B90A2007F0B3
:1060380090FEF7E710BD002207490C2303FB02136B
:106048005968814204D10022C2621A725A607047AC
:106058000132052AF0D17047D01200202DE9F7430C
:1060680089469DF8288011461A469DF82C30064628
:1060780000250C2068431D4FC419C057B04202D1F7
:10608800207A20B12BE00135052DF2D127E0022E30
:106098000FD005DC56B1012E21D1009314480AE037
:1060A8001E2E0DD01F2E1AD1012009E00093114891
:1060B80001E011480093434603F004FB044605E061
:1060C80004F06EF94146044607F004FF4CB10C2376
:1060D80003FB0575267185F808906C6001E00020C7
:1060E80000E0204603B0BDE8F08300BFD0120020D6
:1060F80000440040003801400048004010B5084BFB
:106108001968002201EBC20393F90240844201D1CD
:10611800981C10BD0132052AF4D1002010BD00BF23
:10612800CC120020F0B5027887B08AB94A4C04F145
:10613800280694F8E82100234849595650B281426C
:106148006ED00C333C2BF7D10834B442F1D181E046
:10615800002204920592451C0FF0C6FFC4B260B23B
:10616800FFF7CCFF074618B18DF81040012400E076
:106178000446284620210FF052FF054638B1013564
:1061880028460FF0B1FF0134ADF81200E4B2002642
:10619800284620210FF043FFB0B3451C28460FF0D6
:1061A800A3FF00222E4951F8223083425FFA82FE73
:1061B80004D00132082AF5D1002300E0734651F8D3
:1061C8002320824220D1022E0FD0032E12D05A1E35
:1061D800012ED2B204D0042A13D88DF814300EE060
:1061E800042A0ED88DF8153009E0052B09D88DF84A
:1061F800173004E09A1E052A03D88DF816300134AA
:10620800E4B20136042EC3D1052C04D807B0BDE88A
:10621800F040FFF755BB04AB03CB3860796019E059
:1062280094F8ED010E4B94F8EC5153F82000B4F8B3
:10623800EA21009094F8EF0153F82000019094F8B7
:10624800EE0153F82000029053F82530054804F079
:1062580031FD79E707B0F0BD9C270020D01200205F
:10626800B88E0108CAAC010838B1438811EA0300A6
:1062780003D08B420CBF01200220704730B50A4B77
:106288000A491C680A79042A0AD8134604EBC3038E
:10629800551CEAB29D882842F5D00A71981C30BD79
:1062A8000A71002030BD00BFCC120020B4100020BD
:1062B800014B00221A71E1E7B41000202DE9F047E4
:1062C800877890F803C0214DBBB2C7F1640E03EB89
:1062D80083065C42C3F178005FFA8EFE7600CCF14B
:1062E8006408A4B280B2A3B20FFA83F9B9F1000F1F
:1062F80005DC002B14BFBA464FF0010A00E0F24655
:1063080013FB03F303FB0CF21AFB0AF392FBF3F300
:10631800434403FB09F30A2293FBF2F333449BB291
:1063280025F8023FB1F800904A880A34C9EB020AFE
:10633800A4B21AB202FB0AF24FF47A73844292FBB7
:10634800F3F34B442B80CED1BDE8F087B810002082
:1063580010B544780078002202FB02F3193B63432E
:1063680003F6C413534340F6C411434393FBF1F3BC
:10637800034921F812300132072AEDD110BD00BFC0
:10638800D21000200430114B33F91000B0F5617FB2
:1063980010B506DB40F6330398420246A8BF1A46FA
:1063A80001E04FF461720C78192340F2833013FB3B
:1063B8000404944207DA497813FB01039342B4BFFB
:1063C8000020012010BD002010BD00BF782700204C
:1063D80010B500F1500302788A4203D18478C2785C
:1063E800944204D304309842F5D1002010BD012016
:1063F80010BD1FB5084B1B681B030AD58DF8040098
:1064080001230D2001A98DED030A8DF8053005F053
:1064180035FC05B05DF804FB3C2700202DE9FF475B
:10642800CA4CCB4F23780646002B00F0EA813A6825
:106438006368D31A7C2B40F2E481237A62600133CB
:1064480023724FF0000808F12400C04DC0B202F0DA
:10645800FBFA05F10A0333F9183007EE903ABD4B01
:106468001B88B8EEE77A07EE903AF8EEE77A08F17B
:106478000108C7EE277A9FEDB87A67EE877AFDEEB6
:10648800E77ACDED017ABDF9040002F0CBFAB8F154
:10649800030FD8D1302002F0D7FAB5F9100002F076
:1064A800C1FA02F0C9FA2B7A9A072CD16A6841F22C
:1064B80088339A4218D9102002F0C6FA4FF06408BF
:1064C800686990FBF8F000B202F0ACFA212002F003
:1064D800BBFA686990FBF8F308FB13000028B8BF03
:1064E800404200B202F09EFA142002F0ADFAB4F96C
:1064F800180002F097FA1C2002F0A6FA002002F019
:1065080091FA02F099FA237ADFF840825B0740F0AB
:106518005581022002F098FAD8F81C00DFF8509252
:106528006423323090FBF3F000B202F07BFA0320D0
:10653800B8F9265002F088FA884B1B7813F0040F3C
:106548004FF0050A95FBFAF5ADB20BD030460BF0CB
:1065580032F828B9D9F8003013F0100F18BF002509
:1065680028B205E0D8F828309889B0FBFAF000B2D4
:1065780002F058FAD9F800309E0765D5DFF8F49193
:10658800E68D99F80030A28D704D36014FF0640801
:10659800B6B208FB02325B00B2FBF3F346EA03260D
:1065A800B6B2C3F303231E43062002F04DFA30B2FD
:1065B80002F038FAE38D99F8001001339BB293FB8F
:1065C800F1F201FB1233E385236B9B7B012B05D191
:1065D800392002F039FAB5F92C0019E0AD8D6E2397
:1065E8003A205D43152602F02FFA95FBF6F5AEB278
:1065F800B6FBF8F528B202F015FA08FB15653B2042
:1066080002F022FAA8B2451D0A2095FBF0F000B26C
:1066180002F008FA282002F017FA636B0A2093FBAD
:10662800F0F000B202F0FEF9042002F00DFAA36ABD
:106638009B8913B101F034FA03E0444B986B80F363
:10664800100000B202F0EEF9E36B404E9D0640F1F7
:10665800AA8096F8403098071DD5112002F0F4F969
:10666800B6F842003E4B4FF4F365684390FBF3F0F5
:1066780000B202F0D7F9192002F0E6F9B6F84200A4
:106688004543642095FBF0F595FBF0F300FB1350B0
:1066980000B202F0C7F994F84030B4F8445013F04F
:1066A800020F08BF0025012002F0CEF928B202F03F
:1066B800B9F9092002F0C8F9002002F0B3F9294B12
:1066C80094F846501A88B2F5967F0AD91F4B1B7A60
:1066D80003F00F03072B04D842F20F75954228BF29
:1066E8001546052002F0B0F9236B5B7B0BB928B285
:1066F8001CE0A5F1200307EE903A9FED1B7AF8EE17
:10670800E77AF6EE006AC7EE877ABEEE007AF5EE13
:10671800C07AF1EE10FA58BFB0EE667A77EE877A53
:10672800FDEEE77ACDED017ABDF9040002F07AF9C1
:1067380094F84020054B910703D493F84720012A89
:106748001CD1012384F84730084833E0E0100020CA
:10675800602700202000002000007A442234002016
:10676800A08601007E0000206666E63F2811002012
:106778003C2700207D0000208096184B1B6B5FEDA6
:10678800026A93ED017AD3ED027A27EE267A67EE54
:10679800A67ABDEEC77AFDEEE77A8DED027ACDEDE9
:1067A800037A02A806E0A74A92E8030002AB83E84E
:1067B8000300184602F058F902F03EF9237A282B14
:1067C8001FD1A14B00221A723C263B684FF47A7005
:1067D800B3FBF0F8172002F037F9B8FBF6F5B5FB74
:1067E800F6F006FB1050000200B202F01BF9182068
:1067F80002F02AF906FB158000B202F013F902F044
:106808001BF994F85030904D002B00F03D8107F0B3
:1068180079FA6B6D8D4AC31A9342064640F2C180DD
:10682800002385F85A3085F85C30AB8DDAB21B0A44
:1068380085F8762085F8773085F86C2085F86D30F6
:10684800D5F884203B689A1AD5F88830D97B4FF45C
:106858007A734B439A420ED37D4B1B68C5F884303C
:1068680095F88C30013B012B9FBF102385F85A30D7
:10687800022385F85C300A20626B92FBF0F284F800
:106888007420121284F8752094F84020A36B93FBAF
:10689800F0F384F878301B1284F87930920794F872
:1068A8004630694984F8A73003D42D2381F8A830ED
:1068B80076E0042BD4F84890E76CDFF8A481654AA9
:1068C8008CBF3323322381F8A8304FF0060C624B7B
:1068D80099FBF3F097FBF3F308FB009108FB0378AF
:1068E80003EB83030CFB01F103EB830391FBF2FE43
:1068F800642502FB1E119B0091FBF5F184F89910A9
:1069080009120CFB08FC84F89A109CFBF2F143FA7C
:1069180081F39BB202FB11C292FBF5F284F89E2030
:10692800121284F89C3084F89F201B0AB4F8422085
:1069380084F89D302423534393FBF5F5B4F8BA301B
:1069480084F8A03000EB80001B0A00EB8000800078
:1069580084F8A1300A22B4F84430B3FBF2F303F50B
:10696800FA739BB240FA8EF080B284F8A2301B0A08
:106978004FEAD97984F89700FF0F000A84F89450F9
:1069880084F8A330C5F30725B4F8BC3084F8969092
:1069980084F8980084F89B7084F8955084F8A9309E
:1069A800666594F8BE80284DB8F1000F0DD1D5F872
:1069B800C40007F09BFA012807D90228274F00F0E6
:1069C800388202F021F80123BB70D4F8C8001E4DAC
:1069D800002859D095F8BE703FB1D5F8D03040F6B0
:1069E800B732F31A93420BD84EE00123D5F8C4000E
:1069F80085F8BE30022107F06DFA85F8D47041E0C1
:106A080095F8CC305BB9D5F8C400C5F8C830012179
:106A180085F8BE3007F05EFA01F0F6FF32E0013B80
:106A2800DBB285F8CC3095F8D41095F8D520CBB9E1
:106A38004B1C013285F8D43085F8D520D5F8C40030
:106A48001EE000BFA48E0108E01000203F0D0300E7
:106A58006027002040420F00809698002000002008
:106A6800806967FF0346013213F8017BC5F8C83017
:106A7800781885F8D400D5F8C40085F8D5203946AB
:106A880007F037FAC4F8D06094F8D6309D4DF3B1CA
:106A9800D5F8D830DBB1D5F8DC30C3B1C5F8E03073
:106AA8001B68994AC5F8E430D5F8E8301344187AD9
:106AB800FDF7E0FED5F8E030987908F010FFD5F83A
:106AC800E8300133092B88BF0023C5F8E8308F4D23
:106AD80094F8EC202E688B4B002A00F0E481D3F860
:106AE800F020002A00F0DF8193F8F430013B012BFD
:106AF80000F2D981D4F8F000824F07F0F7F9E0B13D
:106B0800D7F8F00007F0EFF997F8F530D5F80090CE
:106B18007E2B80460ED102231B2887F8F43009D13A
:106B2800D7F8F00007F0E2F920B90123C7F8F89088
:106B380087F8FC3084F8F580DCE7D7F8F8202B6874
:106B48009B1A41F6583293421DD9032387F8F43033
:106B5800A9E16F4A32F8130010B903464FF40360F5
:106B68000133B0F5C06FDBB275D01DD9B0F5006F39
:106B78007AD031D9B0F5036F3ED184F8FD30E36B9C
:106B8800604F99063FD494F8FC1094F8FD30002922
:106B980000F04C812A68921B012ADAD984F8FD306A
:106BA800002384F8FC307EE1B0F5007F42D007D89E
:106BB800B0F5807F47D0B0F5887F00F08580E6E7A4
:106BC800B0F5806F00F0A880B0F5826F00F0ED801E
:106BD800B0F5047FDBD123E0B0F5E26F00F08480EC
:106BE800B0F5E46F00F08580B0F5E06FCFD184F8A0
:106BF800FD30B4F90A1080E0B0F5046F6DD0B0F53F
:106C0800026FC4D1FCE097F840309A07BBD5B7F8BB
:106C1800421024234B431233642193FBF1F1FFE02C
:106C280084F8FD303B4B374F1B689B07ABD5BB8DBA
:106C38000A21F4E084F8FD30364B324F1B68190501
:106C4800A1D5796BECE084F8FD30E36B2D4F5A0742
:106C580099D57969E4E084F8FD302E4B294F1B68FB
:106C68001B0590D5B96BDBE0E16B264A84F8FD3053
:106C78008F0688D592F84010880784D5D90711D592
:106C8800D36C83EAE371002BA1EBE37101EB5101B3
:106C98004FF01902B1FBF2F1ACBF41F0004141F0F5
:106CA80040410EE0936C83EAE371A1EBE371002BA2
:106CB80001EB51014FF01902B1FBF2F1B8BF41F0FD
:106CC80080414FF400608AE084F8FD30E36B0D4F9B
:106CD8005B077FF558AF3969A2E0B4F9181084F85A
:106CE800FD30642359437AE084F8FD30B4F90C1080
:106CF80003E0B4F90E1084F8FD302C2391FBF3F176
:106D08006DE000BFE0100020A48E0108602700207D
:106D1800EAAC01083C27002084F8FD3094F8FE30E6
:106D2800624A0133DBB2032B88BF012382F8FE30AD
:106D380094F8FE1042F2107359435D4B1B78D80744
:106D480048BF01319A0748BF02315F07B4F80031E4
:106D580048BF0431D80748BF0A319A0748BF1431E1
:106D68001F0648BF2831D80548BF28315A0748BFF1
:106D780064311F0748BFC831980548BF01F5C8717D
:106D88009A0648BF01F57A71DF0648BF01F5FA6136
:106D9800580648BF01F57A614FF4806001F000FEA3
:106DA800424B002283F8FC20EDE6E16BDFF8FC8023
:106DB80084F8FD3011F0200717D098F8402012F021
:106DC800020F14BF4FF47A71002112F0010F14BFA3
:106DD8004FF4FA6300230B4494F84610194401F069
:106DE800DFFD002384F8FC30CDE6324B1B68190622
:106DF8007FF5C9AE394601F0D3FD88F8FC70C2E6CC
:106E080084F8FD30E36B294F9A067FF5BCAE97F8FE
:106E180040309B077FF5B7AEB7F84430642159433B
:106E280001F0BEFD002387F8FC30ACE684F8FD30A5
:106E380039E0BB7823B1C5F8C06087F80280C4E5A3
:106E4800D5F8C030F31AB3F57A6FFFF4BEAD01235D
:106E5800D5F8C400BB7007F046F80746D5F8C4005B
:106E680007F041F87F067FF4B0AD8A2802D08E285B
:106E78000CD0AAE5EB6B98067FF5A7AD95F8BE3068
:106E8800002B7FF4A2AD05F18D0306E095F8BE3026
:106E9800002B7FF49AAD05F15803C5F8C8302D23AF
:106EA80085F8CC3091E504B0BDE8F087E01000200B
:106EB800223400203C270020084BDA68D10709D487
:106EC800DA68D20608D4DB6813F0040F14BF032075
:106ED80004207047012070470220704700200240BC
:106EE80003788B4286BF024B33F8110000207047AD
:106EF800E811002070B5344C054606F003FFA3697D
:106F0800A061C31AB3F5FA5FE36182BF002384F876
:106F1800203084F8213094F820302BB9A12D02BFFD
:106F2800294A012182F8211094F82110264A31B10A
:106F3800D118EDB2013381F8225082F8203094F84C
:106F4800205094F84330AB423CD11F4B93F8443067
:106F5800052B02D0062B03D02FE000200BF03CFAC3
:106F680094F823301E2B28D100200246C1B26B1E94
:106F780099421ADA214491F822300821DBB283EAD7
:106F88000206F60744BF83F01803C3F3460301F172
:106F9800FF3154BF5B0843F0800311F0FF01C2F3D7
:106FA8004702ECD101301A46E0E7234493F8223037
:106FB8009A4202D103200BF00FFA002384F8213003
:106FC80084F8203070BD00BFE811002010B50446D9
:106FD800B0F900000AF0FFFEB4F902000AF0FBFE67
:106FE800B4F90400BDE810400AF0F5BE10B5044637
:106FF80000680AF0F0FE60680AF0EDFEA068BDE8DF
:1070080010400AF0E8BE2DE9F74F0120FFF750F9CC
:10701800002488B3012C2FD8194E4FF04C0909FBD6
:1070280004FA06EB0A0808F19007BD7815B1013497
:10703800E4B2EEE790F9003090F804E01846114BFE
:1070480003228DE8240001212A4653F82E30FFF749
:1070580005F8834660B106F14800504429464A467F
:107068000EF0A7FF01231C44C8F848B0BB70E4B277
:107078000120FFF703F9CCE703B0BDE8F08F00BFAC
:10708800E8110020B88E010800212A2210B5114805
:107098000EF08FFF104B002219461048105C83F841
:1070A800E80104240520013283F8ED4182424FF0C3
:1070B800000483F8EC0183F8EF4183F8EE0103F153
:1070C8000803EAD10123A1F8EA31522381F8E63115
:1070D80010BD00BF822900209C2700200AAD0108AE
:1070E80010B5FFF7E9FE4FF43024012806D11CB192
:1070F800FFF7E2FE013CF8E7052010BD002C08BFB1
:10710800052010BD70B50646441E14F8011F89B14C
:10711800094D28460EF083FF0028F6D005F1080334
:1071280098423FBF054B401BC018A31B38BF80F8CF
:107138008831EAE770BD00BF2DC301089C270020F5
:107148000120002108F0DCBBF0B5184A92F8E030C5
:10715800D2F8E4701546042B11D807EBC3025E1C65
:10716800941CF6B209D013469288D10705D510426F
:1071780003D008E00131052908D13346EBE785F84B
:10718800E0300020F0BD93F802E00021074C0C220B
:1071980004F1E80C02FB01F31CF803209645E9D141
:1071A800234484F8E060D3F8EC00F0BDE811002037
:1071B80020F01F01012300F01F00024A83408B507A
:1071C800704700BF140401400023036043608360DC
:1071D8008381036143618361C361036243628362A4
:1071E80070478A68036810B50C6A14430A69144327
:1071F8004A6914438A691443CA6914434A6A14439E
:107208008A6A23F4FF4323F0700322431343036085
:107218008B8943600B6883604B68C36010BD02684C
:107228004FF6FE73134003600023036043608360DE
:10723800C360294B984201D1284A27E0284B98423D
:1072480001D1264A2AE0274B984201D1234A2DE052
:10725800254B984201D1214A30E0244B984201D174
:107268001E4A33E0224B984204D11C4A536843F427
:1072780070032EE01F4B984204D1184A536843F01C
:10728800706326E01C4B984204D11C4A536843F0B3
:107298000F031EE01A4B984204D1184A536843F072
:1072A800F00316E0174B984204D1144A536843F48C
:1072B80070630EE0144B984204D1104A536843F4AB
:1072C800704306E0114B984204D10C4A536843F4CA
:1072D80070235360704700BF08000240000002405E
:1072E8001C000240300002404400024058000240A6
:1072F8006C00024080000240080402400004024082
:107308001C04024030040240440402405804024075
:1073180001F0030301F0FC0101F1804101F5803126
:1073280010B59B008C680F229A4024EA02028A60FA
:107338008A68984002438A6010BD0A888B88F0B535
:107348004C880E89CD88C2B9026A22F00102026215
:107358008269016A22F0F3021A4342EA061344F0F2
:10736800010421F00A02144383610462836923F053
:107378000C03836183691D431FE0042A016A1ED13F
:107388004FF6EF720A4002628269016A1B0222F418
:10739800734243EA06332401134344F010044FF6C2
:1073A8005F720A40A4B2224383610262836923F4B4
:1073B80040638361836943EA05258561F0BD082A36
:1073C8001DD14FF6FF620A400262C269076A4FF692
:1073D8000C7111404FF2FF523A4042EA042443EA4A
:1073E80006130B4344F480749BB2A4B2C3610462D5
:1073F800C2694FF6F3731340C361C3691FE04EF6C9
:10740800FF720A400262C169026A40F6FF470F40F4
:1074180045F6FF7111401A0242EA063341EA043484
:107428003B4344F480549BB2A4B2C3610462C26972
:107438004FF2FF331340C3612D02C369ADB21D4340
:10744800C561F0BD036A23F001030362036A70B5E6
:10745800446882690D6822F4803222F07302154371
:107468008A8923F0020313438A881343134A9042FC
:107478000FD002F5006290420BD002F540629042B4
:1074880007D002F58062904203D002F580629042F4
:107498000DD1CA89CE8823F0080313430A8A24F43D
:1074A800407414434A8A23F00403334314438A681C
:1074B800446085614263036270BD00BF002C0140D7
:1074C800994A536803F00C03042B2DE9F04105D0C9
:1074D800082B06D095490160B3B916E0934B0360B9
:1074E80012E053685468C3F38343991CE30349BF0C
:1074F800D36A8F4B8D4C03F00F0344BF0133B4FBA9
:10750800F3F34B43036000E000235168894FC1F354
:1075180003117D5C0168EDB221FA05F444605668F8
:10752800C6F30226BE5D24FA06FEC0F808E05668D7
:10753800C6F3C226BE5DF6B2F440C460D2F82C8011
:10754800C8F3041808F00F0C07EB4C0C18F0100FD8
:10755800BCF810C01FFA8CFC07D0BCF1000F04D097
:10756800B3FBFCFCC0F810C000E00161D2F82CC0ED
:10757800CCF3442C0CF00F0807EB48071CF0100F55
:107588003F8ABFB204D01FB1B3FBF7F7476100E0F1
:107598004161176BFF065ABF644F87618161176BA2
:1075A800BF065ABF614FC761C161176B7F065ABFDB
:1075B8005E4F07620162176BFF0506D5994204D139
:1075C800AE4202D14F00476200E04462176BFF04ED
:1075D80006D5994204D1AE4202D14F00876200E03D
:1075E8008462176BBF0506D5994204D1AE4202D119
:1075F8004F00C76200E0C462176B7F0506D5994249
:1076080004D1AE4202D14F00476400E04464176BD6
:107618003F0506D5994204D1AE4202D14F00876496
:1076280000E08464176BBF0406D5994204D1AE42CA
:1076380002D14B00C36400E08464156B3A4BAD077C
:1076480001D1046315E01C6B04F00304012C01D183
:1076580001630EE01C6B04F00304022C02D14FF40A
:10766800004305E01B6B03F00303032B01D12F4BF1
:107678000363146B2C4B14F4403F02D1C0F834E080
:1076880018E01C6B04F44034B4F5803F01D1416329
:1076980010E01C6B04F44034B4F5003F02D14FF401
:1076A800004306E01B6B03F44033B3F5403F01D1C0
:1076B8001E4B4363146B1C4B14F4402F02D1C0F8CB
:1076C80038E018E01C6B04F44024B4F5802F01D195
:1076D800816310E01C6B04F44024B4F5002F02D140
:1076E8004FF4004306E01B6B03F44023B3F5402F2F
:1076F80001D10E4B8363146B0B4B14F4401F02D162
:10770800C0F83CE020E01C6B04F44014B4F5801F82
:1077180001D1C16318E01C6B04F44014B4F5001FD8
:107728000AD14FF400430EE00010024000127A0024
:1077380000093D00240000201B6B03F44013B3F53F
:10774800401F01D1134BC363126B134B12F4400F4C
:1077580003D1C0F840E0BDE8F0811A6B02F44002A2
:10776800B2F5800F02D10164BDE8F0811A6B02F412
:107778004002B2F5000F02D14FF4004306E01B6B44
:1077880003F44003B3F5400F01D1024B0364BDE895
:10779800F08100BF00127A0000100240F0B500230B
:1077A8000E681C460125A54005EA060EAE452BD1FC
:1077B8000F797A1E012A15D8856803229A4025EA8E
:1077C800020282604D7982689D40154385608288F7
:1077D80092B222EA0E0282808A798588A2402A43E0
:1077E80092B28280032205689A40D2431540056010
:1077F80005689F402F430760C7681740CA7902FA97
:1078080003F547EA0502C2600134102C03F10203B4
:10781800C8D1F0BD38B52DED048B4A4C0368C4F8C7
:1078280024318388A4F82831013A0D46072A42D822
:10783800DFE802F0040A101822292F35B4F82431A1
:107848000B80B4F8263113E0B4F826310B80B4F875
:10785800243105E0B4F824315B420B80B4F82631BA
:107868005B4205E0B4F826315B420B80B4F8243162
:107878006B80B4F828311DE0B4F824315B420B80EA
:10788800B4F8263112E0B4F826310B80B4F824316C
:107898000CE0B4F824310B80B4F8263105E0B4F8D4
:1078A80026315B420B80B4F824315B426B80B4F81C
:1078B80028315B42AB80244B93F83030002B3ED10B
:1078C800B5F9003094ED4E0AD4ED4B7A09EE103A32
:1078D800B5F9023008EE103AB8EEC88AB5F90430A6
:1078E800B8EEC99A28EE000A08EE903AA7EE890A7F
:1078F800F8EEE88AD4ED517AA7EEA80A0EF068FDF2
:1079080094ED4F0AD4ED4C7A288028EE000AA7EEB1
:10791800890AD4ED527AA7EEA80A0EF059FD94ED23
:10792800500AD4ED4D7A688028EE000AA7EE890A3D
:10793800D4ED537AA7EEA80A0EF04AFDA880BDEC54
:10794800048B38BDE811002024000020F8B54A4B0C
:107958004A4C1B68D4F850219A1A002AC0F28B802E
:1079680003F5C333A033C4F8503104F5AE70D4F82E
:1079780058319847424B04F5AE701A780146FFF724
:1079880049FF404B197811F0040F04F5AE751A46FB
:1079980014D0D4F85031C4F8643100233A4818445C
:1079A8000026A0F874613948EE5A1E5206301E525D
:1079B8000233062BF2D121F00401117094F87421DE
:1079C8002E4BAAB13049B3F85C21B1F87401121AF0
:1079D800A3F85C21B1F87601B3F85E21B1F878110B
:1079E800121AA3F85E21B3F86021521AA3F8602195
:1079F800D4F86411214A00293DD0D2F850315B1ADD
:107A080023498B4202F5B47002F5B7711DD8214A9B
:107A1800938A9BB283F008039382002335F81320DE
:107A280030F9137016B2B7424FEA4304C4BF174F78
:107A380027F813200F5FB742B8BF174E03F10103B1
:107A4800B8BFA253032BE9D1F8BD0023134CC2F8E9
:107A5800643130F9135031F913200133032B2A44D0
:107A68004FF0020592FBF5F224F8022FF1D1BDE8A0
:107A7800F84003F005BDF8BD00340020E8110020EF
:107A880023340020201100209C27002050130020C0
:107A98007FC3C90100040048561300200E290020A6
:107AA800104BDFED117A1B689A89104B1B6883F322
:107AB8001003D31A07EE103AB8EEC77A27EE277AE2
:107AC80007EE902AF8EEE77AC7EE277AFDEEE77A16
:107AD80017EE900A6428A8BF642020EAE070C0B2BC
:107AE800704700BF081100200000C842181100208C
:107AF800094B1A68137844F6FB7103EB431300FB38
:107B080003135078C0EB0030B3FBF0F39078B3FB6D
:107B1800F0F080B2704700BF0811002008B50A488D
:107B280090F8763100EB43030A22B3F8861189B244
:107B3800A0F88E1100F5C87006F0DEF980B2FFF7E4
:107B4800D7FF024B188008BDE81100200C11002057
:107B5800426A806A131A5842584170474171704707
:107B680043799B070AD5436A8269D154436A0169FC
:107B78000133B3FBF1F201FB12334362704707EEA6
:107B8800900AF8EEE77ADFED0C6A9FED0C0AF5EE45
:107B9800C07AF1EE10FAD4BFB1EE677AC7EEA67AD2
:107BA80008B5D8BFC7EE267A27EE800A03F014F985
:107BB800034B83ED000A08BD8096184B35FA8E3CBE
:107BC8007800002038B50D4B0D4D1A8A0D4B1968F9
:107BD800498811421C4603D006F094F8286007E053
:107BE80006F090F82B68984282BFC01A064B1860BE
:107BF80023685868BDE83840FFF7DABA000400483F
:107C0800001400208C0700200400002003460A46C8
:107C180090F84602D96A9B7902F0C2BB437913F007
:107C2800010310B504460DD001F090FF58B1236A46
:107C38006269E168D05C0133B3FBF1F201FB1233F6
:107C4800236210BD184610BDF8B59B4B1B6804464F
:107C5800187818B1012800F068819BE2242C974D10
:107C68000CD006D80A2C00F0D9800D2C00F0D68054
:107C780046E12A2C06D02C2C04D041E128716871E9
:107C8800A8714EE18E4B69792F798C4A002058549F
:107C98002FBB1978D771472921D1597850291ED17E
:107CA8009978472907D1D978472904D119794129E1
:107CB80001D10121D1719978814A522903D1D17812
:107CC8004D2900F0918299787D4A472907D1D178CA
:107CD800532904D11279562A04BF0322EA71EA799A
:107CE800764E022A39D0032A4CD0012A40F08580EA
:107CF800BA1E072A00F28180DFE802F004080F1399
:107D08001A257F2A09F09AFBA86076E01B78532B86
:107D180073D1AB685B42AB606FE009F08FFBE86042
:107D28006BE01B78572B68D1EB685B42EB6064E033
:107D38001B78302B634B1A788CBF42F0020222F07A
:107D480002021A7059E0002009F0D8FB287454E0A8
:107D5800002009F0D3FB68824FE0072F06D0082FD8
:107D68004BD1012009F0CAFBF08246E0012009F05E
:107D7800C5FB41F2184358434FF47A73B0FBF3F054
:107D8800B0823AE0022F07D0032F0AD1002009F071
:107D9800B5FB4D4B187030E0002009F0AFFB307692
:107DA8002BE02AD93A1F9210337E0132D2B2013B1E
:107DB80002EB8303DBB2102B1FD8F91EC2F10102BC
:107DC80001EB8202D2B2012A0BD0042A11D1002081
:107DD8005E1E09F093FB3D4B98553D4B00229A558A
:107DE80007E05E1E3B4A0020935509F087FB3A4B9B
:107DF80098553A4A136801331360304B2A2C18BF40
:107E08009A7907F101074FF000000CBF0122544096
:107E18002F7168710CBF5A769C7182E0687E0028C9
:107E280047D02F4B13F8012D2E495A708B42F9D1A8
:107E3800234A224C13785278402B85BF373B1B01CD
:107E48001B01DBB298BF03F0F003402A8CBF373A1E
:107E5800303AD2B21344AA79DBB29A4226D121230E
:107E68000B702149E0790B681E4A013301280B6029
:107E78000AD002281CD1722313701C4BA28A1A80C4
:107E88001B4BE28A1A8013E0672313700D4B1B7893
:107E98009F070ED5174BA2681A60E2685A60164B06
:107EA800227C1A70154B628A1A8002E03F230B70FD
:107EB800002000236B7634E0B00700200014002077
:107EC800682700202011002070100020A110002039
:107ED800911000207110002081100020A4150020AE
:107EE800D0020020BC020020B01500202211002082
:107EF80058100020281100202611002024110020ED
:107F08006B79687E0E2B9FBFA34A591C5171A34AF7
:107F180098BFD454A04A18B993795C40947100E092
:107F28000020003018BF0120F8BD9B4B997E00222D
:107F3800082900F22F81DFE801F0050B0F15202B2F
:107F480048606A00B52C40F02581DA7601223AE0D3
:107F5800622C08BF022236E003229A761C775C77EF
:107F68009C7717E104229A765A7F997FDC7722441E
:107F7800D2B25A770A449A770CE105229A765A7F48
:107F8800997F1C842244D2B25A770A449A7701E135
:107F980006229A765A7F997F2244D2B25A770A44A7
:107FA8009A771A8C02EB0424A4B2B4F5AC7F88BF8C
:107FB800794A1C8484BF0121D17600225A84002C7E
:107FC80040F0E88007229A76E4E05A7F997F2244BD
:107FD800D2B25A770A449A775A8CB2F5AC7F3CBF32
:107FE8006D49891802F1010238BF81F82440198CC3
:107FF80092B291425A84E5D9CCE008229A765B7F06
:10800800A34200F0C780644B0122DA760DE0644D8C
:108018009A7615F8012D6A70624A9542F9D1997FCE
:108028005D4AA14206D03F232B705F4A5368013353
:108038005360AFE05D48016801310160D07E10B146
:108048003E232B70A6E021212970D17F062941D03B
:1080580004D8022907D0032923D0F8BD122959D002
:10806800302967D0F8BD502129705149946A4C6075
:10807800D46A0C60516B4FF47A7491FBF4F14D4C57
:10808800218092F87C114C4A19B1117841F0020113
:1080980002E0117821F002011170012283F87D219C
:1080A80069E05321297092F82910CE0705D592F876
:1080B8002820D51E6A426A4100E0024602F001010A
:1080C80083F87C11002A56D13B490A7822F0020233
:1080D8000A7050E04F21297092F82F10CC0705D56F
:1080E80092F82E20D11E4A424A4100E0024602F090
:1080F800010183F87C1122B92F490A7822F0020283
:108108000A702E4A93F8531011702D4AB3F8501084
:10811800118030E0562129702A49946B0C8042F274
:108128001074D16B91FBF4F1274C2180012182F866
:108138007E1120E04921297092F82810234A10293D
:1081480088BF10211170224914780022A2420ED251
:10815800204D0E7A5655204D4E7A56551F4DCE7AE3
:1081680056551F4D11F80C6F56550132EEE71D4953
:108178000A6801320A6093F87D31074A002B3AD029
:1081880092F87E31BBB3002182F87D1182F87E110E
:108198001846F8BD0020F8BD00140020682700200C
:1081A800D0020020BC02002090070020B01500205B
:1081B8002811002024110020201100202611002061
:1081C8007E0000202211002058100020701000208E
:1081D800241400207110002081100020911000202C
:1081E800A1100020A41500201279432A7FF46BAD5A
:1081F8000222EA7167E5F8BD0449054B0968187061
:1082080000225A6199611A77704700BF60270020E1
:108218009007002010B5121A07EE902A5B1A2DED70
:10822800028BF8EEE78A07EE903A184B059CB8EEF9
:10823800E78AD3ED007A28EE278A28EE080AA8EE06
:10824800A80A0EF06BFBDFED127A049B20EE270ADA
:10825800F0EE480ABCEEC00A83ED000AB1EE680AE7
:108268000EF0B8F9DFED0B7A9FED0B7AE0EE077AA6
:10827800BDEC028BFDEEE77A17EE903A002BBCBFFF
:1082880003F50C43A033236010BD00BF7800002025
:108298002C7D8E3F00A00C46A00CB34544F25063E1
:1082A800984203DDA0F50C40A0387047034B984274
:1082B800BCBF00F50C40A030704700BFB0B9FFFF4D
:1082C80073B51A4C036823600B686360184D006827
:1082D800184EFFF754FC184B009395E8030094E8F8
:1082E8000C000196FFF796FF144B32681A60686815
:1082F800636813491B1A07EE903A124B286893EDEE
:10830800007A23681B1A0B600F4BF8EEE77A1A60A5
:108318000E4B67EE877A1B68FDEEE77ADA880C4B1E
:10832800C1ED017A1A8002B070BD00BFCC260020D2
:1083380028110020D8260020D42600201427002049
:10834800DC260020780000200C270020600F002089
:10835800082700204279DFED2A5A2A4B9FED2A5A36
:1083680007EE902AF8EE677AC27BC7EEA57AB2EEDE
:10837800047AC3ED007A07EE902AF8EE677A234A6A
:10838800DA60C7EEA57AC3ED017A8179204B07EE52
:10839800901AF8EE677A017CDA60C7EE877AC3ED47
:1083A800007A07EE901A817E06EE101AF8EE677AC8
:1083B800B8EE466AC7EEA57A86EE056AC3ED017A7D
:1083C80083ED026AC179134B06EE901A417CDA609C
:1083D800F8EE666AC6EE876A07EE101AC17EC3ED2C
:1083E800006A07EE901AB8EE477AF8EE677A87EED9
:1083F800257AC7EE857A83ED017AC3ED027A704754
:108408000000C842E426002000007A440000FA4434
:10841800F42600201827002010B50C4C23789B0761
:1084280013D50B4B1B78042B0FD90A4A0A4B10683B
:1084380052685A601860FFF7A2FB084B1A88084B6D
:108448001A80237843F00103237010BD2011002007
:1084580026110020281100205C100020F8100020B0
:1084680028270020044B1A78044B0AB1044A00E07C
:10847800044A1A60704700BF3227002038270020BE
:108488000000A0410000A0C11C4B1B681B0307B5DE
:1084980030D51B4A1B4BD2ED007A1B788DF8003083
:1084A800B2EE047A67EE877A174B9FED187A1B783D
:1084B8008DF80130FCEEE77A0A2017EE903AD2EDFB
:1084C800017A8DF8023067EE877A6946FCEEE77A22
:1084D80017EE903AD2ED027A8DF80330FCEEE77A87
:1084E80017EE903A8DF80430094B1B788DF805305B
:1084F80003F0C4FB03B05DF804FB00BF3C27002079
:10850800502700202E2700204C27002000007A4406
:1085180032270020054A137883F001031370044AB8
:1085280000231360034A1360AEE700BF3227002020
:108538004827002044270020094A13781844C0B26D
:1085480010F0800F18BF803810701346054A19784C
:108558001378994201BF00231370014A13707047C2
:10856800752F0020742F002010B50A4B0A4A1B787B
:1085780042609C18094A046012789A4225BFD31AAF
:108588000B60C3F1800300232EBF4B600B604A6071
:1085980010BD00BF752F0020762F0020742F0020FB
:1085A8001FB5684602A9FFF7DFFF044B02981B6856
:1085B80003440398184405B05DF804FB280600201E
:1085C8002DE9F04F89B0824601930023029103926E
:1085D8009946039A934205DA029A52F82320013306
:1085E8009144F6E7019B4D46002B56D101F092FFCE
:1085F800002852D101987CE002223F4E8DF81C20C1
:108608001A0C4FF480578DF81D2006201A0A8DF891
:108618001E208DF81F3001F0A1FF3785062008F0D5
:108628009FFC364BB76101221A700020378507A9D5
:10863800042208F0BDFC029FD04626464FF0000BEE
:10864800039B9B451EDABC4657F8042B4FEA8B0365
:10865800002A47D0B24235D332465AF80310CDF833
:1086680014C00020049308F0A3FC049BDDF814C098
:108678005AF8032032444AF80320DCF800309E1BE5
:10868800CCF800601C4B4FF480529A611C4A136866
:108698002D1B1C44019B14604BB345B3184B1B683E
:1086A800DCB22A19B2F5807F164AD2688CBFC4F5AD
:1086B80080742C4693429FD3134A00231370134AA5
:1086C800137014E00020D8F8001008F071FC57F877
:1086D800043CD8F80020F61A1344C8F800300023E8
:1086E80047F8043C0BF1010B08F10408A8E7C5EBB7
:1086F800090009B0BDE8F08F0004004825060020F5
:108708002806002010000020742F0020752F00205C
:1087180030B50B4C0B4D22782B789A4285B00CD093
:10872800684602A9FFF720FF0123684602A9022232
:10873800FFF746FF00232B70237005B030BD00BF44
:10874800752F0020742F002030B50E4D0E4C2A785E
:1087580023789A4285B011D0684602A9FFF704FF32
:10876800002302A902226846FFF72AFFFFF7E4FE6A
:1087780020782B781B1A5842584100E0012005B098
:1087880030BD00BF752F0020742F002038B50E4C67
:108798004FF4805545F2082001F0E0FE25850620BB
:1087A80008F0DEFB094BA56101221A70C720258558
:1087B80008F0D6FB064AA56100231370054A13701A
:1087C800054A136038BD00BF000400482506002094
:1087D800742F0020752F002028060020FFF7F2B91B
:1087E800FFF7F0B9FFF7EEB930B50028104C114A81
:1087F800B8BF40423C2590FBF2F304FB03006843FA
:108808000D4D90FBF2F22D682D7B25B903EB830308
:1088180003EB830301E0C3EB031302EB83030B8039
:1088280004FB02024FF47A7392FBF3F24A8030BDE4
:10883800806967FF8096980010110020022803D0F5
:10884800431E584258417047064B1B681B7823B19A
:10885800054B1868C0F3C0407047044B1878C0F344
:1088680080007047FC050020F40F0020223400200F
:10887800A0F17D03012B70B504460D460A4E05D8BC
:1088880030687D2105F035FB84F0200430682146EE
:1088980005F02FFB35B12B881C4404EB142404F09D
:1088A800FF042C8070BD00BFD011002010B50A4C09
:1088B8005E280146206805D15D2105F01AFB206875
:1088C8003E2105E05D2903D105F013FB20683D2119
:1088D800BDE8104005F00DBB8015002037B51A4BD8
:1088E8001A4C1B491B4A20B11B480088B0F5805F11
:1088F80021D2164D09881278ADF804108DF806209B
:108908009B798DF8073001A8291D04220DF036FB4C
:10891800C0B101986860532009F01CFAA08809F0DA
:108928004BFAA07909F048FAE07909F045FA0A4BC0
:1089380000221A8006E0098812789B79A180A2712A
:10894800E371E8E703B030BDF03300208015002064
:10895800E011002020110020C03100202DE9F8434B
:108968000E4B93E8800305460E460024B44213DA02
:108978007B1933F9140008EB050333F9142009EBCC
:10898800050333F914301344022293FBF2F3C01A9F
:1089980009F021FA0134E9E7BDE8F8831C3000202A
:1089A80030B585B004AC002524F8025D0091ADF81F
:1089B800060021461020FFF75BFF9DF806002146C0
:1089C800FFF756FF9DF807002146FFF751FF9DF876
:1089D80000002146FFF74CFF9DF801002146FFF7F4
:1089E80047FF9DF802002146FFF742FF9DF803006C
:1089F8002146FFF73DFF9DF80E00C043C0B229464F
:108A0800FFF736FF05B030BD10B5054C206805F0FE
:108A18006DFA18B1206805F066FAF6E710BD00BFD8
:108A2800A411002010B50446C0B2FFF73FFFC4F3FD
:108A38000720BDE8104039E7024B5E21186805F0B1
:108A480058BA00BF8015002038B5064C05465E218F
:108A5800206805F04EFA20682946BDE8384005F040
:108A680048BA00BF8015002013B5044601A9006864
:108A7800FFF7BAFE1320FFF7E7FFBDF90400FFF781
:108A8800D1FF1B20FFF7E0FFBDF90600FFF7CAFF83
:108A98002320FFF7D9FF2368002BB4BF53204E20B3
:108AA800FFF7C0FF01A96068FFF79EFE1220FFF7DD
:108AB800CBFFBDF90400FFF7B5FF1A20FFF7C4FF8D
:108AC800BDF90600FFF7AEFF2220FFF7BDFF636880
:108AD800002BB4BF57204520FFF7A4FF02B010BDFC
:108AE800674B73B51878674DFFF7A8FE2B7883425C
:108AF800044620D0C8B1644B1B68E3B193F9000069
:108B080002230093614B1B685B78003318BF012375
:108B1800019304214FF416530022FDF79FFA5C4B92
:108B2800186040B101232B7005E0594E3068FDF7FD
:108B380082FA34602C70574B574D1878FFF77EFE39
:108B48002B788342044618D088B1544B1B68A3B1D4
:108B58000022012493F9000000944FF496430192F7
:108B68000821FDF77BFA4E4B186028B905E04C4EFA
:108B78003068FDF760FA34602C704A4B4A4D18781B
:108B8800FFF75CFE2B78834204462E4642D000282D
:108B980037D0464B1A68002A3CD0D37992F90000A6
:108BA800434C002B08BF022302220092002254F8F3
:108BB800233001921021FDF751FA3E4B054618600B
:108BC80040B33D4C94F84A30022B0BD094F89620D1
:108BD800022A01D14C3405E023B1002A04F14C04E7
:108BE80018BF0024354B1C6044B1204600214C229C
:108BF8000DF0DFF90223256084F84A300123337031
:108C080008E02C4E306806F02DFE3068FDF713FAA8
:108C180034602C702A4B2B4D1878FFF70FFE2B78F9
:108C28008342044629D000B3274B1B682BB3274A3D
:108C380093F9000012685278002A0CBF0822092212
:108C48000323009301924FF4614320210022FDF792
:108C580005FA1F4B186080B11E4A012313702B7050
:108C68001D4B1A681D4B1A6007E0194E3068FDF756
:108C7800E2F9184B34601C702C7002B070BD00BF54
:108C880004060020E010002000060020101100203B
:108C9800801500200C060020301100200806002056
:108CA800A411002018060020B61100201406002088
:108CB800B88E0108B811002030120020BC11002025
:108CC80024060020CC110020200600201C060020CD
:108CD800D0110020D411002060270020D8110020D6
:108CE8002DE9F743934C05F00DF8A368C31A002B40
:108CF800C0F2628300F5433303F5A073A3608E4B83
:108D08001D78237BC5F38005EB1A18BF0123257353
:108D18004DB1002B00F05083884B5A789A7001228D
:108D28005A701A702BE0854A2BB1D37843F00203AE
:108D3800D37093785370D67806F0020101F0FF03E0
:108D480039B97E498968411A002903DB06F0010315
:108D580000E0012303F00107784917707BB1F2079F
:108D68000DD50A790132D2B20523B2FBF3F303EB36
:108D78008303D31ADBB2724A0B71D35C4B706F4E0C
:108D8800DFF8088233787BB3F37823F00203F370BB
:108D98006C4B0344AE20B36001F03FFC08B101F016
:108DA80041FC88F80000002800F00683B02001F09C
:108DB80034FC402001F031FC002001F02EFC102092
:108DC80001F02BFC4FF48067013F0020BFB201F097
:108DD800FBFB002FF8D1384601F093FC72785A4B10
:108DE80053F8220001F010FC98F80030002B00F036
:108DF800E3827378062B00F2B482DFE813F00700F1
:108E0800B202180078006D018A01EF014F49504AFB
:108E1800504B514801F039FF012001F072FC4E48D7
:108E280001F0F2FB022001F06CFC4C48AFE14C4F22
:108E38003B689B0735D5DFF85881DFF85891B8F8BB
:108E4800001045480A23B1FBF3F203FB121399F80B
:108E58000010009192B243499BB201F016FF02F054
:108E680055FB012001F04DFC3B4801F0CDFB3E4B8A
:108E780099F800201868B8F80030067906FB123116
:108E880064234B43C1788E1B56430220B3FBF6F68E
:108E9800F6B201F036FC3146152002F0FBFA032643
:108EA80000E001263B681F0540F15B822F4B3049EB
:108EB8001F680968009164232E4997FBF3F226483E
:108EC80003FB127301F0E1FE02F020FB304601F0D3
:108ED80018FC214801F098FBFEF7E2FD0746701CDC
:108EE80001F00FFC1520394602F0D4FA39E20120CE
:108EF800214F01F006FC214801F086FB3B689807EA
:108F08004AD51F4A1448B2F90210B2F9003000914C
:108F1800B2F904201B4901921B4A01F0B6FE02F087
:108F2800F5FA022001F0EDFB0B4801F06DFB03267A
:108F380033E000BF80150020223400209820002054
:108F48000FAD0108404B4C00D88E010814AD010844
:108F58001DAD0108E1A601088D15002024AD01080A
:108F68003C2700202FAD0108081100201411002013
:108F78001811002047AD01081C1100205CAD010844
:108F8800EA10002072AD010881AD010871020020CD
:108F98000C1100207D00002002263B68D9071AD555
:108FA8007C4A7D48B2F90210B2F900300091B2F95A
:108FB80004207A4901927A4A01F067FE02F0A6FA83
:108FC800304601F09EFB744806F1010801F01CFBD5
:108FD8005FFA88F846463B681A0718D5714A6E4802
:108FE800B2F90210B2F900300091B2F904206B49CD
:108FF80001926D4A01F049FE02F088FA304601F00C
:1090080080FB6548771C01F0FFFAFFB23E46674ACD
:109018006249B2F90030B2F902200092644A5E480F
:10902800B2F900200192634A634F01F02EFE02F06C
:109038006DFA304601F065FB574801F0E5FA97ED07
:10904800000A554801F0B6FC53480CF0F6FF06F14B
:1090580001085FFA88F8C0B2B946092809D8431C44
:109068002044DBB220224273E21800219173184693
:10907800F3E7494F99ED010A384401F09BFC02F0EF
:1090880045FA404601F03DFB384601F0BDFA99ED3E
:10909800020A384601F08EFC38460CF0CEFF023644
:1090A800F6B2C0B2092809D82318421CD2B220212E
:1090B8005973A318002199731046F3E73F4AB2F990
:1090C800003000EE103A3844B8EEC00A01F072FCE5
:1090D80002F01CFA304657E00026394F3B78B3427D
:1090E80040F23F810E2E00F03C817008013001F003
:1090F80008FB304608F028FA3B78B34206D920200E
:1091080001F067FA701CC0B208F01EFA0236F6B217
:10911800E3E72C4E2C4996F8A8271F4801F0B5FD27
:10912800012001F0EEFA1C4801F06EFA274B28499D
:109138001F7819483A4601F0A8FD022001F0E1FA2B
:10914800154801F061FA0C2303FB0766214996F8DC
:10915800AB2796F8AA37104801F097FD02F0D6F928
:10916800032001F0CEFA0C4801F04EFA96F8B01739
:1091780096F8AE2796F8AF3707480091164901F0E0
:1091880084FD02F0C3F9042001F0BBFA024801F0A3
:109198003BFAE6E0141000208D15002072AD01089E
:1091A80085AD01084413002029C301083427002095
:1091B800F810002089AD010828240020342400205C
:1091C8004C3300209C2700208DAD0108E0240020AE
:1091D80099AD0108AAAD0108BBAD0108784B1B6821
:1091E8001B0640F1BA80636AA16A764A8B421FBFA8
:1091F800936292F82C30013303F003034FF001011E
:109208004FF0000018BF82F82C3001F086FA94F86D
:109218002C306D4AD05C01F0DCF90220012101F00C
:109228007CFA0026694B9B5D3620C3EBC30393FB96
:10923800F0F0C0B2062828BF06206038C0B2013658
:1092480001F0C7F9102EEDD1614B62491B786248D5
:1092580013F0020F614B1A7814BF59234E2301F003
:1092680014FD02F053F9022001F04BFA5A4801F0BC
:10927800CBF95B495B4B4E680A68574892FBF3F29F
:10928800594996FBF3F301F000FD02F03FF9032082
:1092980001F037FA5048554E01F0B6F9544B55498C
:1092A8001A884D4801F0F1FC02F01DF9042001F084
:1092B80028FA494801F0A8F94F4B50491A884648FE
:1092C80001F0E3FC02F00FF904210A2001F025FA6D
:1092D800414801F099F94A49226B3F4801F0D5FC11
:1092E80002F001F9052001F00CFA3B4801F08CF975
:1092F8007268B3684349384801F0C7FC02F0F3F8D4
:1093080005210A2001F009FA334801F07DF9336993
:10931800F2683D493048D21A01F0B7FC02F0E3F890
:10932800062001F0EEF92C4801F06EF9B2683749D1
:10933800294801F0AAFC02F0D6F806210A2001F01B
:10934800ECF9254801F060F93149234815220CF061
:10935800A1FE02F0C8F8072016E7F37843F00203ED
:10936800F3704DBB2B4B9B79032B9BBF2A4A9B1851
:109378003F251D7F0021122001F0CFF9284601F07A
:1093880028F91320002101F0C8F9244B1B78002B81
:1093980014BF5220212001F01CF91420002101F0F3
:1093A800BCF994F83450084B585D013505F00305B5
:1093B80001F00FF984F8345003B0BDE8F08300BF22
:1093C8003C27002080150020CDAD0108A110002009
:1093D80020110020D2AD01088D1500202611002093
:1093E8002811002080969800E3AD0108900700201E
:1093F80022110020F0AD010858100020F8AD010836
:10940800FFAD010806AE01080FAE010816AE01084F
:10941800BC020020F0330020D88E01084E33002013
:10942800026BC168034610B5406942B11A6C8C1AC8
:10943800013A005D08BF0A46C0B21A6410BD1A6A34
:10944800805C01328A4228BF0022C0B21A6210BD75
:10945800436B13B190F844007047836A406A1B1A43
:10946800584258417047036B13B15B68016C01E0C7
:10947800C369016A8B423CBFC2689B18581AC0B2C4
:109488007047836A8169426B1944D160416A994285
:109498009DBF0169CB1A5360CB1A96BF0023536056
:1094A80083624FF0000380F84430136888BF8162FC
:1094B80043F0010313607047436A8269D154436AD9
:1094C80002690133934228BF00234362436B1BB1F7
:1094D8001B68DB0705D4D4E7026D136843F08003EB
:1094E80013607047F0B5046D8668236823F00103A4
:1094F80023608379054613F0020F40790CBF4FF0C3
:10950800000E4FF4005E13F0040F14BF4FF4806791
:10951800002710F0010F14BF0421002183072068E1
:1095280020F001002060626822F440524EEA0202F4
:109538006260226822F4B05323F00C0348BF41F064
:1095480008013B430B432360A36895B023F44073A1
:10955800A3606846FDF7B4FF284B9C4201D10C9BE1
:109568000EE0274B9C4201D10D9B09E0254B9C4204
:1095780001D10E9B04E0244B9C420CBF0F9B109B17
:109588002268A879170448BF5B00B3FBF6F206FB14
:109598001233B3EB560F236828BF01321E0441BFB4
:1095A8004FF6F073C2F34201134041EA03026B79AC
:1095B80092B213F0020FA28100F0010114BF4FF420
:1095C80000320022DC0748BF42F480322B6D11B113
:1095D80059680A4302E0596821EA02025A609A6807
:1095E80001074CBF42F0080222F008029A601A688C
:1095F80042F001021A6015B0F0BD00BF003801400A
:109608000044004000480040004C0040417169E7B8
:10961800816067E7026D036B70B50446D5699BB935
:10962800A90611D5C36A1BB1908C80B298470BE08C
:10963800E169928C40694E1CD2B2E6614254E169FC
:10964800E268914228BFE361616BA1B92A0612D58D
:10965800636AA26A9A42236D09D0501CA669A06267
:10966800B25C1A852369984205D3A16203E01A689F
:1096780022F080021A602B0742BF236D08221A626B
:1096880070BD0D4B0D484FF400525A600C4A1168DA
:109698004FF6FE730B401360426B11684FF6FE7372
:1096A8000B401360426A836A9A4200D0E9E60123BC
:1096B80080F84430704700BF000002400C260020AC
:1096C800440002402DE9F0471E46A64B8CB0984254
:1096D800894690469DF8505040F08580A24BA34A99
:1096E8001A60A34A5A6102F580729A614FF4807237
:1096F800DA601A619F4A1A63143A5A63A2F548421B
:10970800203ADA6404329A64C3F8088018659A4BE0
:109718009A6942F480429A615A6942F001025A6198
:1097280002238DF80830032315F0010A8DF809305B
:109738004FF000038DF80A3014BF022301232C07D1
:109748008DF80B3019D54FF090444FF400770197FE
:109758008AF001038DF80A30636A23F0F00363622C
:10976800636A43F070036362204601A9FEF716F8A6
:10977800BAF1000F27D1A76125E0B00710D50CA9D1
:109788004FF4007341F82C3D4FF09040436A23F0AA
:10979800F0034362436A43F070034362FDF7FEFF40
:1097A800F10710D50CA94FF4806341F82C3D4FF018
:1097B8009040436A23F470634362436A43F4E0636E
:1097C8004362FDF7EBFF0E238DF8003000220123E2
:1097D80068468DF801308DF802208DF80330624C10
:1097E80007F01CFC0BE1654B984276D1644B5F4A4D
:1097F8001A604FF48072DA601A61624A5A6102F59F
:1098080080729A615C4AC3F808801865D36943F48A
:109818000033D36102238DF80830032315F0010AC1
:109828008DF809304FF000038DF80A3014BF022379
:1098380001232A078DF80B3019D54FF090444FF4C7
:10984800804701978AF001038DF80A30636A23F094
:1098580070636362636A43F0E0636362204601A950
:10986800FDF79CFFBAF1000F27D1A76125E0B307E8
:1098780010D50CA94FF4804341F82C3D4FF090408F
:10988800436A23F070634362436A43F0E0634362D0
:10989800FDF784FFF70710D50CA94FF4004341F8F2
:1098A8002C3D4FF09040436A23F070434362436A73
:1098B80043F0E0434362FDF771FF26238DF8003043
:1098C8000022012368468DF801308DF802208DF8BA
:1098D80003302B4C07F0A2FB91E02B4B984240F051
:1098E8000F812A4B214A1A604FF48072DA601A619C
:1098F800274A5A6102F580729A611F4AC3F80880A4
:109908001865D36943F48023D36102238DF80830A6
:10991800032315F0010A8DF809304FF000038DF884
:109928000A3014BF022301232C078DF80B3033D5DE
:10993800184C4FF4806701978AF001038DF80A30BC
:10994800636A23F470636362636A43F4E063636287
:10995800204601A9FDF722FFBAF1000F40D1A76107
:109968003EE000BF003801400C260020F88E0108B8
:10997800B815002058000240001002400044004082
:10998800B8250020B81700200048004064250020B2
:10999800B819002000040048B0070FD50CA94FF4EF
:1099A800806341F82C3D5848436A23F4706343624E
:1099B800436A43F4E0634362FDF7F0FEF1070FD515
:1099C8000CA94FF4006341F82C3D4F48436A23F437
:1099D80070434362436A43F4E0434362FDF7DEFEAB
:1099E80027238DF800300022012368468DF80130C6
:1099F8008DF802208DF8033007F010FB434CC4F8B3
:109A08002C900027012384F844302762E761A7627D
:109A180067626671C4F80880A5712046FFF762FD89
:109A2800F20734D5236B002B2AD001A8FDF7CCFB15
:109A3800E36C01934FF480530A9380230693E36801
:109A4800ADF8103020230993206B636902930B97BC
:109A58000597079708970397FDF7E1FB01A9206B86
:109A6800FDF7BFFB236B216D1A6842F001021A60F3
:109A78008A6842F040028A605B689BB2236406E011
:109A8800236D20221A621A6842F020021A60B30776
:109A98002FD5636B43B301A8FDF796FBA36C019325
:109AA8004FF480530A93802306932369ADF810304E
:109AB80000251023606B03930B9505950795089572
:109AC8000995FDF7ACFB606B01A9FDF78AFB636B99
:109AD8001A6842F002021A60226D5D605D60936848
:109AE80043F08003936004E0226D136843F0800321
:109AF8001360226D136843F001031360204600E0F1
:109B080000200CB0BDE8F087000400486425002060
:109B18001FB50123ADF808300023ADF80C30ADF8BF
:109B28000A30094BADF804101B78ADF80620012B5C
:109B380008BF032301A908BFADF80C30FDF7FDFBF2
:109B480005B05DF804FB00BF24010020437913F041
:109B580001031FBFC36803F1FF32C369006A1DBF59
:109B6800181A1040C0B21846704790F83B3210B52A
:109B78007BB990F83A3290F83942A34209D2B0F84A
:109B8800401201229A400A430133A0F84022DBB276
:109B9800F3E710BD8379DB07D0F8343144BFB1FA5D
:109BA80081F149095A681B8909B193617047138586
:109BB80070476E4B6E4A9FED6F7AD2ED007ADFEDFB
:109BC8006E4ADFED6E3A30B51C88B3F90AE01D8A9B
:109BD80006EE904AB8EEE76AF8EE666ADFED687A54
:109BE800B3F9044067EEE67AB7EE004AE6EE077A84
:109BF8009FED647A67EE666A9FED637AE6EE076A20
:109C080027EEA77A07EE904AB3F902409FED5F6A04
:109C1800F8EEE77A67EE277A07EE104AB8EEC77AC9
:109C2800DC89E6EE877AB6EE007AFDEEE76A87EE23
:109C3800866AC3ED066AF8EEE66AD2ED017A9A8979
:109C4800E6EE874A06EE90EAB3F908E09FED507A0F
:109C580005EE90EAF8EEE66AF8EEE55A66EEA46AD2
:109C680065EEA45A66EEA46AB3F806E0E6EE875AF3
:109C780065EE875AA5EEA34AF0EE445A04EE10EAC0
:109C8800B8EE444A25EE844AB5EE404AF1EE10FAA1
:109C98005BD02DB205EE905A24B224EEA45A07EEFA
:109CA800104AF8EEE55A12B265EE255AB8EEC75AD0
:109CB80065EEA35A64EE854AB0EE007AE4EE875A60
:109CC800B5EE007A65EE875A07EE102AB8EEC75A45
:109CD8009FED307ADFED306AB3F91620E5EE075ACA
:109CE800F8EEE77A9FED2D7A76EEE77ADFED2C6ACB
:109CF800E5EEC77A05EE902AB0EE677ADFED297AAD
:109D0800B3F91420B3F9123067EE277A07EE102A58
:109D1800C7EE847AF8EEE55AB8EEC77A65EEA75A28
:109D280027EE877A65EEA75A27EE237AA5EEA67A5C
:109D3800F0EE476A07EE103AB8EEC77A36EE877A41
:109D4800DFED196AE7EE267A01E0DFED187A18B13F
:109D5800FDEEE77AC0ED007A31B1FDEEC67A6422F5
:109D680017EE903A53430B6030BD00BF90020020BD
:109D7800B81B00200000003700007AC70000003838
:109D8800000000390000803A000080380000A0453B
:109D9800000000360000804700008049000080393C
:109DA800000000300050C3450000803D0000000066
:109DB800704770471FB50123ADF80830ADF804109F
:109DC800002301A9ADF80A30ADF80C30ADF8062033
:109DD800FDF7B3FA05B05DF804FB38B5A0F51374C8
:109DE8006379A579DB0744D594F8383205F0010585
:109DF800EBB1226B1068C36A5B08436294F83C328B
:109E080023B1B4F842320133A4F84232917A6A009D
:109E1800FFF7D0FF012384F83B32002384F839325E
:109E280084F83A3284F83832A4F8403238BD94F8CD
:109E38003B32012B04BF94F8393284F83A32204679
:109E4800FFF793FE94F83B22236B3AB9012284F87A
:109E58003B221868997A05FA02F207E0002284F892
:109E68003B2295421868997A08BF0222BDE838401B
:109E7800A0E738BD10B5A0F5127494F83C22BAB921
:109E8800A36A616A994228D0591CA069A162C35C7F
:109E98002069DBB25B0043F400738142A4F83E32D0
:109EA8004FF00A0384F83D3228BFA262012312E072
:109EB80094F93D327BB1B4F83E124B08A4F83E3217
:109EC800204601F00101FFF765FE94F83D32013BA1
:109ED80084F83D3201E084F83C3294F83832002BA3
:109EE8004ED194F839320133DBB2092B84F8393278
:109EF80003D12046BDE8104037E60A2B40D194F83C
:109F08003B322BB9B4F8403243F00103A4F8403295
:109F18006379D9071CD5B4F84002820501D4C30778
:109F280005D4B4F844320133A4F8443210E0E36AAB
:109F3800C0F347000BB198470AE0E3696269D0545F
:109F4800E369E1680133B3FBF1F201FB1233E3612A
:109F5800012284F8382294F83B220023012A84F84D
:109F680039320DD1A27984F83B32236B12F0010FFC
:109F78001868997A0CBF02220022BDE8104019E740
:109F880010BD7620F421312203F076BC13B50622E9
:109F980004466B4603211E2003F0F2FB9DF80020C7
:109FA8009DF801309DF8021043EA02231BB21B4AB8
:109FB80007EE903A92ED007AF8EEE77A67EE877A44
:109FC80092ED027AFDEEE77A17EE903A23809DF83B
:109FD800033043EA01231BB207EE903AF8EEE77A22
:109FE8009DF8041067EE877A92ED017AFDEEE77A24
:109FF80017EE903AA3809DF8053043EA01231BB27F
:10A0080007EE903AF8EEE77A67EE877AFDEEE77AA0
:10A0180017EE903A638002B010BD00BF58000020D0
:10A0280007B5F7216B460622762003F0A9FB9DF8B9
:10A0380000309DF801100C4A1B0343EA01139DF8F8
:10A04800021043EA111353609DF803309DF8041081
:10A058001B0343EA01139DF8051043EA111313602B
:10A0680003B05DF804FB00BFB81B00201FB5044611
:10A0780002210C2001220DF1070303F081FBC8B374
:10A088009DF80730DB0735D50321062202AB0C20EB
:10A0980003F076FB0C20092101220DF1070303F0E0
:10A0A8006FFB38B39DF8073013F00C0F22D19DF8E1
:10A0B80009209DF8083043EA0223C3EB83339B0051
:10A0C8009DF80B2023809DF80A3043EA0223C3EB56
:10A0D80083339B009DF80D2063809DF80C3043EA84
:10A0E8000223C3EB83339B00A3800C200A210122A7
:10A0F80003F0C2FB04B010BD07B50A2100220C20F2
:10A1080003F0BAFB142003F024FE0A210F220C20CE
:10A1180003F0B2FB0A2003F01CFE01AB102103225E
:10A128000C2003F02DFB0A2003F013FE0A21002265
:10A138000C2003F0A1FB0A2003F00BFE0DF1030332
:10A14800022101220C2003F01BFB0DF1030309215E
:10A1580001220C2003F014FB0A2101220C2003F039
:10A168008BFB03B05DF804FB074B1B681869074BB2
:10A1780020F01F0200F01F01D25801238B401A4221
:10A1880001D0FDF715B87047B00200201404014053
:10A198002DE9F0437C4A136887B0904693B11A685A
:10A1A8001AB17A49486902434A619A88ADF8002091
:10A1B80002228DF803209868002269468DF8022053
:10A1C80003F0C8F9322003F0C4FD002111221E203B
:10A1D80003F052FB012160221E2003F04DFB642096
:10A1E80003F0B7FD02A8FFF7D1FE00240A27264690
:10A1F8002546022101221E2003F03EFB322003F0F7
:10A20800A8FD02A8FFF7C2FEBDF90820BDF90A1093
:10A21800BDF90C308A421444A8BF0A4693421D4433
:10A22800A8BF134613F5805F0E4404DD013FE0D15B
:10A238004FF0010901E04FF000091E200021122211
:10A2480003F01AFB0A27022101221E2003F014FB47
:10A25800322003F07EFD02A8FFF798FEBDF9082022
:10A26800BDF90A10BDF90C308A42A4EB0204A8BF5C
:10A278000A469342A5EB0305A8BF134613F5805F72
:10A28800A6EB010602DD013FDDD101E04FF0000938
:10A2980007EE904A9FED3E7A3E4FF8EEE77A0021AE
:10A2A800C7EE277A70221E20F0EEE77AC7ED007A13
:10A2B80007EE906AF8EEE77AC7EE277A9FED367ACE
:10A2C800F0EEE77AC7ED017A07EE905AF8EEE77AF2
:10A2D800C7EE277AF0EEE77AC7ED027A03F0CCFAF8
:10A2E800012120221E2003F0C7FA1E20022100228D
:10A2F80003F0C2FA642003F02CFDB9F1000F04D179
:10A308004FF07E533B607B60BB60D8F800301E4C3A
:10A318001A7B002A35D01A7D002A32D01B498A6957
:10A3280042F001028A61187B197DFCF7F1FF23686E
:10A338009A689B88128A134223D0184803F0B8FD04
:10A3480023681869FCF734FF23681B690493002607
:10A358000C23012504A88DF815308DF814608DF8AC
:10A36800165006F079FE23688DF806605B7D8DF83F
:10A37800043001A803238DF805308DF8075006F046
:10A388004DFE07B0BDE8F083B00200200010024087
:10A3980000406F465800002001C05E4671A10008C9
:10A3A8002DE9F04F544D1E464FF4147305F108047F
:10A3B800434385B080469146E718A24610B92B441E
:10A3C8004E4A03E0012805D14D4A2B449A631032C6
:10A3D800C3F83C214FF4147303FB08F3EC180AEBA1
:10A3E800030203F59C734748A06034325344616309
:10A3F800E261236200224FF0010B4FF48071D4F820
:10A408003C3161610320A2626262A1612263E2625F
:10A4180084F8442284F840B284F84122A4F84A22FD
:10A42800A4F84C22C4F810906073A67384F84E8286
:10A4380004F59C7258681B8901924FF0020C03A91D
:10A44800ADF80C308DF80EB08DF80FC0CDF800C007
:10A4580003F080F8A36BDDF800C0597B58681B89AE
:10A468008DF80E1003A9ADF80C308DF80FC003F06D
:10A4780071F859463846FFF78DFB322003F069FC26
:10A48800019A214BD2F804B0B3FBF9F1B1F5803F42
:10A4980003D3012BF8D95B08F6E74FF4147404FBD7
:10A4A80008F805EB0809584689B2482208F51278D9
:10A4B80006F050F80AEB0804144BC9F85032002291
:10A4C8005846214606F09CF8D9F8385016F0010F86
:10A4D8000CBF022200222868A97AFFF76BFC0C4BFC
:10A4E800C9F854322846211D002206F089F838465A
:10A4F80005B0BDE8F08F00BFB81B0020D8A5010843
:10A50800F8A50108108F010800A24A047D9E0008E2
:10A51800E39D00080F4B73B518781C4698B10523C6
:10A528000D4D8DF800304FF4805600238DF8013022
:10A5380001A82E856946022206F03AFDAE619DF813
:10A54800050000F0010000F00100207080F001001B
:10A5580002B070BD2506002000040048064B70B507
:10A568001D6806461C46FFF7D5FF18B923685B1B14
:10A57800B342F8D970BD00BF60270020F7B50323A8
:10A588008DF80430030C8DF805308DF80700030AA8
:10A5980006200F4614468DF80630FFF7DFFF78B126
:10A5A800084D4FF4805601A904222E85002006F09C
:10A5B800FFFC38460021224606F0FAFCAE61204630
:10A5C80003B0F0BD00040048024640213C2003F0DF
:10A5D80053B970B500EB8000094CA0F1A1059C3877
:10A5E80025440444074B15F8010F1E787040FFF707
:10A5F800EBFFA542F6D13046BDE87040E4E700BF66
:10A60800288F01082434002010B5441E14F8010FC7
:10A6180010B1FFF7DEFFF9E710BD024680213C20AC
:10A6280003F02AB910B5D420FFF7F7FF8020FFF711
:10A63800F4FFA820FFF7F1FF3F20FFF7EEFFD3203C
:10A64800FFF7EBFF0020FFF7E8FF4020FFF7E5FFEB
:10A658008D20FFF7E2FF1420FFF7DFFFA120FFF7AF
:10A66800DCFFC820FFF7D9FFDA20FFF7D6FF12205A
:10A67800FFF7D3FF8120FFF7D0FFCF20FFF7CDFFF3
:10A68800D920FFF7CAFFF120FFF7C7FFDB20FFF74C
:10A69800C4FF4020FFF7C1FFA420FFF7BEFFA6209C
:10A6A800FFF7BBFFAF20FFF7B8FFA620FFF7B5FF06
:10A6B800AE20FFF7B2FF2020FFF7AFFF0020FFF723
:10A6C800ACFFB020FFF7A9FF4020FFF7A6FF00204E
:10A6D800FFF7A3FF1020FFF7A0FF4FF48064013CB1
:10A6E8000020A4B2FFF770FF002CF8D18120FFF7FB
:10A6F80094FFC820FFF791FFAF20FFF78EFF0120DE
:10A7080010BD08B55038C0B2FFF787FF0020FFF72B
:10A7180084FF1020BDE808407FE7503910B5044693
:10A72800C8B2FFF77AFF04EB4400400004EB44048E
:10A7380000F00E00FFF771FFC4F3C3001030BDE84E
:10A7480010406AE7F0B50124B0FBF4F58D4201D35F
:10A758004C43F9E70026D4B1B0FBF4F504FB15002F
:10A76800B4FBF1F41EB9002D01DC002CF3D1092D46
:10A7780003F1010EEFB204DD002A14BF3725572577
:10A7880000E030253D441D7001367346E3E71C7038
:10A79800F0BDF0B50124B0FBF4F58D4201D34C4374
:10A7A800F9E70026D4B1B0FBF4F504FB1500B4FBBF
:10A7B800F1F41EB9002D01DC002CF3D1092D03F1B1
:10A7C800010EEFB204DD002A14BF3725572500E03B
:10A7D80030253D441D7001367346E3E71C70F0BD1B
:10A7E80003685A1C0260197070472DE9F843089EE7
:10A7F800002B07468846144614BF4FF030094FF027
:10A808002009334613F8012B0AB9254603E0002C2A
:10A81800FBDD013CF6E7002D04DD38464946C0471C
:10A82800013DF8E724EAE4743546A01B284415F8EE
:10A83800011B11B13846C047F7E7BDE8F883024B62
:10A84800186803F056BB00BFD80E002090ED017ABF
:10A8580007EE901AB5EE407AF1EE10FA01BFF8EE65
:10A86800E77A9FED0E7A67EE877AB7EE007A04BF33
:10A87800C7EE277AC0ED017A90ED017AD0ED007A23
:10A8880030EE877A30EE670AC0EE870AE0EE807A0B
:10A89800B0EE670AC0ED007A704700BFDB0FC94011
:10A8A80010B50278202A034600F10100F9D0092AE0
:10A8B800F7D02D2A03D10346BFEE000A04E02B2A65
:10A8C80008BF0346B7EE000ADFED387A1A4613468A
:10A8D80012F8010BA0F13001CCB2092C0AD807EE0E
:10A8E800101AB8EEC77AF2EE046AA7EEA67AF0EE6E
:10A8F800477AECE72E2816D1F2EE046A1146B0EE3C
:10A90800666A0B4611F8012B303AD0B209280AD8EA
:10A9180007EE102AB8EEC77A87EE267A66EE866AC0
:10A9280077EE877AEDE71A7802F0DF02452A35D10B
:10A938005A782D2A02D10233012004E02B2A14BFB1
:10A94800013302330020013B002213F8011F303984
:10A95800CCB2092C03D80A2404FB0212F5E7B2F59D
:10A968009A7F28BF4FF49A721346B7EE007A072BE6
:10A9780005D9DFED0F6A083B27EE267AF7E702F0E4
:10A9880007032BB1F2EE046A27EE267A013BF8E7BB
:10A99800F0EE476A20B1C7EE877A03E0F7EE006A67
:10A9A80067EEA67A20EE270A10BD00BF000000005F
:10A9B80020BCBE4C30B52DED028B87B0B0EE408A7E
:10A9C8000C220021054603A80BF0F3FAB5EEC08A65
:10A9D800DFED2A7AF1EE10FACCBF38EE278A38EE8E
:10A9E800678ADFED277A28EE278A6946FDEEC87A5E
:10A9F80017EE904A84EAE470A0EBE47006F0CAFD12
:10AA0800002CACBF20232D2368468DF80C300BF0AA
:10AA180014FB012807D130238DF80D308DF80E3046
:10AA28008DF80F300CE0022805D130238DF80D3059
:10AA38008DF80E3004E0032804BF30238DF80D3064
:10AA4800694603A80BF0DCFA03A80BF0F6FA033802
:10AA5800C4B2224603A928460BF01CFB00232B5541
:10AA6800284608490BF0CCFA03AB284619190BF015
:10AA7800C7FA284607B0BDEC028B30BD6F12033A07
:10AA880000007A444FAE010870B5064615460846E0
:10AA9800B6FBF2F414B12046FFF7F6FF05FB146489
:10AAA800024B1B5D00F8013B70BD00BF51AE0108B1
:10AAB8002DE9F04F814689B08A4616461C46002586
:10AAC8003178002900F0DD80252902D0013648467A
:10AAD80075E07278302A08BFB278A2F1300319BF46
:10AAE800B71C4FF0000BF71C4FF0010B092B4FF070
:10AAF800000819D8A2F13003D9B2092905D80A22C9
:10AB080002FB083817F8012BF4E7A2F16103052BC3
:10AB180002D8A2F1570305E0A2F14103052B03D89F
:10AB2800A2F137030A2BEADD6C2A31D13A78642A7C
:10AB380007F1010600F083800BD8252A3DD003D801
:10AB4800002A00F09E80BBE7582A0CD0632A19D04F
:10AB5800B6E7732A22D002D86E2A37D0B0E7752A12
:10AB68005CD0782AACD1271D2068A2F15804624233
:10AB78004FF01001624155E02CD9582A32D0632A8F
:10AB88002AD13E4648462178271DD04701350FE097
:10AB9800642A64D00ED9732A14D13E4623680093E0
:10ABA8004846514642460023FFF71FFE271D05442D
:10ABB8003C4685E7252ADFD13E4648462521D04731
:10ABC80001357DE70AD86E2A06D13E46236804344B
:10ABD8001D6075E7002A54D03E4671E7752A26D0D5
:10ABE800782AF9D1A2F1580304F1040C5A422068DA
:10ABF800CDF80CC04FF010015A4105ABFFF7A2FD8C
:10AC0800DDF80CC03E46644605AB00934846514605
:10AC180042465B46FFF7E9FD054451E72068271DDA
:10AC28000A21002205ABFFF7B4FD3C46ECE704F12E
:10AC3800040CCDF80CC020680A210022DDE720684A
:10AC4800002804F1040708DA2D238DF81430404257
:10AC58000DF115030A210022E5E705ABFAE72068A4
:10AC6800002804F1040C0ADA2D238DF81430404230
:10AC78000DF11503CDF80CC00A210022BEE705AB83
:10AC8800F8E7284609B0BDE8F08F0EB40FB505AB5C
:10AC9800019053F8042B0649039301A8FFF708FF16
:10ACA800019B00221A7004B05DF804EB03B07047F2
:10ACB800E9A700080FB413B50B4904AB08680B49A2
:10ACC80053F8042B09680193FFF7F2FE0446084B7A
:10ACD800186803F002F90028F9D0204602B0BDE850
:10ACE800104004B0704700BFFC000020F8000020AE
:10ACF800D80E002080EAE073A3EBE0738B4206DBFA
:10AD0800002801DD401A704702D00844704700202F
:10AD18007047FDEEC07A17EE903A2033402B43D8A7
:10AD2800DFED237AB4EEE70AF1EE10FA04DDDFED89
:10AD3800217A30EE670AF3E7DFED1F7AB4EEE70A0F
:10AD4800F1EE10FA04D5DFED1B7A30EE270AF3E7AF
:10AD5800DFED1A7AB4EEE70AF1EE10FA04DD30EE10
:10AD6800670A37EEC00A0AE09FED157AB4EEC70A03
:10AD7800F1EE10FA44BF30EE270A37EE400A60EED3
:10AD8800007ADFED106A9FED107AA7EEA67ADFED64
:10AD98000F6AE7EE876A9FED0E7AA7EEA67A20EE95
:10ADA800276AA6EE070A70479FED0A0A704700BF98
:10ADB800DB0F4940DB0FC940DB0F49C0DB0FC93F40
:10ADC800DB0FC9BF9A7C2E36FAAF4FB93587083CDE
:10ADD800A4AA2ABE00000000DFED027A30EE270A9E
:10ADE80097E700BFDB0FC93F38B52DED068B90ED17
:10ADF800008AB0EE480A0C460546FFF7EDFFB0EEB4
:10AE080040AAB0EE480AFFF784FFD5ED018AB0EEFC
:10AE1800409AB0EE680AFFF7DFFFB0EE408AB0EE66
:10AE2800680AFFF776FFD5ED02AAF0EE408AB0EE89
:10AE38006A0AFFF7D1FFF0EE409AB0EE6A0AFFF710
:10AE480068FF60EE0A6A69EE297AF0EE665AE7EE64
:10AE5800A85A29EE8A6A29EE007A69EE889A29EEBC
:10AE6800489A28EE400A28EE0A8AC4ED035AF0EE02
:10AE7800465AE7EE685AE6EEA87AA6EE687AC4ED76
:10AE8800009AC4ED028A84ED059A84ED088ABDEC27
:10AE9800068B84ED010AC4ED045A84ED067AC4EDEC
:10AEA800077A38BD10B52DED048B8AB090ED009A65
:10AEB800D0ED028A90ED018A0446084601A9FFF701
:10AEC80093FFDDED047A9DED017A68EE277AE9EECD
:10AED800077A9DED077AE8EE877A9DED027AC4ED50
:10AEE800007ADDED057A68EE277AE9EE077A9DEDBE
:10AEF800087AE8EE877AC4ED017ADDED067A28EE65
:10AF0800278ADDED037AA9EE278ADDED097AA8EE16
:10AF1800A78A84ED028A0AB0BDEC048B10BD074BEA
:10AF28001A8822EA0000904210B518801C4602D008
:10AF3800012002F073FF208810BD00BFE01100203F
:10AF4800064B1A881043904210B518801C4602D050
:10AF5800012002F063FF208810BD00BFE01100202F
:10AF6800024A936823EA0000906070479C270020FB
:10AF7800024A936818439060704700BF9C270020DE
:10AF880008B5104B1A780023D9B2914207D20E495E
:10AF980051F823100968002008600133F4E73220D3
:10AFA80002F0D7FE094B1B685A0309D5084B9B686A
:10AFB8005B0305D440F2DC50BDE8084002F0C9BE8E
:10AFC80008BD00BF00250020042500203C270020E4
:10AFD8009C270020454A68232DE9F341137040F26D
:10AFE800D4735380BE231371EF2382F8D137002323
:10AFF80082F8D23719461646F25C0133514040F2C6
:10B00800D4729342F8D1394B83F8D217384B1A6966
:10B01800120604D5374A5A6002F188325A6004276A
:10B028000020013F17F0FF0750D0314B3422DA607F
:10B03800002444B1002356F804800193FCF750F82B
:10B048000428EED117E0FCF74BF80428E9D1284D85
:10B058002B6943F002032B61274B6B612B6943F08B
:10B0680040032B61FCF73CF82B69042823F002030A
:10B078002B61DFD0D5E71E4D2B6943F001032B610F
:10B0880004F1006303F57E331FFA88F21A80FCF797
:10B0980027F8042810D1194B23440193019B4FEA48
:10B0A8001848A3F80080FCF71BF82B69042823F044
:10B0B80001032B6105D0B4E72B6923F001032B6151
:10B0C800AFE7043440F2D4739C42B2D1084A136902
:10B0D800042843F08003136102D106F085FA10B901
:10B0E8000A2002F0B3FE02B0BDE8F0819C270020E0
:10B0F800002002402301674500F8030802F803080E
:10B1080010B50E4C2068FBF723F92068047A00225A
:10B1180002FB02F3193B634303F6C413534319219B
:10B1280093FBF1F3064921F812300132072AEFD1D7
:10B138000449BDE81040FBF7C1B800BF5410002017
:10B14800A80E0020E02800202DE9F04106F04CFA76
:10B1580010B90A2002F07AFEA44CA549A54D40F288
:10B16800D47220460AF01AFF94F8A837022B84BF3D
:10B17800002384F8A83794F8A8274FF4CC7101FB72
:10B1880002F303F5387023442044286093F834030D
:10B1980003F54C73022801FB024284BF002018719A
:10B1A80092F83433944A13700C2202FB0343934AF7
:10B1B80003F2AA731360A26846F2090313401BB98D
:10B1C8004FF40050FFF7D4FEA368D80703D54FF417
:10B1D8000050FFF7C5FEA368590409D50820FFF7FA
:10B1E800BFFE4FF40050FFF7BBFE0120FFF7B8FE8B
:10B1F800A3681A0706D54FF40050FFF7B1FE0120E7
:10B20800FFF7AEFEA3689B0402D54020FFF7A8FE17
:10B2180094F8D221754B2AB193F8D62112B10022A5
:10B2280083F8D621764B774E1E604FF0000C6746A8
:10B2380004EB0C03B3F8EAE14FEA5E0101F0773161
:10B248004FEA9E0303F03333C1EB0E00C11A4FEAF5
:10B25800DE0303F01133CB1A03EB23131EF00108AE
:10B2680003F00F324FF0FF0392FBF3F3C3EB03231A
:10B2780018BF0137A2EB030318BFFFB2012B0ADD89
:10B28800022B40F0B080B8F1000F00F0AC801EF047
:10B29800BC0F00F0A8800CF1080CBCF1280FC7D136
:10B2A800013F012F00F29F80FFF72AFF3022002183
:10B2B8005548564F0AF07DFE554BD5F800801F6063
:10B2C800544B002108F17900C3F80080FBF780F89F
:10B2D800514B80F001001870504B07F126021A609C
:10B2E8004F4B07F1CC021A6098F8000003F0D2F92E
:10B2F80028684C4B00F5C5721A60FDF72BF84A4BCD
:10B30800DFED4A6A07F18A021A60494B00221A8067
:10B318009A71484B07F12A021A602B68464A93ED46
:10B32800187A03F219111160444A03F28911116065
:10B33800434A07F108011160424A1760424A07F17F
:10B3480092011160414A07F19C0111604049536123
:10B3580067EE266A0E60B6EE007AB4F8661187EEDC
:10B36800267A101D07EE901AB4F86811F8EE677A7D
:10B37800C2ED027A07EE901A93F85C10117193F8F7
:10B388007810517194F8D5111174F8EE677AB3F802
:10B398001611C2ED037A07EE901A2E492E4A08605C
:10B3A80003F1640111602D4A2D4982ED007AF8EE0F
:10B3B800E77A9FED2C7A2C4A0B60C7EE277A2B4947
:10B3C8009FED2B7A67EE877AC2ED007A03F1680267
:10B3D8000A60284903F211130B60274B1F60274BA3
:10B3E8001A60BDE8F081FBF74FFE5DE79C2700205F
:10B3F80000F803082C100020E0240020541000203E
:10B40800B8320020242900201C0F0020E02800204A
:10B41800500F0020540F00200C000020B807002017
:10B42800FC050020600F0020080F0020DB0F4940BA
:10B43800F03300200C080020DC200020DC0900206C
:10B44800882300208C230020F008002060200020A2
:10B45800B409002010240020502400204C2400208F
:10B468008407002000006144EC08002078070020D1
:10B478004C3D0F44DC080020E40800208006002032
:10B4880008B5FFF7A7FDFFF75FFE0120BDE80840FC
:10B4980002F0C4BC642928BF6421F8B510FB01F58B
:10B4A8006424064695FBF4F40027E4B2FBB2A342F9
:10B4B80004D29F20FFF78DF80137F7E7B4420BD28B
:10B4C800C4EB84101421C4EB800095FBF1F5663DB4
:10B4D8002844C0B2FFF77DF80134E4B2B44201D287
:10B4E8009A20F7E7F8BD08B507480AF0A6FDC0B2EC
:10B4F80009280246044B04DC01302021C0B29954CB
:10B50800F6E700221A5408BD8D15002008B5074833
:10B518000AF093FDC0B21428044B04D8421C202121
:10B528001954D0B2F7E700221A5408BD8D1500202F
:10B538002DE9F74FA74C02F0E5FB26686568A76878
:10B54800861BF643451BC71BED43FF43F60F80469A
:10B55800ED0FFF0F2EB93FB9002D00F08682B946D6
:10B568002CE04FF0000929E0B14627E003EB8A0BF5
:10B57800BBF802301A050ED413F4805F1DBF964A3B
:10B588009BF801101268954A954B14BF52F8212078
:10B59800126843F82A20BBF80230D80516D499055A
:10B5A8000AD5904B1B7813F0040F0CBF8E4A8F4AB4
:10B5B8008B4B126843F82A2009F10109207B8C493A
:10B5C8005FFA89FA82450B68D0D326E0894A50464B
:10B5D800594605F081F8884B1B885A0603D5504612
:10B5E8005946864A16E0580703D550465946844AB4
:10B5F80010E0190703D550465946824A0AE09A07CF
:10B6080003D550465946804A04E0DB07D4D57F4A23
:10B618005046594605F060F8CEE7DFF808E2009397
:10B62800BEF906307822A3F57A7353434FF47A7241
:10B6380093FBF2F303F22B1301930022F3465FFA14
:10B6480082FE864517D2009B03EB820EBEF802E00D
:10B658001EF4806F0DD0DFF88891019B39F822E045
:10B6680040F2671A9E449EFBFAFC0AFB1CEE29F87E
:10B6780022E00132E3E74DB308F5C333A03363603A
:10B68800637B544A13BB9373614B1B6813F0020F1F
:10B698000AD0DFF894E19EF800E0BEF1000F03D075
:10B6A8004FF0010E82F80EE0DA0506D5594B5B79AA
:10B6B8001BB1A37B43F00203A3734A4B1B7813F01F
:10B6C800050F02BFA37B43F00403A37394F80EE0B5
:10B6D800BEF1000F03D13F4B5B7B002B4FD094F89A
:10B6E8000DC01CF0010FACF10C031DD1BCF1030F10
:10B6F80007D8DFF8E8903C4A1EF0040F08BF4A4616
:10B7080000E0364AACF1040CBCF1070F05D8DFF8AD
:10B718001CC11EF0010F18BF6246DBB2032B0ED806
:10B728001EF0020F3C4B06E0DBB2032B06D82F4B72
:10B738002A4A1EF0020F18BF1A4600E0274A4FF0A7
:10B74800000C5FFA8CF383420DD20B6803EB8C0379
:10B758005B881B0642BF224BD2F8009043F82C901E
:10B768000CF1010CEDE785B1BEF1000F08D0637B49
:10B77800184A0133DBB2142B06D1002304E025B1AB
:10B78800637B002BF3D100E05373002E52D0234A81
:10B79800B2F90250B2F90020002DB8BF6D42002A5C
:10B7A8004FF03203B8BF524295FBF3F592FBF3F228
:10B7B800EDB2D3B2AB4238BF2B46194A13B192FB54
:10B7C800F3F300E0134643442360E37B014A7BBB69
:10B7D80001232EE078200020D8200020A8A6010808
:10B7E800220E00202234002084A5010874A5010837
:10B7F800B4100020CC910108E0110020D29101087A
:10B80800D8910108DE910108E4910108EA91010844
:10B818003C270020F03300208CA5010800110020EF
:10B82800400D0300782700206C11002094A5010822
:10B838000023D3738E4D8F4B2D78E27BADB9002F4B
:10B8480000F00E818C4B267B1A788C4B8C4D93F82C
:10B8580000C08C4BD3F800E00B6802F00402002112
:10B86800D2B203EB86060F46B5E01AB9864A1A61CA
:10B87800002508E0854AFAE70A68AB00D6187688FA
:10B88800760604D40135EBB28342F5D3D7E7804E70
:10B89800B6F90060192E25DD12F803E094F814C0FB
:10B8A80026690EF00F09E1450CDCDFF8C8C19CF8E9
:10B8B80015C0BCEB1E1FDEBFDFF8D8E1D6F800C00C
:10B8C80043F80EC012F803E094F816C00EF00F0902
:10B8D800E14533DBDFF89CC19CF815C0BCEB1E1FAB
:10B8E8002CDC26E0193629DA12F803E094F814C0A3
:10B8F80026690EF00F09E1450CDCDFF878C19CF8E9
:10B9080017C0BCEB1E1FA2BFDFF888E1D6F800C045
:10B9180043F80EC012F803E094F816C00EF00F09B1
:10B92800E1450BDBDFF84CC19CF817C0BCEB1E1FD0
:10B9380004DBD6F800E0574E43F806E0544EB6F95B
:10B948000260192E1BDD12F803C094F814E0266972
:10B958000CF00F09F1450CDCDFF8189199F81590F7
:10B96800B9EB1C1FDEBFDFF82CC1D6F8009043F8F6
:10B978000C90D25C02F00F0CF4451EDD82E71936FC
:10B9880080DA12F803C094F816E026690CF00F0963
:10B99800F1450CDBDFF8DC9099F81590B9EB1C1F2A
:10B9A800DEBFDFF8F0C0D6F8009043F80C90D25C08
:10B9B80002F00F0CF445FFF665AF94F817E0BEEB04
:10B9C800121FA2BF334A36689E505BE758880005AD
:10B9D80004D404330435B342F8D122E04AB101EB70
:10B9E8000C0A06209AFBF0F900FB19A001280DDCCF
:10B9F80001E057B9012793F801900EEB89003EF852
:10BA080029A090F80290C07803E0174600208146EC
:10BA18008246013125F802AC85F800906870C9B2F9
:10BA2800D7E7164A1378013B13F0FF0308BF062334
:10BA38001370114B1B785B0741BFBBF90630A3F5A8
:10BA48007A7303EBC3034FF47A7243BF93FBF2F3A9
:10BA58000133DBB20123104A92FBF3F34344A360A2
:10BA680003B0BDE8F04F01F097BC03B0BDE8F08F1C
:10BA78004E3300207820002022340020640000206B
:10BA8800240E0020D820002090A50108A8A60108AF
:10BA980000110020220E0020400D0300344B354ACF
:10BAA8001B68126810B51A60334A116859605168EA
:10BAB8009268DA60314A9960116819615168926830
:10BAC8009A612F4A59611168D961516892685A621E
:10BAD8002C4A196211881985518859859188D2880C
:10BAE800DA85294A99851188198651885986928854
:10BAF8009A86264A1188D9865188198719469288C4
:10BB080021F83A2F224A10780022824206DA214C84
:10BB180034F8124021F8024F0132F6E71E4A128823
:10BB2800A3F864201D4A1288A3F866201C4A1188CD
:10BB3800A3F86C1051889288A3F87020194AA3F8CA
:10BB48006E1012689A66184A3B21126892FBF1F24D
:10BB5800B2F5967FC8BF4FF0FF325A67134A128872
:10BB6800A3F87820124A5289A3F85E2010BD00BFBE
:10BB78001C30002000340020302200203C2200200D
:10BB8800482200200011002014100020EA10002094
:10BB9800002500203010002076130020CC0E002055
:10BBA80044130020F410002004000020501000204E
:10BBB8001A10002070B5472006F0CCF8174B1B6808
:10BBC8001B0307D5164B174A5B6810681B68C01A19
:10BBD80006F0F2F8144E154C154D307806F0ECF8D6
:10BBE80023682868C01A06F0F6F863686868C01AFF
:10BBF80006F0F1F80F4B188806F0DEF80E4B18889F
:10BC080006F0DAF80D4B188806F0D6F83378237466
:10BC18002B68A3606B68E36070BD00BFA031002093
:10BC28001C3000200034002026110020083000209D
:10BC38002811002024110020221100205810002073
:10BC48000A4A138801331380094A136801331360C1
:10BC5800084A138801339BB2202B01BF00231380AD
:10BC6800054A138808BF013313807047C03100208C
:10BC7800A8310020AC310020AE31002038B53A4B55
:10BC88001B78083B012B05460C466BD8452006F06F
:10BC980061F8284606F05EF80C2D23D004D80A2D4A
:10BCA8000AD014D835B138BD0E2D4BD02ED3FF2D68
:10BCB80050D038BD206849E0207806F04BF862790A
:10BCC8006378002A14BF80200020184300E0207801
:10BCD80006F040F8A07806F03DF8E07806F03AF86B
:10BCE80020793BE0B4F9000006F05CF8A07806F093
:10BCF80031F8E07806F02EF8B4F9040006F052F8AE
:10BD0800B4F90600BDE8384006F04CB863782078EE
:10BD18008BB180F0800006F01DF8A468E0B206F050
:10BD280019F8C4F3072006F015F8C4F3074006F025
:10BD380011F8200E12E006F00DF86068BDE83840F2
:10BD480006F049B8206806F037F86068BDE8384062
:10BD580006F032B8054805F081FF0020BDE83840FC
:10BD680005F0F8BF38BD00BFF82F002076AE0108F7
:10BD78002DE9F04FBF4B8BB018880193002840F095
:10BD8800A380BD4EFCF7AAFDFFF788FE3468492062
:10BD980005F0E0FFB94B2546186806F00DF855F890
:10BDA800040B06F009F82846FBF720F904F1100007
:10BDB800FBF71CF904F11C081027B14D01232A6870
:10BDC800BB40134203D0D8F8000006F004F801374E
:10BDD800132F08F10408F0D1AA4F04F12800FBF74B
:10BDE800F5F8B7F84431B4F92E00C01A05F0E4FFAD
:10BDF8002B6813F4805FB84608D0A34BB4F86400EE
:10BE08001B88181AC0F30D0005F0D6FF2B6899049B
:10BE180003D5B4F8660005F0CFFF2B685A0503D5A3
:10BE280004F16C00FBF7D2F82B681B0502D5A06E55
:10BE380005F0D1FF2B685F0402D5606F05F0CBFFDA
:10BE48002B68180403D5B4F8780005F0B5FF04F1A1
:10BE580030002746FBF7BAF804F13600FBF7B6F8CE
:10BE6800B8F8443137F93C0FC01A05F0A5FF4FF078
:10BE78000108864B1B78984509DA37F9020FB4F99F
:10BE88003C30C01A05F0A7FF08F10108F1E72B685C
:10BE9800990505D5B4F95E00A0F2DC5005F09BFFCA
:10BEA80032687B487260B260121A9110794A4A432C
:10BEB800531C032293FBF2F202EB42029A1A7C23F0
:10BEC80003FB0203336068E2734B744A1B68116812
:10BED8008B4206D00AA9002041F8203D1360FFF7E5
:10BEE800CDFE684A019B92F8CE171B8892F8CF07BF
:10BEF8000B44013BB3FBF0F200FB12338B4280F0A2
:10BF080017825D4F0120FCF7E9FCFFF7C7FD5020C1
:10BF18003E687D6805F01EFFBA683B6810681B68BC
:10BF28007A6803441068A3EB400005F054FF6A6880
:10BF380073689B1A0293AA68B3689B1A0393EA680A
:10BF4800F36802A89B1A0493FBF750F82A6933692F
:10BF58009B1A02936A6973699B1A0393B369AA6966
:10BF68009B1A04930023194602AA52F8212002F1D1
:10BF780020003F2842D802F108000F2806D80232D4
:10BF8800032A04D9002B08BF012300E00223013152
:10BF98000329E9D1012B02980ED0022B21D0039B53
:10BFA80003F003039B0000F0030043EA0010049B26
:10BFB80003F0030318430CE000F00F0040F04000CA
:10BFC80005F0C8FE0498039B00F00F0040EA031038
:10BFD800C0B205F0BFFE06F11C0B05F11C081024C9
:10BFE8006FE000F03F0040F0800005F0B3FE9DF8E0
:10BFF8000C0005F0AFFE9DF81000EAE702224FF0B2
:10C00800000802AB4FEA880853F8223003F1800198
:10C01800FF2910D903F50041B1F5803F02D248F05D
:10C02800010808E003F50003B3F1807F34BF48F04E
:10C03800020848F0030812F1FF32E2D268F03F002C
:10C04800C0B205F087FE02AC0DF1140A08F0030334
:10C05800022B207807D0032B22D0012B29D105F001
:10C0680079FE607825E005F075FE607805F072FECF
:10C07800A0781EE0AC3100201C300020A831002040
:10C08800A03100209C2700209C31002000250020A2
:10C0980028300020DF7BEFBDB4310020B031002014
:10C0A80005F058FE607805F055FEA07805F052FEC0
:10C0B800E078043405F04EFE54454FEAA808C5D18F
:10C0C80089E7B84901220B68A2401A428A4606D07D
:10C0D800DBF80000D8F80030C01A05F07CFE013407
:10C0E800132C0BF1040B08F10408EAD106F1260021
:10C0F80005F12601002331F9024F30F9022F121BF6
:10C1080002AC44F823200133042BF4D103214FF06F
:10C1180000094FEA89035FFA83F902AB53F821203B
:10C128006AB102F108000F2802D849F0010906E0B7
:10C138008032FF2A94BF49F0020949F0030911F13E
:10C14800FF31E6D2484605F005FE00240DF1080B44
:10C15800A04609F00302022A16D0032A1DD0012A9C
:10C1680038D1B8F1000F05D1DBF800402401E4B262
:10C1780090462FE0DBF8000000F00F00204305F0A8
:10C18800E9FD4FF0000825E0B8F1000F0CD0DBF80E
:10C198000000C0F30310204316E0B8F1000F08D1E7
:10C1A8009BF8010005F0D6FD9BF8000005F0D2FDD4
:10C1B80010E0DBF80000C0F30330204305F0CAFDAF
:10C1C800DBF80000C0F3071005F0C4FDDBF8004001
:10C1D8002401E4B20BF1040B06AB9B454FEA990925
:10C1E800B7D1B8F1010F02D1204605F0B3FDDAF856
:10C1F800003013F480541FBFB6F86420B5F86410FB
:10C20800521A029218BF01249A040AD50AAA02EB0C
:10C218008401B5F86600B6F86620121A41F8202C99
:10C228000134580513D502AA02EB840C06F16A0EF4
:10C2380005F16A0000223EF9021F30F9028FC8EBAF
:10C2480001014CF822100132032AF4D103341905F4
:10C2580008D50AAA02EB8400A96EB26E521A40F8F9
:10C26800202C01345A0408D50AAA02EB8400696F0D
:10C27800726F521A40F8202C013418040BD50AABFF
:10C2880003EB8402B5F87810B6F878305B1A42F8F8
:10C29800203C013400E0FCB1012C03D1029805F0E8
:10C2A8009AFD19E0631E002002AA400052F82320DC
:10C2B800C0B20AB140F00100013BF5D505F04AFDD6
:10C2C8004FF0000802AB53F8280008B105F083FDD1
:10C2D80008F10108A045F5DB30200321FCF73EFBFF
:10C2E80036200321FCF73AFB2F4B3C201978FCF74A
:10C2F80035FBDAF80030990506D5B6F95E00B5F9D0
:10C308005E30C01A05F067FD3A6828487B687A6095
:10C31800121A9110264ABB604A43531C032293FB0E
:10C32800F2F202EB42029A1A7C2303FB02033B60FF
:10C33800204B1B681A0630D51F4C204D22682B68ED
:10C348009A420BD162686B689A4207D1019B1B889D
:10C35800102B11D11A4B1B885B060DD1482005F014
:10C36800F9FC206805F037FD606805F034FD2368A6
:10C378002B6063686B600EE0124A104B11782A7CC0
:10C38800914208D1104A99681068884203D15268CE
:10C39800DB689A4201D0FFF70DFC05F04DFC0BB0AD
:10C3A800BDE8F08FA03100200025002028300020B3
:10C3B800DF7BEFBD3C2700205C1000200830002008
:10C3C800AE31002026110020281100202DE9F84F59
:10C3D8000C9E3A4CC2EB030B0B9BF61A63680029C0
:10C3E80014BF4FF0060A4FF0040A01330546904681
:10C3F80013D1236853455ED2314A324852F823207C
:10C40800032B98BF294605F093FC636801336360EA
:10C418002D4B002205461A7013E0002511E02B4A27
:10C428001278954240DA0B9BE3B109FB06F2995C5E
:10C4380001228A40264909680A4213D163680133F8
:10C448006360D4F804900A9B1C4F9945E7DB2BD115
:10C458000A2005F07FFC3B6801333B604FF0FF3357
:10C468007B6021E0184A117821B12C2005F072FC7C
:10C47800013501E001211170226809FB0BF308EB7B
:10C48800030752B958F8030005F0E8FB97F90410C0
:10C498004B1C0544D2D00F4802E03A440E481179AB
:10C4A80005F046FC0544C9E7206850452CBF00202C
:10C4B8000120BDE8F88F0020BDE8F88FB8310020D2
:10C4C800F091010881AE010890200020880000202A
:10C4D800A031002090AE0108FCAD010838B5002459
:10C4E8000B4D6059254403F0B1FA696811B1094848
:10C4F800FEF7E0FBA96811B10748FEF7DBFB074828
:10C50800103403F0A3FAB4F5F07FE9D138BD00BFC9
:10C5180008920108B4AE0108BAAE010801B90108D1
:10C5280070B50546284609F088FD064658B91A4BE5
:10C538001A485A791A4B03EB8203BDE87040D3F8C6
:10C54800DC11FEF7B7BB28461649324609F07EFDD6
:10C5580060B91548154C03F079FA54F8041F19B15D
:10C568001348FEF7A7FBF8E7124805E00024124B32
:10C5780053F8241021B91148BDE8704003F066BA99
:10C588002846324609F062FD01340028EFD1024BFB
:10C598000B4D5C71C6E700BF9C270020C0AE0108A8
:10C5A80008920108CCAE0108D1AE0108E493010855
:10C5B800E4AE010801B90108E893010866AC010876
:10C5C800DCA90108F0B585B0044609F036FD082855
:10C5D80026D1621EE01D1F4912F8013F096819445F
:10C5E800497801F00301022908BF203B82421370F9
:10C5F800F1D1254604F1080715F8016B16483146B4
:10C6080009F00DFD20B12846314609F008FD10B1AA
:10C61800F9F756F91CE0BD42EED12046FAF772FD53
:10C628000E4803F013FA00230D4A1A4404A992F89D
:10C6380088210A440849595C02F80C1C0133082B6C
:10C64800F2D1002307488DF80C3001A9FEF732FB20
:10C6580005B0F0BD8C0000202DC30108E8AE01082C
:10C668009C270020A5B70108264B274C1D68206889
:10C6780080B5F9F7D5FC2846F9F7D2FC206841794E
:10C688008A0703D441F0020101F024FC1F4B082261
:10C698009A611F4B1A6812F4003F1F461FBF0623FA
:10C6A8006371E37923F001031CBF43F00203E371D4
:10C6B800206801F01BFC90B1144E08233385124BFF
:10C6C800186801F010FC8046FBF7BEFA08B104F0C8
:10C6D800CDF82846414601F00CFC0823B3612846F2
:10C6E80001F004FC38B12846266801F0FCFB01463D
:10C6F800304601F0FEFB3B689B03D9D5FCF7F0FA06
:10C70800D6E700BFFC240020942000200004004845
:10C718003C2700202DE9F041054609F08EFC2C4B02
:10C7280004469E6888B92B4803F090F92A4B53F8C1
:10C73800241041B10123A340334202D02748FEF719
:10C74800B9FA0134F2E7264821E02846254922466D
:10C7580009F07CFC58B92448244C03F077F954F8C4
:10C76800041F0029EFD01D48FEF7A4FAF7E72B783D
:10C778002D2B03BF013504F1FF344FF001084FF0B2
:10C7880000080026144B53F8267027B91848BDE84E
:10C79800F04103F05BB928463946224609F056FCB9
:10C7A80098B90120B040B8F1000F03D0FEF7D8FBCC
:10C7B800104802E0FEF7DCFB0F4803F047F9394662
:10C7C8000E48BDE8F041FEF775BA0136DAE700BF5A
:10C7D8009C270020EEAE010850940108E4AE010841
:10C7E80001B90108CCAE0108F8AE01084C94010863
:10C7F80066AC010804AF01080DAF0108A4B7010831
:10C8080010B5084803F022F9074B00241C741C6477
:10C81800064B1C7001F0F4FC03F062FB044B1C6037
:10C8280010BD00BF15AF010894200020253400205A
:10C83800FC24002070B5064600240A4BE518AA8897
:10C8480016420AD0E1580848FEF734FA2846002173
:10C8580003F089F8054803F0F9F81434B4F5486F83
:10C86800EBD170BDDC97010841AF010801B901089F
:10C8780008B50848FEF71EFAFBF788FFFDF74AFEE1
:10C8880018B9642001F065FAF8E70348BDE80840E4
:10C89800FEF710BA4BAF010858AF01082DE9FF4168
:10C8A8000A48068885684488B0F80480C768FBF79A
:10C8B80077FECDF800800290019731462A4623463C
:10C8C8000348FEF7F7F904B0BDE8F0811000002036
:10C8D80060AF0108F0B504788BB005460CB10024B0
:10C8E80036E04A4B19680E2303FB041101F58C70DE
:10C8F800B1F91D51B1F91921B1F91B31009591F820
:10C908002051019591F82151029590F90700039063
:10C9180001F590713E4891F90210049121460134C5
:10C92800FEF7C8F9082CDCD16DE02D2B14D1072CAB
:10C938001BDC284609F0D8FB0AAB661C03EB440451
:10C9480024F8100C15F8013F303B092BFAD934466E
:10C958002B78002BE9D104E0A3F13002092A09D889
:10C96800E5E7082CBDF8182009D00BB0BDE8F04069
:10C97800F8F7A6BF202BF8D101352646E7E7072AA6
:10C98800F3D8BDF81A00214BA0F2EE2189B240F28B
:10C99800DC55A9421B68E8D8BDF81C10A1F2EE24AA
:10C9A800A4B2AC42E1D8BDF81E7004B23EB2A642B1
:10C9B800DBDB0DB2AE42D8DCA542D6DBBDF92440A4
:10C9C800642CD2D1BDF8266034B2112CCDDCBDF870
:10C9D8002050B42DC9D8BDF82240B42CC5D812B205
:10C9E8004FF00E0E0EFB0233A3F81B116421A3F8BF
:10C9F8001901A3F81D7183F8205183F8214183F8A8
:10CA08001F1183F822610BB0F0BD00BF2C1000206D
:10CA1800BDAF0108F0B504468FB0204609F00DFB04
:10CA2800C5B225BBAC48AD4C03F010F894F8D6104D
:10CA380009B9AB4854E049B294F8D42094F8D530F9
:10CA4800009194F8D710019194F9D810029194F9B3
:10CA5800D910039194F8DA100491A24829460135B7
:10CA6800FEF728F9102D04F10704DFD1E1E720468D
:10CA78009D49052209F0EAFA0546B8B929469B48B6
:10CA8800702209F096FA9A4B196828460E2303FB80
:10CA9800001301300022082883F8232183F8242179
:10CAA80083F8252183F82621F0D113E12046914906
:10CAB800042209F0CBFA05462046002D4AD1202150
:10CAC80009F0ADFA002800F00581461C304609F04F
:10CAD800B4FA2C460746884B53F824502DB987489A
:10CAE8000FB0BDE8F040FEF7E5B830462946FAB287
:10CAF80009F0ACFA01340028EDD1784A02F170014E
:10CB08001646002382F8DA3082F8D63082F8D5301B
:10CB180082F8D43007328A42F3D1794901EBC40153
:10CB280091F8A022934210DAD1F8A472C3EBC302A1
:10CB3800B0183A4400F1D4011768C0F8D47090884E
:10CB4800888092798A710133E7E729466D48FEF7B4
:10CB5800B1F890E06C49072209F078FA05462046BA
:10CB6800002D4AD1202109F05AFA064609F065FA43
:10CB7800C4B274BB6548FEF79DF821466448013489
:10CB8800FEF798F80E2CF8D15548FEF793F80024D4
:10CB980060482146FEF78EF80025554A5E48116820
:10CBA8000E2202FB04120123D2F823215B49AB4079
:10CBB80013425B4B05F1010508BF1946FEF77AF8E9
:10CBC8000E2DEAD146480134FEF774F8082CDFD15F
:10CBD80080E03046534909F08BFA2C4600284CD0A7
:10CBE800022C4FD009F080FA06AB4E4943F82400D6
:10CBF800002009F07DFA0134F0E74A4909F078FA93
:10CC0800002460B1082C38D009F06EFA06AB45490B
:10CC180043F82400002009F06BFA0134F1E7082CEE
:10CC28002BD1069B0F2B28D8DDF81CE0BEF1070F8F
:10CC380023D8089F0D2F20D8099E06F16402C82A20
:10CC48001BD80A9DFF2D18D80B98642815D80C9965
:10CC5800642912D8884210DA0D9C032C0DD8324A68
:10CC6800C3EBC303134483F804E05F719E71DD7165
:10CC7800187259729C722D4CCFE60FB0BDE8F04087
:10CC8800F8F71EBE069B072B20D807990D291DD83B
:10CC98000278722A0DD06E2A18D1154A12680E2011
:10CCA80000FB032301228A40D3F8231121EA020260
:10CCB80009E00F4A12680E2000FB032301228A4074
:10CCC800D3F823110A43C3F8232101E0F8F7F8FD4C
:10CCD8000D4CA2E60FB0F0BDE5AF01089C2700207F
:10CCE80001B9010810B0010836AC0108702800200D
:10CCF8002C10002061AC0108E893010866AC01081B
:10CD08000892010875AC0108DDAF0108BEAE010844
:10CD18002CB00108FCAD010831B001087CBB01084A
:10CD280036BC010835B001086C280020DCA90108D0
:10CD38002DE9F743047805468CB9324D95F8A312CE
:10CD4800B5F8A02295F8A2322F4800912146013467
:10CD5800FDF7B0FF102C05F10405EFD14FE009F005
:10CD6800C3F90F28044636DC2846202109F057F974
:10CD7800264EE4B2D6F84480451CA4000027284675
:10CD880009F0B2F95FFA87F9B9F1010F83B208D057
:10CD9800B9F1020F0BD0B3F5B47F25D2726C1353DF
:10CDA8000AE0FF2B20D8736C2344987004E0FF2B13
:10CDB8001AD8736C2344D87028462C2109F02FF90F
:10CDC800054608B1013502E0B9F1020F0CD101376F
:10CDD800032FD4D113E00E480E4900220F2303B0CD
:10CDE800BDE8F043FDF766BF08EB0400002104220C
:10CDF80009F0DFF803B0BDE8F043F8F761BD03B010
:10CE0800BDE8F0839C27002037B00108942000205B
:10CE1800D5AB0108F4AB01082DE9F0412DED048BE9
:10CE2800B3498AB0044609F0CDF8B2490028204633
:10CE38000CBF0126072609F0C5F8AF49002820468F
:10CE480008BF022609F0BEF8002808BF0426F1072B
:10CE580040F10681A948AA4C02F0F8FD002002F032
:10CE6800FDFBA84802F0F2FDA74802F0EFFD627949
:10CE7800A64BA74803EB82032546D3F8DC11FDF740
:10CE880019FFA448FDF716FF4FF00008274695ED57
:10CE9800058AB5EE408AF1EE10FA04D19E48FDF7F6
:10CEA80009FF002570E09D48D5ED069A95ED079A93
:10CEB800D5ED088A4146FDF7FDFEB5EEC08AF1EED4
:10CEC80010FA02D5202002F0B9FDB0EE480A06A8F3
:10CED800FDF770FD01469248FDF7ECFEF5EEC09AAD
:10CEE800F1EE10FA02D5202002F0A8FDB0EE690A92
:10CEF80006A8FDF75FFD01468948FDF7DBFEB5EEA4
:10CF0800C09AF1EE10FA02D5202002F097FDB0EE9B
:10CF1800490A06A8FDF74EFD01468148FDF7CAFEFD
:10CF2800F5EEC08AF1EE10FA02D5202002F086FD57
:10CF3800B0EE680A06A8FDF73DFD08F101080146B4
:10CF48007848FDF7B7FEB8F10C0F05F110059ED132
:10CF5800A4E749B294F8D42094F8D530009194F815
:10CF6800D710019194F9D810029194F9D91003912E
:10CF780094F8DA1004916C4829460135FDF79AFEB9
:10CF8800102D04F1070403D094F8D6100029E0D13D
:10CF980000254FF00E0808FB05F80024634A926C40
:10CFA80042440123D2F80A20A340134240F094805F
:10CFB80001340E2CF2D10135082DEAD15C485D4CC4
:10CFC80002F044FDD7F8088054F8041F19B15A48F4
:10CFD800FDF770FEF8E70D46584B53F8254054B15D
:10CFE8000123AB4013EA080F03D055482146FDF74B
:10CFF80061FE0135F0E7534802F028FD21467B1811
:10D008000AAA93F8883113444F4A8A5C03F8102C13
:10D0180001310829F3D1002306A94C488DF82030A6
:10D02800FDF748FE4A4802F011FD4A48F9F77AF838
:10D03800494802F00BFD4748F8F748FC474802F01A
:10D0480005FD4448FFF774FE4548FDF733FE4020D0
:10D05800FFF7F0FB434802F0F9FC3E48F8F778FF89
:10D06800B20726D5404802F0F1FC404802F0EEFC39
:10D07800384802F033FB3E4802F0E8FC3548F8F740
:10D08800A6FB3C4802F0E2FC3248F8F7AFFE3A480B
:10D09800FDF710FE2F48F8F727FD384802F0D6FCB8
:10D0A8002C48FFF717FC2E48FDF704FE8020FFF7F9
:10D0B800C1FB730716D5324802F0C8FC314802F0AC
:10D0C800C5FC244802F0E4FA2548FDF7F3FD4FF4C7
:10D0D8008070FFF7AFFB05E0294622462A48FDF796
:10D0E800E9FD65E70AB0BDEC048BBDE8F08100BF3F
:10D0F8004BB00108BFB4010852B0010858B001088C
:10D108009C27002066B0010878B001080892010841
:10D1180084B001088FB001089CB00108A9B00108CB
:10D12800BDAE0108A5B70108B1B0010894200020E0
:10D13800D0B001084C940108E0B0010850940108EF
:10D14800EEB00108FBB001082DC3010807B10108C2
:10D1580010B10108DCA901081FB101082BB10108B1
:10D1680001B9010839B1010846B1010859B10108EE
:10D1780067B1010871B1010880B101088EB10108D9
:10D188009AB10108ABB10108BDB1010810F80A3C19
:10D198000133DBB20A2B84BF10F8131C044A00F8D1
:10D1A8000A3C82BF002322F8113000F80A3C70477D
:10D1B800A0320020334A136C90681944081A40F6CC
:10D1C8008C23984270B513469160D06051603BD96A
:10D1D800127893F945108A4210460BD1111F08297D
:10D1E80008D893F84610182901D8013103E083F8CC
:10D1F800442002E0002183F8461093F94440214975
:10D20800A24219D191F84740B4B10C31002494429C
:10D2180006DA1D4D51F8046F25F814600134F6E75D
:10D228000C2805D01849002421F810400130F7E7F0
:10D23800164801780131017083F845200022012148
:10D248001A7083F8471070BD92F84710C9B1A0F260
:10D25800EF2440F2DA518C4208D811780B2905D80E
:10D268000B1D0131117042F8230070BD002283F8B4
:10D278004720074B03F13002002143F8041F934273
:10D28800FAD170BD28010020A032002041060020FC
:10D2980034010020024A136C0133194411647047A9
:10D2A80028010020024B53F820301B681960704792
:10D2B80004250020064B53F820301A681B89A1F575
:10D2C8007A7159434FF47A7391FBF3F11160704707
:10D2D80004250020054B98420CBF054A054A1388CF
:10D2E80001339BB213800020704700BF00540040F8
:10D2F800F00F0020F20F002038B510F80E2C50F86F
:10D30800043C04465AB9012200F80E2C20F80C1CE3
:10D31800997A18680222BDE83840FCF7F9BB30F862
:10D328000C2C20F80A1C891A89B220F8081C084A13
:10D3380010F80F0C002522F8101004F80E5C18687D
:10D34800997A2A46FCF7E4FB04F8065C38BD00BF6E
:10D35800A0320020044B53F820301BB107289CBF93
:10D368001B681960704700BF50020020074A136805
:10D378009B060AD5064B00211970064908684FF626
:10D38800FE7303400B602023536070470000024087
:10D39800213400201C0002402DE9F047664D2B681F
:10D3A80066490A78581C02F0FF068E460AB1034601
:10D3B800F6E72B60687BAB6895F80C80AA7B37464C
:10D3C80039B2202900F09B80DFF880C10CEB810383
:10D3D8003CF82110DC789B78C3F1FF039BB2002B4B
:10D3E80065D0C3F1FF0363434FF03C0C1B12B1FB44
:10D3F800FCF9B9F1050F5DD8DFE809F0030B1A292C
:10D408003A4AE01ADAB24143B1FBFCF01044C0B228
:10D4180051E0B1FBFCF00CFB101189B2DAB2C1F19A
:10D428003C01E31A4B432046B3FBFCFC94442CE03C
:10D43800B1FBFCF00CFB10115FFA83F8E21A89B219
:10D448004A43B2FBFCF24244D2B2204632E0B1FB7E
:10D45800FCF90CFB191189B25FFA83F8E01AC1F1E3
:10D468003C014843B0FBFCF04044C0B2224621E0F6
:10D47800B1FBFCF80CFB1811D8B289B2E31A01FB16
:10D4880003F2B2FBFCFC224684445FFA8CF412E0FF
:10D49800B1FBFCF80CFB181189B2D8B2C1F13C0100
:10D4A800E31A4B43B3FBFCF20244D2B203E0224638
:10D4B800204600E044464FEA042C4CEA004C4CEA73
:10D4C800020C172306F117014FF0010808FA03F8B8
:10D4D800C91A18EA0C0F89B2DFF8748014BF4FF02C
:10D4E80011094FF0090913F1FF3308F80190E9D247
:10D4F80018360137B6B2BFB2114BA04660E7AA731F
:10D50800AB60104AE98001238EF800300E4985F897
:10D518000C8040F22A336873AE80536000234B625C
:10D528000B889BB243F001030B80136843F001039F
:10D538001360BDE8F08700BFE02000202134002000
:10D54800EC2000201C000240002C0140220E00208C
:10D55800D102002073B506460D46002401232A880F
:10D56800A34013421AD0AA78009302F003038DF85F
:10D578000430EB78022B03D0032B0CBF03230123C9
:10D588008DF805303046C2F301136946C2F38102B3
:10D598008DF806308DF80720FAF700F90134102CC1
:10D5A800DCD102B070BD2DE9F04F734EF57B074614
:10D5B8000C4687B011469A4600686B1C9146224675
:10D5C8004FF0020BF37302F077FF3B897868ADF8F0
:10D5D800043001A98DF806B08DF807B0FFF7BAFF3F
:10D5E8000023ADF80A30ADF81230ADF816307023CC
:10D5F8000193BA7A3C68CDF80CA0012306F1100813
:10D608002D01ADF808304FF48073A844ADF810B080
:10D61800ADF814300C2A7ED8DFE802F0077D7D7D56
:10D628000F7D7D7D387D7D7D5E00204601A9F9F75F
:10D6380009FFA36943F0080326E0236A4F4823F053
:10D6480010032362236A6168A26922F0807222F4BF
:10D65800E642844242F4E04206D000F5006084428B
:10D6680002D043F0300307E023F0E00321F44061E7
:10D6780043F0300341F480616160A261C4F838A0CE
:10D688002362A36943F40063A36144E0236A3B482F
:10D6980023F480732362226A6168E369844223F079
:10D6A800730343F0700306D000F50060844202D093
:10D6B80042F4407207E022F4606221F4405142F4DF
:10D6C800407241F480516160E361C4F83CA0226279
:10D6D800E36943F008031DE0236A284823F48053D4
:10D6E8002362226A6168E369844223F4E64343F4CF
:10D6F800E04342F4405203D000F50060844201D177
:10D7080041F480416160E361C4F840A02262E369AA
:10D7180043F40063E3613A7B3B681AB15A6C42F404
:10D7280000425A641A8892B242F001021A80BA7A08
:10D738000C2A18D8DFE802F0071717170B17171766
:10D748000F1717171300721903F134010AE0721941
:10D7580003F1380106E0721903F13C0102E0721985
:10D7680003F14001116135444046A5F818906B61FA
:10D7780007B0BDE8F08F00BFE0200020002C01407A
:10D78800F8B53A4E3A4C4000C7B24FF420453068DD
:10D79800C4F8D050D0F818E01EF4004F05D0AE46BB
:10D7A800013DBEF1000FF5D116E0D0F804E0314D8F
:10D7B8000EEA050545F490353D4345604FF4204594
:10D7C800C4F8D050D0F818E01EF0020F2DD1AE46A4
:10D7D800013DBEF1000FF5D1C4F8D0501FE0294635
:10D7E800013D0029F8D081694906F8D5C4F8D05020
:10D7F80020494568294041F0007141F4105141EA3F
:10D808000241394341604FF42041A2B13068856933
:10D818006D071ED411F1FF31F9D2C4F8D010FFF70B
:10D8280059FD003018BF0120F8BD4FF42045816232
:10D83800C4F8D050D7E73068C4F8D0100B468269D6
:10D8480092060CD41A46013B002AF8D1C4F8D0300D
:10D85800E5E7416A03F8011B013AD2B2D3E7C4F8FD
:10D86800D0302023C3610120F8BD00BFEC0F002099
:10D87800E0200020009800FC400070B5C5B2324896
:10D88800324B00684FF42044C3F8D0408669360410
:10D8980004D52646013C002EF8D113E046682C4CEE
:10D8A800344044F0807444F490342C4344604FF482
:10D8B8002044C3F8D0408669B60729D42646013CDF
:10D8C800002EF8D1C3F8D0401CE02146013C0029C5
:10D8D800F8D081690E06F8D544681D49214041F009
:10D8E800007141F48031294341604FF42041C3F86D
:10D8F800D0108469A40711D40C460139002CF8D142
:10D90800C3F8D010FFF7E6FC003018BF012070BD47
:10D918004FF420448162C3F8D040DAE782624FF4C2
:10D928002042C3F8D0208169890606D41146013AFD
:10D938000029F8D1C3F8D020E4E7C3F8D020202389
:10D94800C361012070BD00BFEC0F0020E020002063
:10D95800009800FC034B4FF4004208B19A617047ED
:10D968001A85704700080048034B4FF4004208B17D
:10D978001A8570479A6170470008004838B5294CE5
:10D988002DED048B94ED008AB0EE480A0546FDF7AC
:10D9980023FAF0EE408AB0EE480AFDF7BAF994EDA2
:10D9A800019AB0EE408AB0EE490AFDF715FAF0EE9A
:10D9B800409AB0EE490AFDF7ACF995ED017AD5ED3C
:10D9C800027A95ED006A68EE676A27EE088AE7EE44
:10D9D800286A68EE000A67EE807AE6EE290AB0EE59
:10D9E800660AE7EEA80A08F0F5FDDFED0F7A20EEEB
:10D9F800270ADFED0E7A80EE270AD4ED027A30EEA0
:10DA0800270AF2EE047A80EE270A08F0E1FCBDEC62
:10DA1800048B83B21A0444BF00F5B47083B218B201
:10DA280038BD00BFB42100200000E144DB0F4940AD
:10DA38002DE9F04F2DED028B85B0074602939C4BE4
:10DA48001B889807934636D5109B9A48DC89B0F90D
:10DA580000301B1B03F2F31540F2E632954203D85F
:10DA6800002BB8BF5B4201E04FF4FA73B0F9022013
:10DA7800121B02F2F31440F2E630844203D8002A63
:10DA8800B8BF524201E04FF4FA729342B8BF13464E
:10DA9800C3F5FA73052293FBF2F30A22643B53435E
:10DAA8003A7FD2105343642293FBF2F3134423EAE0
:10DAB800E373DBB200E064230093CB1C0193B84608
:10DAC8000025019BDFF810A213F8016F0193022DC6
:10DAD8004FEA450905D1BAF904301B365E43761181
:10DAE80046E075493AF8152031F91510022012FB65
:10DAF8000011CBF10002914203DB59450A46A8BF49
:10DB08005A466E49029B31F90940141B33F9152016
:10DB1800144404F0A3FD88B107EE904A684AB8EEB1
:10DB2800E70AB2EE048A505D80EE080A03F002FBB1
:10DB380020EE080AFDEEC07A17EE904A5C4A128879
:10DB4800D10712D43AF909301B365E4393074FEADE
:10DB580026160DD5BB7C5C439DF900305C436423DD
:10DB680094FBF3F406EB241602E03E7A7443261184
:10DB7800544B042433F9093093FBF4F4524B03F16A
:10DB88000C02341BAA5C924698F801205146624365
:10DB98004A43642192FBF1F297F85110D21108EE32
:10DBA800102A59B103F11000B8EEC80A00EBC500FD
:10DBB800D3ED0A0AFCF74AFEBDEEC08ADFF808E199
:10DBC800424B98F80B6018880EF12C0300FB04F206
:10DBD80053F82510D21206FB0216B6F5001F3C4A70
:10DBE800A8BF4FF400169642B8BF16460EF1380289
:10DBF80043F8256052F8253042F82540E31A0EF123
:10DC080044014FF6FF720009B2FBF0F043430EF1F6
:10DC1800500051F8254050F8252040F825409B1128
:10DC2800224441F8253097F850101A444FEA850CE1
:10DC3800761300EE102A79B10EF15C00B8EEC00A36
:10DC480000EBC500DEED0A0ACDF80CC0FCF7FEFDBE
:10DC5800DDF80CC0BDEEC00A98F8153010EE102A99
:10DC680018EE101A5A43534653431A463144642354
:10DC780092FBF3F3174A1B12194422F8091018EE05
:10DC8800100A02F1080101354CF8010002F11401F3
:10DC98002032032D4CF801604CF8023008F10108DD
:10DCA8007FF40FAF05B0BDEC028BBDE8F08F00BF6D
:10DCB800E0110020782700201C34002034270020A1
:10DCC8003896010814100020B4210020E80F002025
:10DCD8000000E0FF28220020001100201FB5084B9B
:10DCE8001B681B0309D58DF80400029100230D2041
:10DCF80001A98DF80530FDF7C1FF05B05DF804FBFB
:10DD08003C27002010B50A4A0A4B11689B68126824
:10DD18009142F8D1084AD2F8A0404FF47A7000FB3B
:10DD280004F2D31AB3FBF4F300FB013010BD00BFBB
:10DD38006027002010E000E0B421002038B5044638
:10DD4800FFF7E0FF0546FFF7DDFF401BA042FAD3CF
:10DD580038BD10B504462CB14FF47A70FFF7EEFFCA
:10DD6800013CF8E710BD024A13680133136070479D
:10DD780060270020064BD3F8A42010B51C4602B13A
:10DD88009047D4F8A83013B1BDE81040184710BD2B
:10DD9800B4210020014B1B68184700BF083400203D
:10DDA80010B50020FFF7F6FF074B00241C7004F0A5
:10DDB8002FFC064B83F8AC40C3F8B040A3F8B4403E
:10DDC800C3F8B84010BD00BFB2330020B421002012
:10DDD80010B510B9BDE81040E2E700230C225A4301
:10DDE8000C4C1119125D824203D00133102BF5D16E
:10DDF80010BD094BD3F8B80018B14A784078824270
:10DE080006D20022C3F8B810A3F8B420C3F8B02093
:10DE180010BD00BF3C960108B421002010B5400099
:10DE28001428A8BF14200023074A022199540B4440
:10DE380099181424834201F8014CF5DBFF21D154D1
:10DE48000F20BDE81040C3E74025002038B540F258
:10DE5800DB15124B082268439A61851E0B24013C8E
:10DE680014F0FF0412D00D4A938A9BB283F0080382
:10DE780093822846FFF76DFF0120FFF78BFF1920DB
:10DE8800FFF767FF0020FFF785FFE8E7044B054A27
:10DE98001A60054B054ADA6038BD00BF0004004827
:10DEA800FC9F0020EFBEADDE00ED00E00400FA05A7
:10DEB8000749D1F8A4300A462BB1D1F8A8300BB1E4
:10DEC8000F20C3E7012302EB8303C3F8A4007047C4
:10DED800B421002003685B69184703681B69184769
:10DEE8000368DB68184703689B68184703685B6822
:10DEF800184703681B6818472DE9F84FB0F9023036
:10DF0800934218BF00232DED028B18BF03700578CC
:10DF180004460E469146002D40F08B8007EE902A6D
:10DF28009FED770AF8EEE77AB6EE008A27EE800AC8
:10DF3800DFED747A20EE270AA04620EE080A08F0E2
:10DF4800BDFADFED716A60EE266AB7EE006AB0EEE0
:10DF5800667AA0EE007A40F2DC536365D0EE006A80
:10DF68001023A4F8523037EE067A76EE866AC6EEAB
:10DF7800077A1823A4F85030274684ED046A27EE60
:10DF8800807A27EE007A77EE075A84ED017AC4ED9D
:10DF9800025A70EE005A84ED037AB8EE007AA5EEC4
:10DFA800807A27EE877A67EEA67A84ED057AC4ED43
:10DFB800067ADFED567A98ED047A27EE277AF0EEA6
:10DFC800678AB5EEC07AF1EE10FA4CBF77EE487A60
:10DFD80077EE087A013517EE900A04F071FDD8ED56
:10DFE800017A67EEA87AC7E90E01F5EEC07AF1EE7C
:10DFF80010FA4CBF77EEC87A77EE887A08F10408F1
:10E0080017EE900A04F05CFD032DC7E9080107F13B
:10E018000807CED1A6F2DC531B042367E3676367C6
:10E02800C4F88030A367C4F884300123A4F80290B0
:10E038002370D4F85490B4F95280636A276A206F29
:10E04800E26FD4F840C0D4F88010C4F88020C9EB3F
:10E05800060606FA08F64FEAE67B734307FB0B331E
:10E068002667A7FB06671F44636C656F60674FEA06
:10E07800E27B53430CFB0B3EACFB02237344B61A02
:10E0880067EB0307E36AA26AC4F884104FEAE07BEF
:10E09800434302FB0B3EA2FB00237344B6185F41C7
:10E0A800E36CA06CB4F95020A5674FEAE17B4B43C1
:10E0B80000FB0B33A0FB01011944636B361A206B7C
:10E0C8004FEAE57B05FB03F300FB0B3367EB010726
:10E0D800A0FB050119448019794104F0C7FC08F137
:10E0E800FF3201239340E067C01841EBE3714246D9
:10E0F80004F0BCFCBDEC028B4844BDE8F88F00BFBF
:10E108006F12833ADB0F4940F404B53F0000804B9F
:10E118002DE9F0410024224B1E78E0B2B0420CD227
:10E12800204B33F81010204B53F820301BB10B282C
:10E1380001D8DB6898470134EDE71C4B1B685B038B
:10E148002CD500242346E2B2B24227D2164F57F804
:10E15800242055689D424FEA840817D0284602F0CB
:10E1680023FAEFF31283502282F3128810496A6A65
:10E178004FF0280E0EFB00100132C0F8E0206A694B
:10E1880042F001026A61DBB283F3118857F8083064
:10E198001B6800221A6001342B46D4E7BDE8F081E1
:10E1A8000025002030100020042500203C270020F6
:10E1B800B421002008B50E4B1B6813F4805F0D4B8B
:10E1C80014BFD3F8D431D3F8D8319A880A4B1978C8
:10E1D8000023D8B2884204D2084820F8132001331B
:10E1E800F7E7FFF795FF3220BDE80840B1E500BF2B
:10E1F8003C270020B42100200025002030100020FA
:10E208000A4B1A680A4B30B502F48052D3F8D4414D
:10E21800D3F8D85100230AB1A18800E0A98805489D
:10E2280020F8131001330C2BF5D130BD3C2700200A
:10E23800B4210020E224002070B5124D00242146AC
:10E2480005F2DD10702285F8DC4107F0B2FE2146A8
:10E25800D5F850320B4A0B4493F9020080B102F210
:10E26800DD141E680E5108199C8884809B7983717F
:10E2780092F8DC3107310133702982F8DC31E7D1BB
:10E2880070BD00BFB4210020094B1A680E2303FBA0
:10E298000020437AFF2B07D0064A12789A4203D906
:10E2A800054A32F8130000E0808800B2704700BFCA
:10E2B800DC2000204C330020782700202DE9F04393
:10E2C8002DED048BE04C8BB0FFF71CFDD4F85432D5
:10E2D80094ED966AD4F85C62C4F85402C3EB000863
:10E2E80007EE908AB8EE678A0DF1040E002528EE35
:10E2F800066A96F800C0D54804F518712A4677468C
:10E30800D34B33F9123007EE903AF8EEE77AD14B57
:10E3180067EE867AEEEC017ABCF1000F1CD007EEAE
:10E3280090CAF8EEE76AB7EE007AC7EE266A33F9C4
:10E33800123007EE903AF8EEE77A37EE667A67EE33
:10E34800A67AD1ED006AE6EE877AC1ED007AFDEE95
:10E35800E77A17EE903A01E033F81230438030F84C
:10E36800023F0132032A13FB035501F10401C7D10F
:10E37800DFF81C93B84864236B43B9F800506D4329
:10E3880093FBF5F5493D3946ADB2FCF78BFD3B2DC6
:10E39800D6ED016A11D9B4F98032D4ED9F0A07EE9F
:10E3A800903AF8EEE77AAD4BF4EEE70AF1EE10FAA0
:10E3B8001EDD1A7842F008021DE0F7EE007A36EE0C
:10E3C800A77AA54A87EE877A0023A54931F9131061
:10E3D8000133032B07EE901A92ED006AF8EEE77A04
:10E3E800E6EE267A67EE877AE2EC017AEDD1D2E79B
:10E3F8001A7822F0080294ED9E0A1A7008F0EAF8DA
:10E40800B0EE409A84ED000A94ED9F0AD4ED9E7A0E
:10E41800D4ED9D8ADFED939A934D20EE000AF1EE3C
:10E42800688AA7EEA70A08F079FAF0EE400AB0EE7B
:10E43800680A08F0CFF8F0EE408A84ED010A29EE68
:10E44800290A07F0C5FF28EEA90A288007F0C0FFAF
:10E45800864B68801B681A0721D585483946FCF722
:10E4680021FDD6ED026A824AF7EE007A36EEA77AE7
:10E47800002387EE877A7F4931F913100133032B84
:10E4880007EE901A92ED006AF8EEE77AE6EE267A41
:10E4980067EE877AE2EC017AEDD175482AE0764D8D
:10E4A80039462846FCF7FEFC95ED010A95ED007A01
:10E4B800D5ED027A20EE000AA7EE070AA7EEA70A12
:10E4C80008F02CFAB5EE400AF1EE10FA11D0D5EDAD
:10E4D800007AC7EE807AC5ED007AD5ED017AC7EEED
:10E4E800807AC5ED017AD5ED027A87EE800A85ED4E
:10E4F800020A6148FFF742FA604BDFED617A188043
:10E508005E4B9FED607AB3F9003028EE278A07EE5C
:10E51800903A534BF8EEE77AB3F9002067EEC77AE2
:10E52800B1EE499ACDED067A07EE902AB3F90220AA
:10E53800B3F904308DED049AF8EEE77AF1EE688AC3
:10E54800CDED077A07EE902AF8EEE77A07A8CDED29
:10E55800087A07EE903AF8EEE77A04A9CDED058A35
:10E56800CDED097AFCF79EFC73789DED097A012BB5
:10E5780019D1454B1B785B070FD4D4F89032402251
:10E5880093FBF2F29B1A07EE903AF8EEE77A77EEF1
:10E59800877AFDEEE77AC4EDA47AD4F89032402267
:10E5A80093FBF2F301E0B9F800309DED070A07EE9E
:10E5B800903AF8EEE77A37EE677AD4EDA57A8DEDE2
:10E5C800097A94EDA67A38EE077A88EE078A9DEDE7
:10E5D800097A37EE677AE8EE077AB0EE678AC4ED13
:10E5E800A57A07F0F5FED4F89C522978FCF782FB4F
:10E5F800D4F8A0329DED080A1844C4F8A00207F028
:10E60800E7FE2978FCF776FBD4F8A432B0EE480A86
:10E618001844C4F8A40207F0DBFE6978FCF76AFB2B
:10E62800D4F8A832194A18441368C4F8A802434415
:10E638001360D4F8AC320133C4F8AC320BB0BDEC83
:10E64800048BBDE8F08300BFB4210020E81000204F
:10E65800141000202024002028240020201100204D
:10E66800EA1000204C3D0F44342700201C110020E4
:10E67800382400204413002068000020F8100020EF
:10E68800BD37863535FA8E3C22340020043400200C
:10E698002000002001380A4B042804D8DFE800F0E5
:10E6A8000507090B0D00074A08E0074A06E0074A74
:10E6B80004E0074A02E0074A00E0074A1A60704788
:10E6C8008000002055F3000839DA0008892601087F
:10E6D80007F0000865EC0008E5E600082DE9F04FB2
:10E6E8002DED0A8B89B08046059390F8503004913F
:10E6F80002921BB1322BA8BF322300E0012307EEA0
:10E70800903AF8EEE7BADFEDA87AA84B9FEDA8CAD1
:10E718001B88C7EEABBA002B08BF012307EE903A5F
:10E72800B8EEE7AAA34B03932AEE0CCA1A887BEE2D
:10E738008CBA12F0020FCCEE2BBA27D09E4AB2F94F
:10E748000030B2F9022083EAE37182EAE270A1EBB9
:10E75800E371A0EBE27088420446B8BF0C46B4F5FA
:10E76800E17F16DA88429FED95BA05DD002AD8BF09
:10E77800524207EE902A04E0002BD8BF5B4207EE16
:10E78800903AF8EEE77A87EE8BBA04E09FED8CBA00
:10E7980001E0B7EE00BADFF858A2DFED899ACDF8AC
:10E7A80004800AF1080B0AF110070AF11C09002479
:10E7B800F0EE69AA834931F914307F4909EE103A1D
:10E7C800B8EEC99A31F91430F5EE047A29EE279A91
:10E7D80008EE103A039BBDEEC99A1988F8EEC97A7B
:10E7E8009FED799A89074FEA440627EE899AB8EE91
:10E7F800C88A00F08180754931F9143007EE903AE3
:10E80800F8EEE77AB0EE007AE8EE077A029B584213
:10E81800FDEEE77A17EE901A814203DB8B42A8BF20
:10E828000B4618466A49059B715E401A33F9141065
:10E83800084407EE900AF8EEE78A03F00FFF48B1A4
:10E848006449F2EE049A88EEA90A085D02F072FCA7
:10E8580060EE298A98F81C30DFED5F6A0AEE903A7C
:10E8680098F8083007EE903AF8EE677AF8EE6AAA58
:10E8780068EEA77AB1EE047A67EEA67A2AEE877A6E
:10E88800FDEEE77A17EE901AF1EE477AFDEEE7AA69
:10E898001AEE903A994208DBFDEEC7AA1AEE903AB2
:10E8A8008B42A8BF0B460AEE903AD9ED007AE8EE03
:10E8B8008C7ABBEE0E7AF4EEC77AF1EE10FAF8EE27
:10E8C800EAAA09D4B3EE0E7AF4EE477AF1EE10FA1A
:10E8D800C8BFF0EE477A01E0F0EE477AC9ED007A5A
:10E8E80098F8123009EE903AF8EE699A67EEA97A2C
:10E8F800DFED3A9A67EEA99A039B1988CA0779D47B
:10E908003048305E0028B8BF4042B0F5206F02DDC5
:10E918000020386026E0019B9FED317A5B7868EE35
:10E92800077A07EE103AB8EE477A87EE877AD7ED7E
:10E93800007A37EE497AE7EE0C7A9FED2A7AF4EE00
:10E94800C77AF1EE10FA09D49FED277AF4EE477AE8
:10E95800F1EE10FAC8BFF0EE477A01E0F0EE477A20
:10E96800C7ED007A019BD7ED007ADB7A08EE903A82
:10E97800F8EE688A8B0768EEA77ADFED1C8A67EEE7
:10E98800A88A3BD538EE6A8AF0EE6A7AEBEE087A06
:10E9980078EEE98AB0EE678AF0EE697AEBEE287ACB
:10E9A800F0EE678A2AE000BF83F9223EE80F0020D4
:10E9B800BD378635E0110020001100200000E1433A
:10E9C8000000000014100020CDCC4C401C34002066
:10E9D80034270020389601086F12033C0AD7A33D5C
:10E9E8000000A043000040C3000040430AD7233C76
:10E9F80064240020F0EE698AB0EE6A8A85499FEDAA
:10EA0800867A635C98F8511007EE903AF8EEE77A48
:10EA180067EEC97AA7EE878A59B18048804DB0EE73
:10EA2800480A00EBC400D5ED000AFBF70FFFB0EE73
:10EA3800408A9AED007ADBED007A7A49AAEC019ACD
:10EA480039EE477A635C784D87EE0C7A043709F122
:10EA5800040909EE103A37EE677AB8EEC99AEBEE78
:10EA6800877A38EE280AEBEC017A67EE897A9FED0F
:10EA78006F9A27EE899A30EE490A07F0A9FCBDEE95
:10EA8800C88A6B49A85318EE103AFDEEE88AB1EE31
:10EA9800499A18EE902A41F82430BDEEC99A654B80
:10EAA800654E43F8242019EE102A46F82420019ACE
:10EAB80006910132019207930CB901247AE6049A6F
:10EAC8005E4B9479B3F90430640028345C435C4BA2
:10EAD800B3F9043000EE103ABAEECF0A07F078FC2A
:10EAE8006411201A002C07EE900AB8BF6442322C39
:10EAF800F8EEE76A534A02DD0023936026E0BDEE94
:10EB0800CAAA1AEE103A23F0030307EE903AB8EEB9
:10EB1800E7AADFED4D7A98F80D30CAEE277A07EEAE
:10EB2800103AB8EE477A936826EE877A67EE277A26
:10EB3800FDEEE77A17EE901A0B4444498B42A8BFC2
:10EB48000B4643498B42ACBF9360916093685B135B
:10EB5800B3F5807FA8BF4FF480736FF0FF02934234
:10EB6800B8BF134607EE903AF8EEE78AFDEEE67A6C
:10EB780098F8032017EE903A53439B1107EE903A0A
:10EB8800344B1B78032BB8EEE78A14D9B8F84E201B
:10EB9800B2F5FA7F0FD2FDEEC87A534217EE901AFB
:10EBA800994204DB914217EE903AA8BF134607EE4C
:10EBB800903AB8EEE78A98F8511049B1184B2648B0
:10EBC800D3ED000AB0EE480AFBF740FEB0EE408AEB
:10EBD80078EE287AFDEEE77ACDED017ABDF80430BB
:10EBE800AB801BB200EE103AB8EEC00A07F0F0FB9B
:10EBF800069BA880BDEEC88AFDEEE88A83ED028AEE
:10EC0800079BC3ED028A0023B36009B0BDEC0A8BF1
:10EC1800BDE8F08F88240020A69B443BC421002037
:10EC2800DC2100208B24002028220020F7CC9238F9
:10EC3800302200203C220020482200200011002021
:10EC480014100020E021002000803B45FEFFFF0F4C
:10EC5800020000F000250020D42100202DE9F04F0B
:10EC68002DED028B87B000260493C14B0391B3F9B5
:10EC78000280B3F900300292B8F1000FB8BFC8F1B2
:10EC88000008002BB8BF5B429845B8BF9846B8F556
:10EC9800FA7F0746A8BF4FF4FA780090B24601966B
:10ECA800B1463446B34D2B88990757D0B04BB24A7A
:10ECB80033F8143032F91420022013FB0022029B8F
:10ECC8005B429A424FEA440103DB029B9342A8BF8E
:10ECD8001346AA4A31F902B0049A32F91420CBEB50
:10ECE800030303EB020B03F0B9FC88B107EE90BAFB
:10ECF800A34BB8EEE70AB2EE048A185D80EE080A64
:10ED080002F018FA20EE080AFDEEC07A17EE90BA63
:10ED18003B7A642203FB0BF393FBF2F33A7F6FF029
:10ED2800040909FB02F94B4504DB02EB820999450A
:10ED3800A8BF9946934A52F824100BEB010342F2FC
:10ED480010718B42A8BF0B468F498B42B8BF0B4648
:10ED580042F82430BA7C53431B1301932D8805F0E5
:10ED68000303012B38D0824B884933F914A0009B48
:10ED780051F824E093F801C0854B33F9140080EA78
:10ED8800E073A3EBE073B3F5206F4FEA840616DC5B
:10ED98000AEB8A031A0192FBFCF3042290FBF2F0BF
:10EDA800181A8644BEF57A5FA8BF4FF47A5E794B8D
:10EDB8009E45ACBF41F824E041F8243002E000232E
:10EDC80041F824308B597D2693FBF6F6009BDB7ABD
:10EDD8007343402693FBF6F6AA0711D50198C8F5A8
:10EDE800FA7208FB0AF308FB06F54FF4FA7102FB06
:10EDF800093302FB005593FBF1F395FBF1F505E0B0
:10EE0800EB074DBF019D354653464B46604A32F9E4
:10EE18001410042291FBF2F25F49615C4A436FF0DF
:10EE28004F0192FBF1F297F8511013444FEA440B4B
:10EE380008EE103A59B1594B5948D3ED000AB8EECB
:10EE4800C80A00EBC400FBF701FDBDEEC08A504BB9
:10EE5800544A3BF803003BF902302BF8020001B298
:10EE6800101D0C32CB1A50F824E0042193FBF1F169
:10EE780052F8243040F8241073440B4497F850108B
:10EE880042F824E04FEA840C00EE103A79B1434A84
:10EE98004548D2ED000ACDF814C0B8EEC00A00EB20
:10EEA800C400FBF7D3FCDDF814C0BDEEC00A3F4A2E
:10EEB8003F49125D3F4810EE103A5343202293FB1E
:10EEC800F2F318EE102A2A44D21A2BF8012018EE71
:10EED800102A4CF80020384A4CF80250374D5B4253
:10EEE8004CF80530009B013300930CB90124D9E696
:10EEF8001F4B97F80DE0B3F90440039B9B790F3340
:10EF08005B0063435B11224C002B4FF00406B4F9FD
:10EF1800044094FBF6F41D4EA3EB0404B8BF5B4217
:10EF2800322BD6F808C00DDC254B0EFB04CE7345FA
:10EF3800A8BF7346DFF890E07345ACBFB360C6F86E
:10EF480008E001E00023B360FB785C431D4B1B78AD
:10EF5800032B4FEAA4143AD9B7F84E30B3F5FA7F29
:10EF680035D25F42BC4231DB9C42A8BF1C462EE032
:10EF780000110020E01100201C340020342700205C
:10EF88003896010890240020F0D8FFFFE0210020E7
:10EF98001410002080C1FFFF88240020DC210020FD
:10EFA800C421002098240020102200208B24002057
:10EFB80028220020302200203C2200204822002065
:10EFC800FEFFFF0F00250020020000F03C46B3685A
:10EFD800846043F34F33B3F5807FA8BF4FF4807349
:10EFE8006FF0FF06B342B8BF3346E61893600023BC
:10EFF8008E80AB6007B0BDEC028BBDE8F08F2DE9C9
:10F00800F04F2DED028B85B083460293B84B0191EA
:10F018001D88009205F00205ADB295B1B54BB3F964
:10F028000250B3F90030002DB8BF6D42002BB8BFB5
:10F038005B429D42B8BF1D46B5F5007FA8BF4FF49F
:10F048000075D9460026AB4BAB4C33F81610AB4BCA
:10F0580054F8267033F9163083EAE37EAEEBE37E8C
:10F0680008B2BEF5206F4FEA460A4FEA40004FEA61
:10F07800860812DC4FF0040E93FBFEF3C31A1F44FC
:10F08800B7F57A5FA8BF4FF47A579D4B9F42ACBF44
:10F0980044F8267044F8263002E0002344F826306D
:10F0A80054F8087099F80B3099F80140FF115F4344
:10F0B8008F4B1B8844439B074FEAA7174FEAA414BA
:10F0C80056D0904B33F90A30022011FB0031009BD7
:10F0D8005B42994203DB009B8B42A8BF0B468A49DF
:10F0E8003AF90110591A029B33F91630CB1808EE79
:10F0F800103A03F0B3FA68B1B8EEC80A834BB2EE1F
:10F10800048A80EE080A985D02F014F820EE080AD6
:10F11800BDEEC08A7E487F4958F8003018EE102AA4
:10F1280042F2107E13447345A8BF73468B42B8BFA2
:10F138000B4648F800309BF808109BF81C00514318
:10F1480000EB8000C911C0F1000E714503DB81425C
:10F15800A8BF01468E469BF812104B431B13FF1A9B
:10F16800CEEB04046F436C4303EB67270EEB642478
:10F17800624B04213AF9030090FBF1F16648805D87
:10F188004143A4EBA1129BF8511008EE102A69B173
:10F198006248634C0393B8EEC80A00EBC600D4ED8E
:10F1A800000AFBF753FB039BBDEEC08A5D4933F8A9
:10F1B8000A303AF901002AF801300FFA83FEC0EB51
:10F1C8000E0E04209EFBF0F001F1040E0C3158F8ED
:10F1D8000E4058F8013048F8014023449BF850107D
:10F1E80048F80E00034400EE103A59B14C4B4E4813
:10F1F800D3ED000AB8EEC00A00EBC600FBF726FB09
:10F20800BDEEC00A49494A48895D4A4C10EE103A99
:10F2180018EE102A4B435B11D119C91A2AF80010AD
:10F2280048F804204449454A48F801705B4248F8C8
:10F23800023009F101090EB9012604E72D4B2E4EC3
:10F24800B3F90450019BD6F808E09B790F335B00B3
:10F258006B435B11294D002BB5F904504FF004079F
:10F2680095FBF7F7A3EB0707B8BF5B42322B9BF878
:10F278000D500BDC324B05FB07E5AB42A8BF2B4614
:10F28800304DAB42ACBFB360B56001E00023B36062
:10F298009BF8035005FB07F32B4D2D78032D4FEA00
:10F2A800A3130CD9BBF84E50B5F5FA7F07D26F42BD
:10F2B800BB4203DBAB42A8BF2B4600E03B46B56828
:10F2C800A36045F34F35B5F5807FA8BF4FF480752F
:10F2D8006FF0FF06B542B8BF35465E190023868039
:10F2E8008D60936005B0BDEC028BBDE8F08F00BF68
:10F2F800E011002000110020E0210020141000205F
:10F3080080C1FFFF1C3400203427002038960108F4
:10F3180090240020F0D8FFFF88240020C42100207A
:10F32800DC210020AC240020102200208B240020A7
:10F3380028220020302200203C22002048220020E1
:10F34800FEFFFF0F020000F0002500202DE9F04F1E
:10F358002DED028B87B000260493AC4B0392B3F9D2
:10F368000270B3F900300190002FB8BF7F42002B24
:10F37800B8BF5B429F42B8BF1F46B7F5FA7F8246C7
:10F38800A8BF4FF4FA77B1460296B0463446A04D6E
:10F398002B8899075BD0022C59D09C4B9D4A33F897
:10F3A800143032F91420022013FB0022039B5B4225
:10F3B8009A424FEA440103DB039B9342A8BF1346DA
:10F3C800954A31F902B0049A32F91420CBEB0303C1
:10F3D80003EB020B03F042F988B107EE90BA8F4BAA
:10F3E800B8EEE70AB2EE048A185D80EE080A01F06A
:10F3F800A1FE20EE080AFDEEC07A17EE90BA9AF840
:10F408000830642203FB0BF393FBF2F39AF81C20F9
:10F418006FF0040808FB02F8434504DB02EB82089E
:10F428009845A8BF98467E4A52F8243042F2107197
:10F438005B448B42A8BF0B467A498B42B8BF0B4648
:10F4480042F824309AF8122053431B1302932B8856
:10F4580003F00302012A01D1022C3FD172486B4A02
:10F4680030F9140032F914907049019A51F824E0E7
:10F47800567880EAE075A5EBE075B5F5206F4FEAA0
:10F4880084021EDC022C16D009EB8901090191FBCC
:10F49800F6F6042190FBF1F0361AB644BEF57A5F11
:10F4A80062496348A8BF4FF47A5E8645ACBF42F80C
:10F4B80001E0505007E089EAE975A5EBE975642D8C
:10F4C800E2DD0020885059497D26525892FBF6F615
:10F4D800019AD27A7243402692FBF6F69A0713D520
:10F4E800022C11D00298C7F5FA7307FB06F507FB43
:10F4F80009F203FB08224FF4FA7103FB005392FB55
:10F50800F1F293FBF1F508E0DB0704D5022C02D0F9
:10F51800029D424601E035464A46434B33F91410F2
:10F52800042391FBF3F34349615C4B436FF04F01B4
:10F5380093FBF1F39AF85110D3184FEA440B08EEF5
:10F54800103A59B13C4B3D48D3ED000AB8EEC80A11
:10F5580000EBC400FBF77AF9BDEEC08A324B384A9B
:10F568003BF803003BF902302BF8020001B202F12C
:10F5780008001432CB1A50F824E0042193FBF1F16F
:10F5880052F8243040F8241073440B449AF8501071
:10F5980042F824E04FEA840C00EE103A79B1264B89
:10F5A8002848D3ED000ACDF814C0B8EEC00A00EB25
:10F5B800C400FBF74BF9DDF814C0BDEEC00A224ABF
:10F5C8002249125D10EE103A5343202293FBF2F3C6
:10F5D80018EE102A2A44D21A2BF801201C4A18EED9
:10F5E800101A4CF802101B4A4CF802501A4A5B4297
:10F5F8004CF80230019B01340133032C01937FF452
:10F60800C6AE07B0BDEC028BBDE8F08F001100203C
:10F61800E01100201C34002034270020389601080F
:10F6280090240020F0D8FFFF14100020E0210020D3
:10F6380080C1FFFF88240020DC210020C421002095
:10F64800C0240020102200208B2400202822002023
:10F65800302200203C2200204822002007B5064B1B
:10F668000093064B01930649064A074B0748FBF7E8
:10F6780021FB03B05DF804FB0CA70108E1A6010813
:10F6880024AD01081DAD010800A7010834B7010821
:10F6980008B5037833B90C4B0C481978BDE8084015
:10F6A800FBF708BB06F020FD02280CD8064B1870A3
:10F6B800074B0C2202FB0030064B02301860FBF7A8
:10F6C8001FFD0548E5E708BDE024002054B7010800
:10F6D800442F002054100020DCA9010808B5037845
:10F6E8003BB90B4B0B4893F8A817BDE80840FBF74C
:10F6F800E1BA06F0F9FC022808D8054B83F8A807F8
:10F70800FBF768FCFBF720FD0348E8E708BD00BFEE
:10F718009C27002058B70108DCA9010838B50378F0
:10F7280003BB214B1B6801330F2B07D81F490C2241
:10F7380002FB03121C4695682DBB00E01C460134F1
:10F748000F2C01DD002400E005D818490C2202FB2B
:10F7580004129568BDB99C42F1D11548BDE83840FE
:10F76800FBF7A8BA06F0C0FC0F28044605D80F4AD4
:10F778000C2303FB00239D682DB921460D48BDE8E5
:10F788003840FBF797BA084B1C60FEF709FB214687
:10F798002A460948FBF78EFA0C235C43034B185D95
:10F7A800BDE83840FEF714BB740000203C96010801
:10F7B80065B701087BB7010893B7010873B50378EB
:10F7C80013B9F6F77DF83FE001AA204906F0EDFCF1
:10F7D80000240246264625469AB134B1012C08D1A8
:10F7E800104606F081FC064603E0104606F07CFC55
:10F7F800054601AA0020154906F0D7FC0134024647
:10F80800EAE70B2D03D9124812490C230CE0022C0D
:10F8180011D1A6F57A73B3F57A7F08D90C480E4949
:10F828004FF47A724FF4FA63FBF744FA0CE00B4B8F
:10F8380003EB45035E80094B094803EB4503294662
:10F84800B3F90220FBF736FA02B070BD35B00108F3
:10F85800D5AB0108F4AB0108E1B30108E0240020AE
:10F86800AAB7010838B50D4C23688342054606D16E
:10F87800F6F7E1FB204600214C2206F09AFBE36CE8
:10F88800AB4209D12846F6F7D6FB054800214C22A1
:10F89800BDE8384006F08DBB38BD00BF30120020EF
:10F8A8007C120020034B1A68D379591C1344D17178
:10F8B800187A7047C011002010B5FFF7F3FF84B223
:10F8C800FFF7F0FF04EB002080B210BD10B5FFF782
:10F8D800F3FF0446FFF7F0FF04EB004010BD064BB2
:10F8E80010B5044621461868FEF703FB034B1B6856
:10F8F80098796040987110BDC4110020C011002093
:10F9080038B5044624200D46FFF7E9FF4D20FFF7E0
:10F91800E6FF002C084C14BF21203E20FFF7DFFF34
:10F928002368002228469A71FFF7D9FF236893F8C5
:10F938004900BDE83840D2E7C01100200146002048
:10F94800DEE710B50446C0B2FFF7C9FF200ABDE8DC
:10F958001040C4E710B5044680B2FFF7F2FF200C50
:10F96800BDE81040EDE737B5828883680446100685
:10F978000D4641BF2B4991F8A8174FF4CC7000FBF6
:10F988000133D10544BF2849097802F03F0244BF3A
:10F9980001EB410103EB8103042A12D006D8012AA6
:10F9A8000DD0022A32D193F9001030E0102A0AD083
:10F9B800202A0AD0082A29D1B3F9001027E019789B
:10F9C80025E0198823E0196821E093ED000A6846CC
:10F9D800FAF7F0FF01461548FBF76CF905B3D4EDCB
:10F9E800037A6846B8EEE70AFAF7E4FF01461048DA
:10F9F800FBF760F994ED040A6846B8EEC00AFAF716
:10FA0800D9FF01460A48FBF755F909E000210948E2
:10FA1800FBF750F925B10848E1682269FBF74AF974
:10FA280003B030BD9C270020E0240020BDAE0108B3
:10FA3800B6AE0108FCAD0108B9B70108024B014692
:10FA4800D869FEF756BA00BFE024002010B5441E5E
:10FA580014F8011F21B1034BD869FEF74AFAF7E7FA
:10FA680010BD00BFE02400202DE9F74F03781BB933
:10FA78005248FFF7EBFF9EE006F036FB08280446E5
:10FA880099BF21464E484F480821FBF713F94E4BC2
:10FA980093F820200023D9B2914207D24B4951F85C
:10FAA80023100968002008600133F4E772B6013CAE
:10FAB800474A63B2012652F8334002EBC3034FF0C2
:10FAC80090475D6806FA05F84FF0040B4FF4806123
:10FAD8004FF400791FFA88FA39853846A7F8289034
:10FAE800A4F828A0ADF804100DEB0B018DF806B0B2
:10FAF8008DF80760FDF72EFD38460DEB0B01ADF8CC
:10FB080004908DF806608DF80760FDF723FD204608
:10FB18000DEB0B01ADF804A08DF806B08DF8076069
:10FB2800FDF718FD4FF090431B8A5E05FAD46D006F
:10FB380003230122AB40AA40DB4321681143216023
:10FB48004FF090414FF40070A4F828A008850820D1
:10FB5800C1F8180440F6B8314FF09040058A6D0599
:10FB680010D40139F8D14FF40073ADF804300223F2
:10FB78008DF8063001A901238DF80730FDF7EAFC5E
:10FB880062B618E0C4F818802168194021604FF067
:10FB98009041088A4005D0D5208A80B218EA000F23
:10FBA8000C484FF400764FF0080515BF8E610E859E
:10FBB80085610585EBE703B0BDE8F08FC0B70108A4
:10FBC80007B8010833B80108E02400200425002004
:10FBD800F4B6010800040048F7B52B492B4B087808
:10FBE8002B4D1C682B4B05EB80001A882A4BD0F84C
:10FBF800C0101B78294800914FF47A71B4FBF1F1D9
:10FC0800FBF758F826484821FBF754F8254B1F689E
:10FC18000026F3B205EB8302D2F8D010E9B1012433
:10FC28009C403C4217D0220715D01F4AD25C0B20BB
:10FC380000FB0323164A1D4802EB8303D3F8F02088
:10FC4800FBF738F8022C06D1194B93F85C1011B168
:10FC58001848FBF72FF80136DBE71748FFF7F6FEE1
:10FC6800164B17481A68174B9A420CBF164B174B7E
:10FC78001A88174B198892B240F2D47303B0BDE8C2
:10FC8800F040FBF717B800BF6C1100206027002078
:10FC98003C9601080C1100207D0000205EB8010888
:10FCA800A1B801081C11002084000020B1B8010887
:10FCB800E0240020B9B8010801B90108EC0F0020C0
:10FCC800BDB8010800540040F00F0020F20F0020DA
:10FCD800E80F00202DE9F0410024804625460F4E0C
:10FCE800A7594146384606F0E7F958B139460C4855
:10FCF800FAF7E0FF30190021FFF735FE0948FFF752
:10FD0800A5FE01351434B4F5486FE8D11DB906488D
:10FD1800BDE8F0419AE6BDE8F08100BFDC97010834
:10FD280045AF010801B9010866AC01082DE9F04F9B
:10FD38002DED028B83B0054606F07FF9064620B10B
:10FD4800012817D12B782A2B14D15B48FFF77EFEA8
:10FD580000245A4D5A486159FAF7ACFF2819314620
:10FD6800FFF701FE14345748FFF770FEB4F5486FEB
:10FD7800EFD19CE028463D2106F051F9002800F01B
:10FD88008F800346994613F8012D202AFAD0441C87
:10FD9800204606F0A9F980462046FAF781FDC5EB12
:10FDA8000909B0EE408A0026DFF830A1142202FBD0
:10FDB80006F40AF5D07B54F80B70384606F03DF986
:10FDC80003461A4628463946019306F03FF9019B37
:10FDD80000285BD15FFA89F29A4257D10AEB0402F4
:10FDE800D2ED6B7AF8EEE77A0BEB0405B4EEE78A0E
:10FDF800F1EE10FA48DBD2ED6C7AF8EEE77AB4EE61
:10FE0800E78AF1EE10FA3FD8B2F8A431D2F8A82167
:10FE180013F0200F08BF08EE108A1C0641BF2A49BC
:10FE280091F8A8174FF4CC7404FB0122D90544BFFC
:10FE38002649097803F03F0344BF01EB410102EB77
:10FE48008102042B18EE100A0BD004D8013B012BB9
:10FE58000ED810700CE0102B05D0202B06D0082BE4
:10FE680006D1108004E082ED008A01E082ED008A6C
:10FE780039461748FAF71EFF2846002103B0BDECA3
:10FE8800028BBDE8F04F6EE5124803E00136A02E64
:10FE98008AD1114803B0BDEC028BBDE8F04FD5E51F
:10FEA800284603B0BDEC028BBDE8F04F12E703B063
:10FEB800BDEC028BBDE8F08FEFB80108DC970108B4
:10FEC80045AF010801B901089C270020E024002063
:10FED80004B901080FB9010866AC01083C9601088D
:10FEE80008B50748FFF7B2FD064BD869F6F798F84A
:10FEF800FEF760F9FBF744F8034B044ADA6008BDE3
:10FF08002FB90108E024002000ED00E00400FA0504
:10FF180008B50548FFF79AFD01F08AFBFBF75AF888
:10FF2800BDE80840DCE700BF3BB9010808B5044854
:10FF3800FFF78CFDFBF74EF8BDE80840D0E700BF9F
:10FF480051B901086C4B6D4A2DE9F04F5E89146870
:10FF58004FEA062AB4EB0A0A9C884FEA04481C892F
:10FF68004FF000054FF0000B65EB0B0BA4FB0A6785
:10FF780004FB0B77F40944EA476418EB04065C8831
:10FF88004FF000094FEAE7154FEAC438DC8849EB1F
:10FF9800050787B0CDE90467A4FB0A6704FB0B7764
:10FFA800340A44EA076418EB04064FEA27259C89BB
:10FFB8004FF0000949EB0507CDE90067AAFB046784
:10FFC80004FB0B77F40D44EA472414F5FA664FEA6C
:10FFD800E75545F10007B6F5FA6F77F10003CDE96B
:10FFE8000267964667DAA4FB046704FB05F34FF043
:08FFF800050C07EB4307DDE9EE
:020000040801F1
:100000000489A6FB0C230CFB07335F104FEA320672
:10001000B8EB06084FEA920669EB070946EA8376D1
:100020009F10DDE90023921B63EB0703DDE9026704
:10003000CDE90023344A4FF0FF33964277EB0303B8
:10004000CDE9048928DA40F6AC52A4184FF0000339
:100050005D4104FB05F3A4FB044505EB43056FF08C
:100060000602664202FB0566A4FB0223334418EB3A
:10007000020649EB0307CDE904670B26A4FB062320
:1000800006FB0533DDE900455B104FEA3202A41A96
:1000900065EB0305CDE900450AFB0BF3DDE90245FD
:1000A000AAFB0AAB0BEB430B4FEADA7242EA4B02B4
:1000B000A41A4FEAEB7365EB0305CDE90245DEF8C0
:1000C0000440009B019DA4FB032304FB05334FEA7E
:1000D00052584FEA635948EAC328DDE90423B8EBD4
:1000E000020269EB03039946D30B43EA494300B18B
:1000F000036009B1029B0B6007B0BDE8F08F00BF41
:100100007E0200205825002024FAFFFF7720482196
:100110000122FDF7B5BB772058210122FDF7B0BBC6
:1001200007B5002101AB03227720FDF72DFB9DF8D9
:1001300005309DF804001B0243EA00439DF80600C9
:10014000184303B05DF804FB08B5FFF7E9FF014B66
:10015000586008BD5825002008B5FFF7E1FF014BA6
:10016000186008BD5825002013B501220DF10703C2
:1001700004463A216820FDF707FB9DF8073003B1DC
:100180000123237002B010BD13B50622044643219B
:1001900068206B46FDF7F8FAA0B19DF800209DF8A5
:1001A000013043EA022323809DF802209DF80330AA
:1001B00043EA022363809DF804209DF8053043EA5A
:1001C0000223A38002B010BD13B5062204463B21D2
:1001D00068206B46FDF7D8FAA0B19DF800209DF885
:1001E000013043EA022323809DF802209DF803306A
:1001F00043EA022363809DF804209DF8053043EA1A
:100200000223A38002B010BD074B1B681869074B7F
:1002100020F01F0200F01F01D25801238B401A4228
:1002200001D0F6F7C9BF70477802002014040140DE
:10023000F0B52B4D2B7A85B0002B4ED1294C23687D
:10024000002B4AD01A68284E12B171690A437261B4
:100250009A88ADF80020022298688DF8032069463C
:1002600000228DF80220FDF779F9B3691D4F43F0A4
:100270000103B3612368187B197DF7F74DF82268F5
:10028000936894881B8A1C4002D001232B7224E0BF
:100290001648FDF711FE3B681869F6F78DFF3B68BD
:1002A0008DF80C401B69029308230DEB0300012617
:1002B0008DF80D308DF80E6000F0D2FE3B688DF8A1
:1002C00006405B7D8DF8043001A803238DF80530CE
:1002D0008DF8076000F0A6FED7E705B0F0BD00BFBF
:1002E0005825002078020020001002400902010871
:1002F00008B5FFF79DFF6B2180226820FDF7C0FA4B
:100300006420FDF72AFD6B2103226820FDF7B8FA6F
:100310000F20FDF722FD124B19211A786820FDF7F6
:10032000AFFA0F20FDF719FD0E4B1A211A7868203D
:10033000FDF7A6FA1B2118226820FDF7A1FA1C215F
:1003400010226820FDF79CFA372102226820FDF771
:1003500097FA682038210122BDE80840FDF790BADD
:10036000AC0200200000002008B5FFF761FF074B3A
:100370001B7813B1012B03D008BD4FF4006201E0DC
:100380004FF48052024B1A8008BD00BF7C0200204F
:10039000200000202DE9F0410369C76805460E469C
:1003A0001F40002F35D0B7FA87F24FF00043D340FB
:1003B000DB432B611F40A2F11B03042BF1D8DFE8C4
:1003C00003F0221F1C190300746A24B1013C0023AE
:1003D000A4B2736201E0EC6AA4B2D6F82080B8F14E
:1003E000000FDED0D8F80030404621469847D8F8B4
:1003F0000480F4E73068696B07E07068A96B04E07B
:10040000B068E96B01E0F068296C036889B298472D
:10041000C7E7BDE8F08107B52320FDF79EFC682003
:10042000752101220DF10703FDF7AEF928B19DF802
:100430000700A0F168035842584103B05DF804FB7F
:1004400001480249A6E700BF0048014060230020A0
:10045000014802499EE700BF0040014010230020F0
:100460000148024996E700BF00080040E82200204A
:10047000014802498EE700BF00040040C02200206E
:100480004FF08040004985E79822002010B5054CC8
:1004900005482146FFF77EFF04F1C8010348BDE887
:1004A000104077E770220020002C014000440140FA
:1004B000014802496EE700BF002C01407022002075
:1004C000224B10B5224C5A43224BB3FBF2F2038865
:1004D0000139013AA04289B292B29BB20ED004F522
:1004E0000064A0420AD0B0F1804F07D0A4F5983440
:1004F000A04203D004F58064A04202D123F070032F
:100500009BB2154CA04206D004F58064A0421CBFEB
:1005100023F440739BB203800D4BC1629842028565
:100520000FD003F5006398420BD003F54063984267
:1005300007D003F58063984203D003F580639842A7
:1005400001D1002303860123436110BD40420F0007
:10055000002C014000A24A040010004073B505467B
:100560000068FFF7ADFF2A6813889BB243F00103D0
:100570001380EB7A8DF804300124002601A88DF851
:1005800005408DF806608DF8074000F04BFDEB7AD2
:100590001B2B0BD1192301A88DF804308DF80540D1
:1005A0008DF806608DF8074000F03CFD02B070BD8C
:1005B000134B800A984220D00AD84A3B984212D066
:1005C0000133984211D0B0F5801F14D1012070473B
:1005D0000C4B98420BD0013398420AD0023B984210
:1005E00009D104207047022070470320704705207E
:1005F000704706207047FE2070470020704700BFFC
:100600004B00100051001000F8B504680646204663
:100610000F461546FFF7CCFF06284BD8B27A910853
:1006200047B902238B40D4F80CE0DB439BB203EACA
:100630000E03E3600A23204A03FB001342F82370F1
:10064000043342F8235015463FB1B17AE268890875
:1006500002238B409BB21343E360282202FB00522B
:100660002032EFF31286502383F3128803B203EB98
:100670008303DB0003F10C011C3329442B4451F8A4
:10068000047F17B117600A6804329942F7D100233A
:100690001360F3B283F31188282303FB0050036A2D
:1006A0001BB1E36843F0010303E0E2684FF6FE7319
:1006B0001340E360F8BD00BF702200200148F8F746
:1006C000ADBF00BF642500200148F8F7A7BF00BFF9
:1006D000B82500200148F8F7A1BF00BF0C26002074
:1006E00010B54B88DC0641BF2F4B14791B6853F8BB
:1006F000244044BF2D4B43F820404B889B0641BF0C
:10070000294B54791B6853F8244044BF274B43F8C6
:1007100020404B881C070ED5254B0C781B78B3EB7B
:10072000141FA1BF204BD4781B6853F82440A4BFEA
:100730001E4B43F820404B889B070ED51D4B0C7871
:100740001B78B3EB141FDFBF174B54781B6853F8AB
:100750002440DCBF154B43F820404B88DC070FD505
:10076000154C0B78247803F00F03A342DFBF0E4B28
:1007700014781B6853F82440DCBF0C4B43F820402E
:100780004B885B070FD50B780C49097803F00F03F2
:100790008B42A1BF044B92781B6853F82220A4BF60
:1007A000024B43F8202010BDD8200020220E00204C
:1007B0008F2000208D2000208C2000208E20002003
:1007C000254A264826490023F0B5156803700B70AA
:1007D0001C461A462E1976884EB92F5D3FB9037014
:1007E00000230A704B7007781C461A460CE0360549
:1007F00048BF013204F1040403F1010348BFD2B23F
:10080000802CDBB2E6D1EAE7E0B2B8420CD215F8B0
:10081000240006099E4200F00F00A8BF731C9042FE
:10082000A8BF421C0134EFE78A704B70C2F3470146
:1008300002F001020A444C1E0A490B480A70C3F335
:10084000470203F00103134404700849501E084A8C
:1008500008701370F0BD00BFB41000208420002089
:10086000602600208E2000208C2000208F20002079
:100870008D2000202DE9F04FC24BDA682DED028B60
:100880001A61C14A1168D960C0490B6843F020035E
:100890000B60BF4B1978012990460CBF0022012242
:1008A0001A70BC4B1A78910789B040F13D83BA4960
:1008B0000978042940F23883B849097801F0040125
:1008C00001F0FF0011B922F001021A701B78DB075A
:1008D00002D408B1F7F7A4FDB149CA78531C052228
:1008E00093FBF2F202EB82029A1AAE4BCA701B78AB
:1008F000039392000023AC4CDFF8CCC2DFF8D8920F
:100900005CF8231091FBF9F504F1080004F11006DE
:1009100040F82350A54844F8231000FB051142F28B
:10092000107091FBF0F080B226F813004FF0140E17
:1009300004F1140604F13C0A0EFB036E5AF823601E
:100940005EF802704EF80210F61B314444344AF847
:100950002310052691FBF6F109FB051144F823103D
:10096000039C012C4FEA830BE24605D10238B0F517
:10097000797F98BF4BF80C100BB90123BBE7884C6B
:10098000D8F80030226D9FED8A7A8A4E8A4D9B1AE4
:1009900007EE903AF8EE677AD8F800302365C7EE94
:1009A000877A7C4B1B78B7EE008AF4EEC87AF1EEBA
:1009B00010FA58BFF0EE487A13F00103C4ED157A2F
:1009C00012D005AA00927D4B06AA01920CCB9AE8A0
:1009D0000300F7F723FC6421059A069BB2FBF1F2B2
:1009E00093FBF1F3328000E033802B8094F8583091
:1009F0006B48002B3BD0D0ED157AC26DDAF8003091
:100A0000C8EE276A9B1A026E022507EE103AB8EE6E
:100A1000C77ADAF8043027EE267A9B1AFDEEC77AF9
:100A2000B0F9662017EE901A07EE903A644BB8EED4
:100A3000E77AD3ED007A67EE277A67EEA67AFDEEC5
:100A4000E77A17EE903A02FA83F3B0F9642093FB49
:100A5000F5F302FA81F29BB292FBF5F292B2A0F8A2
:100A60006A30A0F86820A0F86630A0F8642001235E
:100A700084F85830534BDAF804101B88DAF8000079
:100A8000474D514E216603F03003E065002B00F026
:100A90004B8205F17403009305F178030193EA6E2C
:100AA0002B6FF7F7BBFB72682B6F9B1A07EE903A20
:100AB000434B326893ED007AEB6EF8EEE77A9B1ABF
:100AC000EB67384B67EE877A1B78FDEEE77A012BF0
:100AD000C5ED207A03D0022B00F0DF8024E2D5EDB3
:100AE000287A3A4BD5ED215A95ED255A95ED156AA0
:100AF00095ED264AD5ED274A35491D68B1EE677A4E
:100B0000BDEEC77AFDEEE77A17EE10EA17EE90CA4F
:100B10000020304A91ED007A52F8207007EE907A6A
:100B2000F8EEE77AA2F1140367EEA57A33F81060C5
:100B3000FDEEE77A283217EE903A9B1B9BB222F823
:100B400010301BB207EE903AF8EEE77A3B4467EEBE
:100B5000857A4400FDEEE77ACDED037A07EE903A10
:100B6000F8EEE77ABDF80C8067EE847AA7EE867A15
:100B7000FDEEC77A17EE902A724531DB6245A8BFB9
:100B800062462EE090070020602700201C11002004
:100B90005A100020201100202611002022340020AD
:100BA000602600205C0F002064260020806967FF1B
:100BB00000007A449A1100209C1100205C10002053
:100BC00078000020E011002028110020600F002094
:100BD000900F0020DC26002080969800DB0FC94093
:100BE000724607EE902AF8EEE77A5FED046AC1EDEF
:100BF000007AFDEEE77A313617EE903A43449AB226
:100C0000AB78D1ED027A07EE103AB8EE477A4B682E
:100C10004F6027EE267AFB1A88EE077AB6B2622E6C
:100C200006EE903AF8EEE66A37EE067AC6EE866A87
:100C300086EE077A76EEE76AE7EE267AC1ED047A69
:100C4000C1ED027A0FD964EEA77ABA4EFDEEE77ACB
:100C500017EE903AB3F5FA6FA8BF4FF4FA63B342B8
:100C6000B8BF334600E0002313441BB240F6B8324D
:100C70009342A8BF1346B04A9342B8BF1346AF4A47
:100C8000A352AF4A142303FB002351F8142B1A601C
:100C9000002840F0498101203BE7AA4BD5F8748039
:100CA0001F68D4F878903E89DFEDA78A4FEA580391
:100CB0009E4228BF1E46B5F8A8301AB29642C3BF5E
:100CC000D5ED157A9FEDA17A67EE877AB6B2C1BFEE
:100CD000FDEEE77A17EE906AF618B6B2C8BFA5F82F
:100CE000A860D4F8AC50C5EB09052846F7F7DAFA46
:100CF0000028D8BF404241F293129042CCBF00205E
:100D0000012088B307EE905AB8EEE70A20EE280AD1
:100D1000FAF703F807EE908AF8EE677A40F6B833F0
:100D200020EE270AFDEEC07ACDED037ABDF80C2047
:100D3000A4F8B02012B29A42A8BF1A467E4B9A423B
:100D4000ACBF09EB02034B4448F6A042934203DDDB
:100D5000A3F50C43A03B04E0002BBCBF03F50C4300
:100D6000A033C4F8B43001E0C4F8B490D4F8B4505F
:100D7000C5F50C53283307EE903AF8EEE77A67EEA4
:100D8000A88AB0EE680AFAF72BF88DED070AB0EEE4
:100D9000680AF9F7C2FFD4ED317AD4ED2E4AD4EDCA
:100DA000155A94ED2F4A94ED305A65498DED060A97
:100DB000B1EE677ABDEEC77AFDEEE77A0DF1180E57
:100DC00017EE10AA17EE90BA0020614AFEEC016AF5
:100DD00032F91030DFF88C9107EE903A07EE106A86
:100DE000F8EEE77AB8EEC77A3C32D6EE877A4FEA69
:100DF000400CFDEEE77ACDED037ABDF90C30B3F58A
:100E00007A7FA8BF4FF47A734B45B8BF4B461FFAA1
:100E100083F922F810900FFA89F207EE902AF8EE83
:100E2000E77A27EEA47ABDEEC77A8DED037A27EE36
:100E3000847AD1ED007ABDF80C90E7EE257AFDEECC
:100E4000E77A17EE902A524503DB5A45A8BF5A4667
:100E500000E0524607EE902AF8EEE77A9FED3D6AF1
:100E6000C1ED007ABA7891ED027A06EE902AF8EE9A
:100E7000666A4A684B6066EE866A9A1AC8EE266A07
:100E8000143106EE102AB8EEC66A76EEA56A86EE32
:100E9000256AC5EEA66A36EE476AA6EE867A01EDA9
:100EA000017A01ED037A25EE077ABDEEC77A17EED7
:100EB000103ABDEEE77A4B4417EE102A13441BB2EA
:100EC00040F6B8329342A8BF13461B4A9342B8BFBC
:100ED00013461A4A2CF802301F4A142303FB00233E
:100EE000C3ED007A08B901206FE73B7923B1642391
:100EF00095FBF3F5194B1D803B8898450DD9D4F827
:100F0000AC30A06FC01AF7F7CDF980EAE072A2EB1F
:100F1000E07242F210739A4206DD114B01221A7000
:100F20000E4BB4F8C8201A8009B0BDEC028BBDE8A6
:100F3000F08F00BF30F8FFFF48F4FFFFE40F002000
:100F4000B80F0020600F0020D30237390000C842DC
:100F5000C8260020DB0FC940900F0020580F00204A
:100F60005C0F002018FCFFFF40F2E9330F4A1289A2
:100F7000920704D4013B9BB2002BF7D10BE00C4A43
:100F800040F2E933107009490989C9070AD4013BC5
:100F90009BB2002BF7D1074A138801339BB2138011
:100FA000FF2070471078C0B2704700BF0038004083
:100FB0000C3800402C27002030B5174B9B894FF48C
:100FC0007A733AB311B10D78013107E0FF2505E0DE
:100FD000013B9BB24FF6FF74A3420FD00E4C248905
:100FE000A407F5D50D4C25700B4D2D89ED070BD4BD
:100FF000013B9BB24FF6FF75AB42F5D1084A13880F
:1010000001339BB2138005E0247808B104700130ED
:10101000013AD6E7012030BD003800400C380040CE
:101020002C2700200C4B0D49DA684378D243C2F3D9
:101030000222C2F10402934002781B010A44DBB28F
:1010400082F8003303780122580903F01F0302FAE3
:1010500003F341F82030704700ED00E000E100E0CC
:10106000036823F01F0202F1804202F5823270B55C
:1010700003F01F011468012303FA01F124EA0101BE
:10108000116002682A4C22F01F0502F01F02295944
:1010900003FA02F221EA02022A510279016802F1FE
:1010A000804221F01F0402F5823201F01F01155920
:1010B00003FA01F12943115102681E4D22F01F0469
:1010C00002F01F02615903FA02F221EA02026251A0
:1010D0000268194C22F01F0602F01F02315903FA70
:1010E00002F221EA0202417932511029026812D13A
:1010F00022F01F0102F01F024E5903FA02F232439E
:101100004A51026822F01F0102F01F020859934061
:1011100003430B5170BD01F1804122F01F0001F526
:10112000823102F01F020C58934023430B5070BDD4
:1011300004040140080401400C040140F0B5BB4C1C
:10114000A3782DED028B013B012B85B000F26A8163
:10115000E578854240F066812379022B00F06281B8
:10116000B34B5B5D6371A3796D00F2EE048A1BB132
:101170006319B3F9083009E06319D4ED037AB3F9C0
:101180000830F1EE677AC4ED037A5B4208EE103A5C
:101190002369A64EB8EEC88A1A0388EE288A35D588
:1011A000D6ED037AFDEEE77A28EE280A17EE903A9C
:1011B000D6ED057A8DF80A30FDEEE77A17EE903A13
:1011C0008DF80B3005F04EF9FCEEC07A96ED060A6C
:1011D00017EE903A20EE280AADF8083005F042F9F3
:1011E000FCEEC07A96ED070A17EE903A20EE280A38
:1011F000ADF80C3005F036F9FCEEC07A0C2017EE95
:10120000903A02A9ADF80E30FAF73CFDD4ED077A1A
:10121000864BF5EE407AF1EE10FA60D1D3ED067A06
:10122000B4EEE78AF1EE10FA04DDDA6883ED068A9F
:101230005A61E8E0F5EEC07AF1EE10FA40F3E3808F
:1012400093F8202042B1022A00F2DD805A6B83ED30
:10125000078AFA329A63D6E0D3ED037A38EE678ACA
:10126000F7EE007AB4EEE78AF1EE10FAACBF012196
:101270000021D3ED0A7A69B19FED6E7A27EE877A65
:10128000DFED6D7AB4EEE77AF1EE10FA58BFF0EECA
:10129000477A03E09FED697A67EE877AC3ED0A7AB1
:1012A0002369624A1B0311D58DF808105379116B1D
:1012B0000B440B205A788DF80920DA7A8DF80A2031
:1012C0005B7D8DF80B3002A9FAF7DCFC0123226B61
:1012D00084F82030637913440022DA7291E0B4EE8E
:1012E000E78AF1EE10FA48BF83ED078AA16B636BC2
:1012F00094ED067AD4ED076A591AC943C90F77EEFF
:10130000667A59B9B7EE006AF4EEC67AF1EE10FAD1
:1013100079DDB4EEE68AF1EE10FA74DDD4ED056AFB
:10132000424BB4EEE67AF1EE10FACCBF012600266D
:1013300066B1D3ED097A9FED3F7A67EE877A9FED2C
:101340003F7AC3ED097AD3ED0B7A0AE0B0EE007A6A
:10135000F4EEC77AF1EE10FA08DDD3ED0B7A9FEDCB
:10136000357A67EE877AC3ED0B7A07E0D3ED097A19
:101370009FED327A67EE877AC3ED097AD4ED097A68
:10138000206B627967EEA87A1044FCEEE77ACDED27
:10139000017A9DF804304370D4ED0B7A2769FCEE96
:1013A000E77A3F03CDED017A9DF8042042750ED512
:1013B00046EA41018DF808108DF80930C37A8DF89E
:1013C0000A300B2002A98DF80B20FAF75BFC94F889
:1013D0002020164B022A11D1D3ED0A7A9FED187AFC
:1013E000196B67EE877A002283F82020FCEEE77AFB
:1013F0005A7917EE903A0A44D37202E0022283F837
:101400002020F7F78BF82544F7F730F8B5F90830C6
:10141000D4ED037A00EE103AB8EEC00A80EE280A46
:1014200037EEC00A05B0BDEC028BF0BD2C270020C2
:10143000BCA40108EC51783F6F12833A0AD7833F6E
:1014400000007A442B4BF0B52B4D1E6805F11000BF
:101450002F78F3192C46597801F00401013501F079
:10146000FF0219B18542F3D10020F0BD224D631B6C
:10147000022B0ADD1AB102EB82025200D2B215F839
:10148000013B303B1A44D2B2F1E70021AC420AD909
:1014900019B101EB81014900C9B215F8013B303B9C
:1014A0001944C9B2F2E72E2F16D1013404200023CB
:1014B0002578771903EB83037F785B007F079BB266
:1014C00044BF303D5B1900F1FF3044BF01349BB293
:1014D00010F0FF00ECD100E00023084841436420F5
:1014E00000FB03130620B3FBF0F3054800FB0230BA
:1014F000F0BD00BF8C0000206827002040420F0094
:101500008096980030B500231A4610498C1894F83C
:101510003C40BCB12E2C06D1013298B18C18044449
:10152000002584F83C5011440A2491F83C10634390
:10153000A1F13004092C9CBF303B5B180E2A03D864
:101540000132E2E7184630BD002030BD2C270020D4
:10155000104B10B50446185CF9F73FF80E4800EB45
:101560004400B0F94C10B1F57A7F05DBB1F5FA6FA4
:10157000A8BF4FF4FA6101E04FF47A71A1F57A71D6
:101580000A23092091FBF3F1BDE81040C9B2F9F735
:1015900085BF00BF2DC301082C270020031EB8BF44
:1015A0002D2210B5B8BF58420C46B8BF01F8012B28
:1015B0000A22F9F76DFA00230370204610BD0B4A8A
:1015C000136913F4805FB2F9523006D0B2F80622E4
:1015D000111A8B4208DD104401E0B2F80802834280
:1015E000B4BF002001207047012070472C27002045
:1015F0000F4B1A78682A17D1598840F2D472914259
:1016000012D11A79BE2A0FD193F8D127EF2A4FF0C1
:1016100000000BD113F8012B5040064A9342F9D138
:10162000B0FA80F04009704700207047704700BF53
:1016300000F80308D4FF03082DE9F04F2DED028BCD
:10164000EB4C85B0002140F2D472204604F0B5FC8A
:10165000E84B04F538721A60E74B00251D70E74B24
:1016600004F2AA721A6068232370022003236371B4
:10167000F9F782FC4FF48070F9F77EFC4FF4167393
:101680002022A4F8663184F86A21FA236E22A4F895
:10169000683184F87A212A230A22A4F8643184F874
:1016A0007B214FF4FA732B22A4F86C3184F87D214E
:1016B0000123212284F8623184F87C3184F87E2170
:1016C00084F884312322002384F87F21C4F8143263
:1016D0004FF4C872C4F818320523A4F8802184F8A6
:1016E000A857A4F87051A4F86E51A4F8725184F868
:1016F000585184F8595184F85A51A4F85C51A4F80F
:101700005E51A4F8605184F8635184F86B51A4F8D9
:101710008251A4F8865184F8115284F8105284F84A
:101720001C5284F81D5284F81F3240F2DC53A4F896
:10173000963140F24C43A4F8983140F26C73A4F80F
:101740009A3140F27533A4F89C3140F64303A4F873
:101750009E3184F81E5284F8905184F891512A46A3
:1017600023469918023200254FF01E0A1C2AA04C6D
:1017700081F8A05181F8A1A1F3D140F27E4140F25D
:101780007E5EDFF870B2A4F84411052340F23A718E
:10179000A4F84CE140F2EA5E01264FF47A774FF468
:1017A000FA68C82219204FF0320984F8D431A4F81D
:1017B00046114FF4C87340F2DC51A4F84EE140F2F8
:1017C000B45EA4F8D821029284F8D5010390A4F85D
:1017D000DC31A4F84A110191A4F850E184F893A1F6
:1017E000A4F8BE81A4F8C281A4F8C681A4F8CA8175
:1017F00084F8D36184F8D66184F8D76184F8DA611B
:1018000084F8E06184F8925184F89451A4F8BC7192
:10181000A4F8C071A4F8C471A4F8C87184F8CC51BC
:1018200084F8D25184F8DE51A4F84871A4F852919A
:10183000A4F8543184F8E361A4F8569184F8E15196
:1018400084F8E25184F8E451F5F722FCDBF800302B
:1018500026744FF00F0CE673A4F80C80A57383F880
:1018600005C04FF0220C83F806C00398D8714FF0E2
:101870000E0C4FF0170E83F810C021204FF0350CDE
:1018800083F815E083F816E083F81AC058744FF017
:10189000550E53204FF0640C4FF0280883F80BA02E
:1018A00083F80CA083F803E0D8764FF02D0E5A2071
:1018B00083F81CC04FF00A0A4FF0780C83F80DE053
:1018C000187283F80AC01D7083F8018083F80280C3
:1018D000DD7583F804909D731D76DD735D7683F866
:1018E00012A083F8098083F814E04FF4FA7EA3F87D
:1018F0004EE0DFF820E1C3F838E0C3F83CE0DFF861
:1019000018E1C3F828E04FF07E5EC3F834E0DFF85A
:101910000CC1DFF80CE19FED3A8AC3F82CC0C3F884
:1019200030C0C3F848E0F7EE087ADFF8F8C0019954
:101930009E774FF04B0E83F8525083F8515083F846
:101940005050C3ED087AC3ED097A83ED108AC3F8CD
:1019500044C083F84CE084F8AA07A4F8B4174120E7
:10196000042184F8AB0784F8AC9784F8AD5784F869
:10197000B15784F8B25784F8AE5784F8AF5784F85B
:10198000B05783F85C101521A3F85850A3F85A50AB
:10199000A3F85650C3F860C083F8648083F86810D9
:1019A0001849D966184919671849596783F8786042
:1019B00083F865801648F5F7A9FBDBF80030029A3A
:1019C00083F814614FF44871A3F8161183F811518C
:1019D00083F8125183F8138183F81851194684F85B
:1019E000CEA184F8CF21A4F8D0715E461CE000BFE0
:1019F0009C2700202C100020E02400205410002000
:101A0000000000009A99193FF6287C3F3D0A773F75
:101A100042C301088FC2F53C00002040CDCCCC3E33
:101A2000000040400000A0400E2202FB05326FF093
:101A3000170082F81901032082F81A016FF02F00B5
:101A400082F81B01072082F81C016FF0230082F846
:101A50001D01052082F81E0101355A2081F8200160
:101A600081F821016422FF20082D81F81F2181F8CF
:101A7000220101F10E01D7D1002183F88911C8217B
:101A8000A3F88A11142183F88C11A3F890211E2148
:101A90004FF4967283F88D11A3F892210121282228
:101AA000A3F8942183F88E112F4B03F1C0021F4637
:101AB00083ED058A10339342FAD12C48002140224D
:101AC00004F07BFA00232A4D274C5959FA180433A5
:101AD0000868C2F8A002382BF5D104F5087000217F
:101AE000802204F06AFA05F13801702204F50870CA
:101AF00004F058FAFEF764FE4FF40020F9F73CFAC0
:101B000036680125314604F58F604FF4CC7284F8B5
:101B1000D05784F8CE5784F8CF5704F043FA04F531
:101B2000C26031464FF4CC7204F03CFA114B1B6892
:101B30001A68C4F8B6275A68C4F8BA279A68C4F86D
:101B4000BE271A68C4F8C2275A68C4F8C6279A681C
:101B5000C4F8CA27022384F8CC5484F8643605B04C
:101B6000BDEC028BBDE8F08F9C2700203C2A0020B2
:101B7000C0A40108541000201549D1F8883043F45E
:101B80007003C1F88830134B1A6842F001021A60E2
:101B90005868114A02405A601A6822F0847222F48E
:101BA00080321A601A6822F480221A605A6822F47D
:101BB000FE025A60DA6A22F00F02DA62186B074AF4
:101BC00002401A6300229A604FF000638B607047F6
:101BD00000ED00E0001002400CC07FF8CCFC00FFDC
:101BE000074B93F8D037012B08D1064A064BD06833
:101BF0001B68834234BF00200120704700207047DB
